:100000000C944E210C947F210C947F210C947F2121
:100010000C947F210C947F210C947F210C947F21E0
:100020000C947F210C947F210C947F210C947F21D0
:100030000C947F210D94DA3C0C947F210C947F2149
:100040000C947F210C94C0350C947F210C947F215B
:100050000C947F210C947F210C9481320D94903C60
:100060000C947F210C946EA60C9464A60C947F21B2
:100070000C947F210C947F210C947F210C947F2180
:100080000C94E3910C947F210C947F210C947F219C
:100090000C947F210C947F210C947F210C947F2160
:1000A0000C947F210C947F210C94B5910C947F21AA
:1000B0000C947F210C947F210C947F210C947F2140
:1000C0000C947F210C947F210C947F210C947F2130
:1000D0000C947F210C947F210C947F210C947F2120
:1000E0000C947F21084AD73B3BCE016E84BCBFFDF8
:1000F000C12F3D6C74319ABD56833DDA3D00C77FF8
:1001000011BED9E4BB4C3E916BAAAABE0000008090
:100110003F05A84CCDB2D44EB93836A9020C50B91F
:10012000918688083CA6AAAA2ABE000000803F004B
:100130000C94A7EC0C941DD20C9403DA0C946DD49F
:100140000D94E91B0C9466D90C944B2A0D94E73658
:100150000C944BD60C9486F30C94E0230C94D4327C
:100160000C9499270C94696E0D94284F0C94BE251D
:100170000C94B9EC0C943C260C9423290C94E26367
:100180000C94DEA60D9497350D944F190C9469D4F8
:100190000C94A6A60C94CBEC0D948C360C944E26A5
:1001A0000C9418DB0D94D3360C9416E60D9461353F
:1001B0000D946B360C945AD60C946F2A0C9464E30D
:1001C0000C9456230D9466350C94502A0C94C62436
:1001D0000C94C5EC0C94F2D90C94C1D90C9413A7CF
:1001E0000C94A96C0C9406DA0C947B260C94E9EC24
:1001F0000C9430D30C9417DA0C94CAF70C9472E672
:100200000C94A4280C943C2A0D94BA360C943E25E8
:100210000C94EFEC0C9464D20C941CDA0C9462D61F
:100220000C94BD230C9496D20C940CA70C94CCFD8A
:100230000C944ED40D9453110C940FDA0C9453E695
:100240000D94B7350C94CFD10D9478350D947C3541
:100250000C942DD40D94D64E0C94EDA60C947DD216
:100260000C9471D90C9454DB0C941CE20C9404EFA4
:100270000C9465D40C94F1280D9496360C940AE6EF
:100280000C94CFA60C9478DA0C9451D20C9467D8C5
:100290000C941FDA0C94C8930C941EA70D94464F2F
:1002A0000C941EE60C9473EE0C9416D30C948F6190
:1002B0000C9412E60C94F7D10C940EE60D945019A0
:1002C0000D94B0360C9497280C94D2FB0D94FC0935
:1002D0000D9473360C94F7D50C9464910D945B03D4
:1002E0000D949B350C9400DA0C94737A0C9438D2EC
:1002F0000C9422E60C9426A70C943C290D94053707
:100300000C9468CF0C9493DA0C948ED10C94C22A7E
:100310000C940A290C94DDEC0C9473D80D94AD3533
:100320000C9409DA0C94EB230C9481CF0C941AE60C
:100330000D94A9350C9400A70D9491350C943BE2D3
:100340000C94D7EC0C9480EB0C945F250C945CD649
:100350000C949C280C94FFD20C9400890C94E8D146
:100360000C94CAD90C94A3250C94FCE30D94783614
:100370000C9488D40C9449910D94C8080D94893D2F
:100380000C942A240C949DDA0C9433D60C942AE60F
:100390000C94D8630C9474D50C94B3EC0D94F13692
:1003A0000C94C5E20C949B270D94A5350C94032264
:1003B0000C9481210C9460D60C94ADEC0C9404A7A1
:1003C0000C942EE60C94A6ED0C94412A0C9442D683
:1003D0000C94DD630C9461D40C949A910C9466D6C1
:1003E0000C94A5D20C9468D60D948D350C9408A766
:1003F0000C9419DA0C94B0F00C94D1D20D94F3351E
:100400000C94E8D20D944A060C940CDA0C944CF53A
:100410000C9445270C9464D60C94462A0C94DBE18A
:100420000C94E3EC0D94EF060D9484350C94FCA62B
:100430000D9480350C94A9240D9487350D945C019E
:100440000C94BFEC0D9479040C94BB6A0C940AD202
:100450000C9441290C94B8D20D948B050D9406365A
:100460000D949F350C948ED40C94F4A60C94BCE19E
:100470000C94D1EC0C94D8280D949E360C94FDD994
:100480000C94A26F0C94A2D60D9442190C9432E6EF
:100490000C94F8A60C9426E60C942DD30D94DD361E
:1004A0000D9482360D94C4360C9465D50C94B6F632
:1004B0000D94A6360D94FB360C945ED60C947F9169
:1004C0000C94B0D50C94C0D10D94B3350C9412DAC1
:1004D0000C9423D50C9475DA0C94A7D10D941519AE
:1004E0004E414E494E495459494E46CDCCCC3D0A19
:1004F000D7233C17B7D13877CC2B329595E6241FFC
:10050000B14F0A000020410000C84200401C4620B4
:10051000BCBE4CCA1B0E5AAEC59D7400407A10F387
:100520005A00A0724E18090010A5D4E80000E87621
:1005300048170000E40B54020000CA9A3B00000078
:10054000E1F505000080969800000040420F000091
:1005500000A08601000000102700000000E8030052
:100560000000006400000000000A0000000000011C
:1005700000000000002C76D888DC674F0823DFC11C
:10058000DFAE59E1B1B796E5E3E453C63AE65199D7
:100590007696E8E6C28426EB898C9B62ED407C6F00
:1005A000FCEFBC9C9F40F2BAA56FA5F490055A2AB7
:1005B000F75C936B6CF9676DC11BFCE0E40D47FEC3
:1005C000F520E6B500D0ED902E03009435770500B8
:1005D00080841E080000204E0A000000C80C33333F
:1005E00033330F986E12831141EF8D2114893BE64E
:1005F0005516CFFEE6DB18D1844B381BF77C1D90D7
:100600001DA4BBE424203284725E228100C9F1243F
:10061000ECA1E53D2741425300504C41003F0053BF
:1006200074617274205072696E740043616E636508
:100630006C005072696E740043616E6E6F74206559
:100640006E746572207375626469723A2000052EBB
:100650002E004D61696E002100486F74656E642044
:10066000746F6F20636F6C64004261636B00507243
:100670006F6365656400536F667420456E647374C0
:100680006F7073004D6F74696F6E004469736162BF
:100690006C65205374657070657273004D3834005A
:1006A0004D34382050726F62652054657374004772
:1006B00032384F0A4D343820503130004C65766561
:1006C0006C20436F726E65727300466164652048EA
:1006D0006569676874004F6666004F6E0042656426
:1006E000204C6576656C696E67004C6576656C209C
:1006F000426564004732394E00486F6D65205A00EC
:100700004732385A00486F6D6520590047323859D2
:1007100000486F6D652058004732385800417574A5
:100720006F20486F6D6500473238004D61696E007B
:1007300050726568656174202420456E64005072B3
:1007400065686561742024204265640054656D709D
:10075000657261747572650019061506436F6F6CDA
:10076000646F776E0050726568656174202400467E
:10077000616E205370656564207E00426564004EA2
:100780006F7A7A6C65004D61696E0050726F6265B8
:10079000205A204F666673657400416476616E630B
:1007A00065204B00466C6F770046616E2053706584
:1007B0006564207E00426564004E6F7A7A6C650045
:1007C0005370656564004D61696E00486F6D696EB8
:1007D00067204661696C6564006F70656E005452F5
:1007E00049474745524544003A20007A5F6D696E9B
:1007F00000795F6D696E00785F6D696E005265709B
:100800006F7274696E6720656E6473746F702073A5
:1008100074617475730A0020746F6F206C6F6E675B
:1008200020657874727573696F6E20707265766575
:100830006E7465640A0020636F6C6420657874725E
:100840007573696F6E2070726576656E7465640A83
:1008500000486F6D652025732573257320466972E6
:100860007374005761726E696E673A20486F6D69E4
:100870006E672042756D702044697669736F7220CF
:100880003C20310A000202040000000000000000C9
:100890000000000000006643000061430000964332
:1008A000000000410000004100000040FFFFFF0089
:1008B00000000100000001000080005555550000B7
:1008C00000400033333300AAAA2A004992240000D2
:1008D000002000C7711C0099991900D145170055D7
:1008E0005515003BB11300244912001111110000ED
:1008F0000010000F0F0F00E3380E0043790D00CCFD
:10090000CC0C00C3300C00E8A20B0064210B00AA41
:10091000AA0A00703D0A009DD80900427B09009296
:10092000240900DCD3080088880800104208000071
:10093000000800F0C10700878707007550070071A5
:100940001C07003EEB0600A1BC060069900600668D
:10095000660600703E06006118060017F405007474
:10096000D105005BB00500B290050062720500552C
:1009700055050078390500B81E0500050505004E2F
:10098000EC040087D40400A1BD040090A704004932
:10099000920400C17D0400EE690400C756040044BF
:1009A0004404005C320400082104004110040000EB
:1009B0000004003FF00300F8E0030026D20300C368
:1009C000C30300CCB503003AA803000A9B03003818
:1009D0008E0300C08103009F750300D0690300509F
:1009E0005E03001D53030034480300913D030033B0
:1009F00033030016290300381F0300971503003046
:100A00000C0300030303000BFA020049F10200BAD1
:100A1000E802005CE002002DD802002DD00200594F
:100A2000C80200B0C0020031B90200DAB10200AA67
:100A3000AA0200A0A30200BC9C0200FA9502005C7E
:100A40008F0200DF88020082820200457C020027BC
:100A500076020027700200436A02007C640200D024
:100A60005E02003F590200C8530200FFFDFCFAF885
:100A7000F6F4F2F0EEECEAE9E7E5E3E1E0DEDCDAF9
:100A8000D9D7D5D4D2D0CFCDCBCAC8C7C5C3C2C0A1
:100A9000BFBDBCBAB9B7B6B4B3B2B0AFADACAAA91A
:100AA000A8A6A5A4A2A1A09E9D9C9A99989795946A
:100AB0009392908F8E8D8B8A89888786848382819A
:100AC000807F7E7D7B7A79787776757473727170AA
:100AD0006F6E6D6C6B6A696867666564636261609E
:100AE0005F5E5D5C5B5A5958585756555453525186
:100AF00050504F4E4D4C4B4A4A4948474646454454
:100B000043424241403F3E3E3D3C3B3B3A39383810
:100B100037363535343332323130302F2E2E2D2CBE
:100B20002B2B2A2929282727262525242323222160
:100B30002120201F1E1E1D1C1C1B1B1A19191818F2
:100B4000171616151514131312121111100F0F0E7C
:100B50000E0D0D0C0C0B0A0A0909080807070606FA
:100B600005050404030302020100000000664300BF
:100B700000614300009643000000000000000000F8
:100B800000000053657474696E67732053746F724C
:100B9000656400454550524F4D20496E6974696146
:100BA0006C697A65640A003B20003A0A0020204DF7
:100BB00036303320002055004C0046696C616D656D
:100BC0006E74206C6F61642F756E6C6F6164206C45
:100BD000656E677468733A0020204D393030204BC1
:100BE000004C696E65617220416476616E63653A9E
:100BF0000020204D3835312058005A2D50726F6238
:100C000065204F66667365740020204D34313320B3
:100C10005300506F7765722D4C6F7373205265636C
:100C20006F766572793A0020440020490020204DFB
:100C300033303420500020440020490020204D3320
:100C400030312050005049442073657474696E67D8
:100C5000733A0020460020480020204D31343520D2
:100C600053004D6174657269616C206865617475CB
:100C70007020706172616D65746572733A00204A0C
:100C8000002020473239205720490020204D34329F
:100C9000302053004175746F20426564204C6576A6
:100CA000656C696E673A0020204D3230362058005E
:100CB000486F6D65206F66667365743A0020580052
:100CC00020530020204D32303520420041647661AF
:100CD0006E6365643A20423C6D696E5F7365676D53
:100CE000656E745F74696D655F75733E20533C6D0E
:100CF000696E5F66656564726174653E20543C6D23
:100D0000696E5F74726176656C5F66656564726159
:100D100074653E20583C6D61785F785F6A65726BE0
:100D20003E20593C6D61785F795F6A65726B3E2049
:100D30005A3C6D61785F7A5F6A65726B3E20453C14
:100D40006D61785F655F6A65726B3E0020540020BC
:100D5000520020204D323034205000416363656CD6
:100D600065726174696F6E2028756E6974732F7374
:100D700032293A20503C7072696E745F616363651A
:100D80006C3E20523C726574726163745F61636390
:100D9000656C3E20543C74726176656C5F61636380
:100DA000656C3E0020204D3230312058004D617876
:100DB000696D756D20416363656C65726174696FFF
:100DC0006E2028756E6974732F7332293A002020C3
:100DD0004D3230332058004D6178696D756D206655
:100DE00065656472617465732028756E6974732F0C
:100DF00073293A0053746570732070657220756EA4
:100E000069743A0020440020204D323030205300D5
:100E10002044697361626C65640A0046696C616DA7
:100E2000656E742073657474696E67733A00202070
:100E30004D3134392043203B20556E69747320694D
:100E40006E2043656C736975730A0020286D6D29E7
:100E5000002020473231202020203B20556E69742D
:100E60007320696E206D6D0000803B4400803B4420
:100E700000002041000096420000A0420000A04275
:100E80000000C8430000BE42D0070000D0070000A9
:100E9000640000004B00000024F4D43050C38E20C6
:100EA000C2A24017828B7011127A910D816CD90AFF
:100EB000A861E108C7586607615143061E4B5D05EE
:100EC000C145A7041A411104093D98037139310342
:100ED0004036DB0265339102D4305402802E1D026D
:100EE000632CEE01752AC501B028A00110278101ED
:100EF0008F2564012B244B01E0223401AC211F011A
:100F00008D200D01801FFC00841EED00971DDF0069
:100F1000B81CD200E61BC600201BBC00641AB2003D
:100F2000B219A8000A19A0006A189900D1179100F7
:100F300040178B00B516840031167E00B31579007A
:100F40003A157300C7146F0058146A00EE13660058
:100F50008813630025135E00C7125B006C125700F4
:100F600015125400C111510070114F0021114B0096
:100F7000D61049008D104700461044000210420070
:100F8000C00F4000800F3E00420F3C00060F3B00A8
:100F9000CB0E3800930E37005C0E3500270E340060
:100FA000F30D3200C10D3100900D3000600D2E00A8
:100FB000320D2D00050D2C00D90C2B00AE0C290094
:100FC000850C29005C0C2700350C27000E0C260030
:100FD000E80B2400C40B2400A00B23007D0B23008E
:100FE0005A0B2100390B2100180B2000F80A1F00B2
:100FF000D90A1E00BB0A1E009D0A1D00800A1D00A2
:10100000630A1C00470A1B002C0A1B00110A1A0065
:10101000F7091A00DD091900C4091900AB09190004
:10102000920917007B091800630917004C09160084
:1010300036091600200916000A091500F5081500E2
:10104000E0081400CC081400B8081400A408140028
:10105000900813007D0812006B0813005808120056
:10106000460812003408110023081100120811006C
:1010700001081100F0071000E0071000D007100071
:10108000C0071000B0070F00A107100091070E0065
:1010900083070F0074070F0065070E0057070E0047
:1010A00049070E003B070D002E070E0020070D001C
:1010B00013070D0006070D00F9060C00ED060D00E4
:1010C000E0060C00D4060C00C8060C00BC060C00A0
:1010D000B0060C00A4060B0099060C008D060B0050
:1010E00082060B0077060B006C060B0061060A00F7
:1010F00057060B004C060A0042060A0038060A0092
:101100002E060A0024060A001A060A001006090024
:1011100007060A00FD050900F4050900EB050900B2
:10112000E2050900D9050900D0050900C705090035
:10113000BE050900B5050800AD050800A5050900B4
:101140009C050800940508008C050800840508002B
:101150007C050800740508006C050700650508009B
:101160005D050700560508004E0507004705070006
:101170004005080038050700310507002A0507006B
:10118000230507001C050600160507000F050700CC
:101190000805060002050700FB040600F504070029
:1011A000EE040600E8040600E2040700DB04060083
:1011B000D5040600CF040600C9040600C3040600D7
:1011C000BD040600B7040600B1040500AC04060027
:1011D000A6040600A00405009B0406009504050073
:1011E000900406008A0405008504050080040600BA
:1011F0007A04050075040500700405006B04050001
:1012000066040500610405005C0405005704050040
:10121000520405004D040500480405004304050080
:101220003E0404003A0405003504050030040400BF
:101230002C04050027040400230405001E040400F8
:101240001A04040016040500110404000D0404002F
:10125000090405000404040000040400FC03040065
:10126000F8030400F4030400F0030400EC0304009A
:10127000E8030400E4030400E0030400DC030400CA
:10128000D8030400D4030400D0030400CC030400FA
:10129000C8030300C503030024F404D9201BC40CB5
:1012A0005C0E9804C4095F0265077101F405F9003A
:1012B000FB04B30048048700C103690058035500CC
:1012C00003034500BE023A008402310053022A00A3
:1012D0002902250004022000E4011C00C8011900B5
:1012E000AF01170098011400840113007101100070
:1012F0006101100051010E0043010D0036010B0089
:101300002B010B0020010B00150109000C01090045
:1013100003010800FB000800F3000800EB000700D1
:10132000E4000600DE000600D8000600D200060039
:10133000CC000500C7000500C2000500BD00040088
:10134000B9000400B5000400B1000400AD000400C1
:10135000A9000400A5000300A20003009F000400F0
:101360009B00030098000300950002009300030017
:10137000900003008D0002008B0003008800020033
:101380008600020084000300810002007F0002004A
:101390007D0002007B00020079000200770001005E
:1013A0007600020074000200720001007100020069
:1013B0006F0002006D0001006C0002006A00010075
:1013C000690002006700010066000100650001007D
:1013D0006400020062000100610001006000010081
:1013E0005F0002005D0001005C0001005B00010085
:1013F0005A00010059000100580001005700010087
:101400005600010055000100540001005300000087
:101410005300010052000100510001005000010082
:101420004F0001004E0000004E0001004D00010081
:101430004C0001004B0000004B0001004A0001007D
:101440004900010048000000480001004700010079
:101450004600000046000100450000004500010074
:10146000440001004300000043000100420000006E
:101470004200010041000000410001004000010065
:101480003F0000003F0001003E0000003E00010060
:101490003D0000003D0001003C0000003C00000059
:1014A0003C0001003B0000003B0001003A0000004E
:1014B0003A00010039000000390001003800000046
:1014C000380000003800010037000000370001003C
:1014D0003600000036000000360001003500000034
:1014E0003500000035000100340000003400000029
:1014F000340001003300000033000000330001001D
:101500003200000032000000320001003100000013
:101510003100000031000100300000003000000008
:10152000300001002F0000002F0000002F000000FD
:101530002F0001002E0000002E0000002E000100F0
:101540002D0000002D0000002D0000002D000100E6
:101550002C0000002C0000002C0000002C000100DA
:101560002B0000002B0000002B0000002B000100CE
:101570002A0000002A0000002A0000002A000100C2
:1015800029000000290000002900000029000000B7
:1015900029000100280000002800000028000000A9
:1015A000280000002800010027000000270000009C
:1015B000270000002700000027000100260000008F
:1015C0002600000026000000260000002600010082
:1015D0002500000025000000250000002500000077
:1015E0002500000025000100240000002400000068
:1015F000240000002400000024000100230000005B
:10160000230000002300000023000000230000004E
:10161000230000002300010022000000220000003F
:101620002200000022000000220000002200010031
:101630002100000021000000210000002100000026
:101640002100000021000000210001002000000016
:10165000200000002000000020000000200000000A
:101660002000000020000000200001001F000000FA
:101670001F0000001F0000001F0000001F000000EE
:101680001F0000001F0001001E0000001E000000DF
:101690001E0000001E000000232C0000B8220000E5
:1016A000561800003A0F0000B8080000B10400000E
:1016B000710200003E01000020423A0020436F7595
:1016C0006E7420413A0042656400453100626564F1
:1016D000002C2073797374656D2073746F7070655E
:1016E0006421204865617465725F49443A2000486E
:1016F000656174696E67204661696C656400486560
:101700006174696E67206661696C6564004D313192
:10171000322053687574646F776E001000C9021030
:10172000012C014001220170011801B0010E01F0ED
:101730000104015002FA00B002F0003003E600D0CC
:1017400003DC009004D2007005C800A006BE0000B3
:1017500008B400B009AA00D00BA000600E9600608B
:10176000118C000015820020197800C01D6E00A0A9
:10177000226400B0275A00902C500000314600E04F
:10178000343C0010383200903A2800603C1E00A023
:101790003D1400803E0A00203F0000544845524D51
:1017A000414C2052554E4157415900546865726D65
:1017B000616C2052756E61776179004572723A20D2
:1017C0004D415854454D50004D415854454D5020C1
:1017D000747269676765726564004572723A204D7C
:1017E000494E54454D50004D494E54454D5020747E
:1017F000726967676572656400202F002042403A75
:101800000020403A0020573A0020573A00496E76AF
:10181000616C69642065787472756465720A007C15
:101820003C3E5E2B3D3F2F5B5D3B2C2A225C004300
:101830004F4D4D554E49434154494F4E0044525926
:1018400052554E004552524F525300494E464F009A
:101850004543484F004572726F7220777269746910
:101860006E6720746F20454550524F4D210A00533A
:10187000544F505045442E20005072696E7465726A
:101880002073746F707065642064756520746F20B8
:101890006572726F72732E204669782074686520B5
:1018A0006572726F7220616E6420757365204D39A8
:1018B000393920746F20726573746172742E202818
:1018C00054656D70657261747572652069732072FC
:1018D000657365742E205365742069742061667485
:1018E00065722072657374617274696E67290A008B
:1018F0004E6F20436865636B73756D2077697468FC
:10190000206C696E65206E756D6265722C204C616D
:101910007374204C696E653A20004E6F20436865F1
:10192000636B73756D2077697468206C696E6520D0
:101930006E756D6265722C204C617374204C696EFB
:10194000653A2000636865636B73756D206D69731C
:101950006D617463682C204C617374204C696E65F2
:101960003A20004C696E65204E756D626572206983
:1019700073206E6F74204C617374204C696E652007
:101980004E756D6265722B312C204C617374204C46
:10199000696E653A20004D313130005365726961DE
:1019A0006C20737461747573206D69736D617463F9
:1019B000680A00776169740A0053442072656164A3
:1019C000206572726F720A00486F74656E642049F8
:1019D000646C652054696D656F757400486F74653B
:1019E0006E642049646C652054696D656F75740A76
:1019F000002121204B494C4C2063617573656420A4
:101A00006279204B494C4C20627574746F6E2F7054
:101A1000696E0A002121204B494C4C20636175738B
:101A2000656420627920746F6F206D75636820692A
:101A30006E6163746976652074696D65202D20631D
:101A4000757272656E7420636F6D6D616E643A209D
:101A5000004D656469612052656D6F766564004D67
:101A60006564696120496E736572746564004D3107
:101A70003030305300627573793A20706175736548
:101A80006420666F7220696E7075740A00627573E7
:101A9000793A2070617573656420666F7220757382
:101AA00065720A00627573793A2070726F636573AC
:101AB00073696E670A00506C6561736520526573C7
:101AC0006574005052494E5445522048414C54458B
:101AD000440025533A20255300706F7765726F6676
:101AE00066004B494C4C45442E20005072696E7480
:101AF00065722068616C7465642E206B696C6C285B
:101B0000292063616C6C6564210A0053544F505066
:101B100045442E20005072696E7465722073746F94
:101B2000707065642064756520746F206572726FD3
:101B300072732E2046697820746865206572726F12
:101B40007220616E6420757365204D3939392074B7
:101B50006F20726573746172742E202854656D70E5
:101B6000657261747572652069732072657365743E
:101B70002E2053657420697420616674657220722A
:101B8000657374617274696E67290A006563686FB2
:101B90003A004572726F723A0042696C696E656113
:101BA00072204C6576656C696E6720477269643A8D
:101BB0000A0021212053544F502063616C6C6564EE
:101BC0002062656361757365206F6620424C546FB7
:101BD000756368206572726F72202D207265737450
:101BE0006172742077697468204D3939390A00218F
:101BF000212053544F502063616C6C6564206265F2
:101C00006361757365206F6620424C546F7563681D
:101C1000206572726F72202D207265737461727408
:101C20002077697468204D3939390A005072696E1D
:101C300074696E67204F626A6563740025532025BE
:101C400069002F2F616374696F6E3A00737461725B
:101C50007400656E6400486F74656E6420746F6F05
:101C600020636F6C640A0053656E64204D31303818
:101C700020746F20726573756D650A00496E736517
:101C800072742066696C616D656E7420616E64208B
:101C900073656E64204D3130380A005265686561A5
:101CA0007420446F6E6500526568656174696E6783
:101CB0002E2E2E005265686561740048656174655A
:101CC000722054696D656F75740053656E64204DA4
:101CD00031303820746F2068656174206E6F7A7AB5
:101CE0006C650A004E6F7A7A6C65205061726B6584
:101CF000640070617573656400506175736500728E
:101D00006573756D65640070726F6D70745F0073DC
:101D1000686F7700627574746F6E00626567696ED4
:101D20000050757267654D6F72650050617573651F
:101D300064004C6F61642046696C616D656E74204F
:101D40005400496E736572742066696C616D656ECE
:101D50007420616E642073656E64204D3130380AE2
:101D600000526573756D696E6700473236204361B6
:101D70006E63656C6564004732362048656174693E
:101D80006E67204E6F7A7A6C650047323620486560
:101D90006174696E67204265640057616974696E99
:101DA0006720666F72206865617475702E0A004640
:101DB00069786564204C656E677468205072696D3F
:101DC0006500446F6E65205072696D696E67004DE5
:101DD000616E75616C207072696D696E672E2E2E52
:101DE000004C656176696E6720473236003F53705C
:101DF0006563696669656420582C5920636F6F724A
:101E000064696E617465206F7574206F6620626FFF
:101E1000756E64732E0A003F2852296570656174DF
:101E20002076616C7565206E6F7420706C617573BF
:101E300069626C653B206D75737420626520617406
:101E4000206C6561737420312E0A003F5370656306
:101E50006966696564206E6F7A7A6C652074656D59
:101E60007065726174757265206E6F7420706C613C
:101E7000757369626C652E0A003F5370656369660D
:101E80006965642066696C616D656E742073697A3A
:101E900065206E6F7420706C61757369626C652E5D
:101EA0000A003F53706563696669656420707269F2
:101EB0006D65206C656E677468206E6F7420706C41
:101EC00061757369626C652E0A003F5370656369C2
:101ED00066696564206E6F7A7A6C652073697A65CD
:101EE000206E6F7420706C61757369626C652E0A68
:101EF000003F52657472616374696F6E204D756C3A
:101F00007469706C696572206D75737420626520E8
:101F10007370656369666965642E0A003F53706576
:101F20006369666965642052657472616374696F80
:101F30006E204D756C7469706C696572206E6F747B
:101F400020706C61757369626C652E0A003F537076
:101F500065636966696564206C617965722068658E
:101F600069676874206E6F7420706C617573696244
:101F70006C652E0A0043292E0A003F537065636981
:101F800066696564206265642074656D7065726160
:101F900074757265206E6F7420706C617573696200
:101FA0006C65202834302D004732362073746172FE
:101FB00074696E672E2E2E0A004F46460A0046614F
:101FC0006465204865696768742000426564204C38
:101FD0006576656C696E6720004661696C65642092
:101FE000746F20656E61626C6520426564204C658B
:101FF00076656C696E670A00496E76616C6964206B
:102000006D6573682E0A0050726F62696E672050AA
:102010006F696E740025532025692F2569002E0AEB
:10202000002F0050726F62696E67206D65736820C3
:10203000706F696E742000202844525952554E2901
:1020400000473239204175746F20426564204C6529
:1020500076656C696E67003F20284C2C522C462C0C
:102060004229206F7574206F6620626F756E6473ED
:102070002E0A003F2856296572626F7365206C65D1
:1020800076656C20696D706C61757369626C652032
:1020900028302D34292E0A00426164205A207661AE
:1020A0006C75650A004E6F2062696C696E656172BD
:1020B00020677269640A00446576696174696F6EAD
:1020C0000025533A2025730046696E69736865647C
:1020D000210A003A207A3A2000206F662000476FDC
:1020E000696E6720746F3A20580043570A002064D5
:1020F00069723A0020616E676C653A0053746172D0
:1021000074207261646975733A004D343820506FE1
:10211000696E740025533A2025642F256400506FA2
:10212000736974696F6E696E672074686520707278
:102130006F62652E2E2E0A003F4C656773206F6616
:10214000206D6F76656D656E7420696D706C61755C
:102150007369626C652028302D3135292E0A003FC5
:102160002028582C5929206F7574206F6620626FC3
:10217000756E64732E0A0050726F6265206F7574FD
:10218000206F6620626F756E6473003F53616D70DF
:102190006C652073697A65206E6F7420706C617550
:1021A0007369626C652028342D3530292E0A004D64
:1021B0003438205A2D50726F626520526570656107
:1021C000746162696C69747920546573740A003FA4
:1021D0002856296572626F7365206C6576656C2080
:1021E000696D706C61757369626C652028302D347F
:1021F000292E0A005374616E64617264204465760E
:10220000696174696F6E3A20002052616E67653AA9
:102210002000204D61783A2000204D696E3A200060
:10222000205369676D613A20004D65616E3A200068
:10223000205200416363656C65726174696F6E3A28
:102240002050005741524E494E4721204C6F772075
:102250005A204A65726B206D6179206C656164203B
:10226000746F20756E77616E74656420706175732C
:1022700065732E0A0020204D61783A20002000204E
:10228000204D696E3A2000536F667420656E64734A
:10229000746F70733A20004D32342053256C6420E3
:1022A00054256C64004739322E3920452573004788
:1022B0003120462564004739322E39205A257300D3
:1022C0004731205A302046323030004731205825DF
:1022D0007320592573204633303030004D3432306E
:1022E00020532569205A2573004D31303620502562
:1022F0006920532569004D32303020442573004752
:10230000323852305859004739322E392045302062
:102310005A300A47315A2573004D31303920532540
:1023200069004D31393020532569004D3432302059
:102330005330205A300020496E76616C6964206504
:1023400078747275646572200047322F47332062BB
:10235000616420706172616D65746572730A005307
:102360006C6565702E2E2E005A2050726F626520AB
:1023700050617374204265640A005A2050726F6283
:1023800065205061737420426564004732384C30D8
:10239000004D3131372050726F6265206661696C83
:1023A00065642E0A4732380A0070726F62655F7288
:1023B00065776970650047323920526574727969B2
:1023C0006E670050726F62696E67204661696C6566
:1023D00064004D31313720426564206C6576656C50
:1023E000696E67206661696C65642E0A4730205A01
:1023F00031300A4D333030205032352053383830A8
:102400000A4D333030205035302053300A4D3330B0
:10241000302050323520533838300A4D3330302098
:102420005035302053300A4D333030205032352073
:10243000533838300A4D3330302050353020533047
:102440000A47342053310070726F62655F666169BC
:102450006C6564004D31313720426564206C6576CF
:10246000656C696E6720646F6E652E00205A3A2095
:102470000020593A200042656420583A20004D65FA
:10248000736820706F696E74206F7574206F66209A
:1024900072616E67650A004D302053746F70004D95
:1024A000312053746F7000436F6E74696E756500F0
:1024B000436C69636B20746F20526573756D652E74
:1024C0002E2E004E6F204D6F76652E00456E6420D7
:1024D00066696C65206C6973740A00426567696E91
:1024E0002066696C65206C6973740A004E6F206DFC
:1024F000656469610A00526573756D696E67205382
:102500004400286E6F2066696C65290043757272FD
:10251000656E742066696C653A20005072696E744D
:102520002074696D653A20000A53746174733A200F
:1025300046696C616D656E7420757365643A200040
:102540002C204C6F6E67657374206A6F623A2000AE
:10255000546F74616C2074696D653A200053746126
:1025600074733A20002C204661696C65643A20003F
:102570002C2046696E69736865643A200050726960
:102580006E74733A200053746174733A2000436F81
:102590006F6C696E672E2E2E0048656174696E67D8
:1025A0002E2E2E0045202553006F6B006F666600AF
:1025B00050184B1844183D182F1844454255473AB7
:1025C000004D31313320530042656420436F6F6CFE
:1025D000696E672E2E2E004265642048656174691D
:1025E0006E672E2E2E00544D334420456E64657266
:1025F00034204F46462E002F2F004D3134352053C6
:102600003C696E6465783E206F7574206F66207239
:10261000616E67652028302D31290A004D32303631
:1026200020580046523A0020466C6F773A20003A14
:10263000200020536572766F2000206F7574206F24
:10264000662072616E67650A00536572766F2000BE
:1026500020643A0020693A0020703A00496E7661A1
:102660006C69642065787472756465720A00206410
:102670003A0020693A0020703A0064697300656E80
:102680000043290A0061626C656420286D696E2030
:1026900074656D702000436F6C642065787472758A
:1026A0006465732061726520004D34323120696E9B
:1026B000636F727265637420706172616D657465B9
:1026C000722075736167650A004D65736820706FCD
:1026D000696E74206F7574206F662072616E676515
:1026E0000A004F666673657473204170706C69658B
:1026F00064004572723A20546F6F20666172210047
:10270000546F6F206661722066726F6D207265660D
:102710006572656E636520706F696E740A00454569
:1027200050524F4D204F4B0A002E0A002028302DCA
:10273000313029002076616C7565206F7574206FCB
:10274000662072616E676500416476616E63652024
:102750004B3D004F4646004F4E00506F7765722D3F
:102760006C6F7373207265636F7665727920004DAC
:10277000383400446F6E65207072696E74696E67DC
:102780002066696C650A004D3737004D33310055BE
:102790004E4C4F41442046494C414D454E54004C0F
:1027A0004F41442046494C414D454E540046494C0A
:1027B000414D454E54204348414E474500436170CA
:1027C0003A004D4541545041434B00434F4F4C4517
:1027D000525F54454D50455241545552450043486F
:1027E000414D4245525F54454D504552415455521A
:1027F0004500424142595354455050494E470041CB
:10280000524353004D4F54494F4E5F4D4F44455333
:1028100000544845524D414C5F50524F544543542B
:10282000494F4E004C4F4E475F46494C454E414D37
:1028300045004155544F5245504F52545F53445FE9
:102840005354415455530053445F57524954450023
:102850005245504541540053444341524400505264
:102860004F4D50545F535550504F525400454D45B5
:102870005247454E43595F504152534552004341E0
:1028800053455F4C494748545F4252494748544E6C
:1028900045535300544F47474C455F4C49474854B4
:1028A0005300534F4654574152455F504F5745527E
:1028B000004255494C445F50455243454E54004CEC
:1028C0004556454C494E475F44415441005A5F507C
:1028D000524F42450052554E4F5554004155544FAA
:1028E0004C4556454C005052494E545F4A4F4200A9
:1028F00050524F4752455353004155544F52455043
:102900004F52545F54454D5000564F4C554D455411
:1029100052494300454550524F4D0042494E4152A5
:10292000595F46494C455F5452414E53464552000B
:1029300053455249414C5F584F4E5F584F464600F1
:102940004649524D574152455F4E414D453A4D61C2
:10295000726C696E20322E302E375F4457372E331B
:1029600020544D3344204534454D444242202841B3
:10297000707220323420323032312032313A3339E1
:102980003A35302920534F555243455F434F444514
:102990005F55524C3A68747470733A2F2F6769749C
:1029A0006875622E636F6D2F496E73616E697479FD
:1029B0004175746F6D6174696F6E2F4D61726C69D2
:1029C0006E2F747265652F437265616C697479440A
:1029D00077696E5F322E302050524F544F434F4C28
:1029E0005F56455253494F4E3A312E30204D4143A8
:1029F00048494E455F545950453A544D334420455B
:102A00006E646572342045585452554445525F43B4
:102A10004F554E543A3120555549443A63656465E3
:102A2000326132662D343161322D343734382D39EC
:102A30006231322D6335356336326633363766663A
:102A40000A0050726F6265204F6666736574205A83
:102A50000050726F6265204F6666736574205A007D
:102A6000290A0020746F20003F5A206F7574206F70
:102A7000662072616E6765202800290A0020746F45
:102A800020003F59206F7574206F662072616E6759
:102A90006520282D00290A0020746F20003F58204F
:102AA0006F7574206F662072616E676520282D0037
:102AB00050726F6265204F666673657420580043DC
:102AC000616E6E6F74206F70656E207375626469DD
:102AD0007220002569730025696D20256973002522
:102AE00069682025696D20256973002569642025A2
:102AF00069682025696D202569730025697920257D
:102B00006964202569682025696D20256973002383
:102B1000646566696E652044454641554C545F00C6
:102B2000626564004B6420004B6920004B702000FC
:102B3000504944204175746F74756E652066696EE6
:102B40006973686564212050757420746865206C11
:102B5000617374204B702C204B6920616E64204B94
:102B60006420636F6E7374616E74732066726F6D30
:102B70002062656C6F7720696E746F20436F6E669C
:102B8000696775726174696F6E2E680A00504944F6
:102B9000204175746F74756E65206661696C65643B
:102BA000212074696D656F75740A00504944204195
:102BB00075746F74756E65206661696C656421203B
:102BC00054656D706572617475726520746F6F20E5
:102BD000686967680A00204B643A2000204B693A14
:102BE0002000204B703A200020436C6173736963AE
:102BF00020504944200A00204E6F206F7665727382
:102C0000686F6F740A002054753A2000204B753AA3
:102C10002000206D61783A2000206D696E3A200016
:102C200020643A200020626961733A2000504944D0
:102C3000204175746F74756E652073746172740AC7
:102C400000504944204175746F74756E652066614B
:102C5000696C6564212054656D706572617475726C
:102C60006520746F6F20686967680A0050494420C6
:102C70004175746F74756E650050494420417574D8
:102C80006F74756E65206661696C656421204261B0
:102C900064206865617465722069640A00A100009F
:102CA000006900A20000006300B00000000900C13C
:102CB0000000004100C20000004100C300000041CC
:102CC00000C40000004100C50000004100C6000033
:102CD000004145C70000004300C80000004500C98E
:102CE0000000004500CD0000004900D10000004E6A
:102CF00000D50000004F00D60000004F00D70000B4
:102D0000007800DC0000005500DD0000005900E004
:102D10000000006100E10000006100E200000061CD
:102D200000E30000006100E40000006100E5000035
:102D3000006100E60000006165E70000006300E854
:102D40000000006500E90000006500EA0000006581
:102D500000EB0000006500EC0000006900ED0000E1
:102D6000006900EE0000006900EF0000006900F15A
:102D70000000006E00F20000006F00F30000006F22
:102D800000F40000006F00F50000006F00F6000086
:102D9000006F00F80000006F00F90000007500FAF5
:102DA0000000007500FB0000007500FC00000075CD
:102DB00000FD0000007900FF000000790004010020
:102DC000004100050100006100060100004300070A
:102DD00001000063000C01000043000D01000063CE
:102DE000000E01000044000F01000064001101000A
:102DF0000064001901000065001A01000045001B75
:102E000001000065001F010000670030010000495B
:102E100000310100006900410100004C0042010046
:102E2000006C00430100004E00440100006E0048A9
:102E30000100006E005801000052005901000072AC
:102E4000005A01000053005B01000073005F0100A5
:102E50000073006001000053006101000073006511
:102E600001000074006F01000075007C0100007A11
:102E7000007D0100005A007E0100007A00920100EE
:102E8000006600E30200007800222000002E001EF1
:102E9000210000507822210000544D902100003C78
:102EA0002D922100002D3EB02100000300BB210027
:102EB0000004003C2200007E00482200007E3D60AD
:102EC000220000213D612200003D00642200003C00
:102ED0003D652200003E3DF12300000700A03000C8
:102EE000003D0021F301000200C2F401000500A230
:102EF000000000EC00B0000000DF00E4000000E192
:102F000000F6000000EF00F7000000FD00FC0000EC
:102F100000F500E3020000EB0087030000A5008F2E
:102F2000030000F40098030000F2009E030000E399
:102F300000A3030000F600A9030000F400AC0300A6
:102F400000E000AD030000E300B1030000E000B2C8
:102F5000030000E200B5030000E300B8030000F244
:102F600000BC030000E400BE030000E300C0030057
:102F700000F700C1030000E600C3030000E5009075
:102F80002100007F00922100007E001A220000E84C
:102F9000001E220000F30088250000FF0002300020
:102FA00000A1000C300000A2000D300000A3009B27
:102FB000300000DE009C300000DF00A03000003D4B
:102FC00000A1300000A700A2300000B100A3300033
:102FD00000A800A4300000B200A5300000A900A69F
:102FE000300000B300A7300000AA00A8300000B4F1
:102FF00000A9300000AB00AA300000B500AB3000E3
:1030000000B600AC300000B6DEAD300000B700AE58
:10301000300000B7DEAF300000B800B0300000B8BC
:10302000DEB1300000B900B2300000B9DEB33000CC
:1030300000BA00B4300000BADEB5300000BB00B604
:10304000300000BBDEB7300000BC00B8300000BC70
:10305000DEB9300000BD00BA300000BDDEBB30007C
:1030600000BE00BC300000BEDEBD300000BF00BEB0
:10307000300000BFDEBF300000C000C0300000C024
:10308000DEC1300000C100C2300000C1DEC330002C
:1030900000AF00C4300000C200C5300000C2DEC670
:1030A000300000C300C7300000C3DEC8300000C4D9
:1030B00000C9300000C4DECA300000C500CB3000BB
:1030C00000C600CC300000C700CD300000C800CEE4
:1030D000300000C900CF300000CA00D0300000CA64
:1030E000DED1300000CADFD2300000CB00D3300088
:1030F00000CBDED4300000CBDFD5300000CC00D6D2
:10310000300000CCDED7300000CCDFD8300000CD5E
:1031100000D9300000CDDEDA300000CDDFDB30003A
:1031200000CE00DC300000CEDEDD300000CEDFDE81
:10313000300000CF00DF300000D000E0300000D1D0
:1031400000E1300000D200E2300000D300E33000A4
:1031500000AC00E4300000D400E5300000AD00E633
:10316000300000D500E7300000AE00E8300000D6A7
:1031700000E9300000D700EA300000D800EB300052
:1031800000D900EC300000DA00ED300000DB00EF89
:10319000300000DC00F2300000A600F3300000DD5B
:1031A00000F4300000B3DEF7300000DCDEFA30005F
:1031B00000A6DEFB300000A500FC300000B000FDE2
:1031C000300000A400074E0000FB0086510000FC08
:1031D0000043530000FA0064FF0000A40065FF00F4
:1031E00000A50066FF0000A60067FF0000A70068BA
:1031F000FF0000A80069FF0000A9006AFF0000AA04
:10320000006BFF0000AB006CFF0000AC006DFF0026
:1032100000AD006EFF0000AE006FFF0000AF007059
:10322000FF0000B00071FF0000B10072FF0000B2AB
:103230000073FF0000B30074FF0000B40075FF00CE
:1032400000B50076FF0000B60077FF0000B70078F9
:10325000FF0000B80079FF0000B9007AFF0000BA53
:10326000007BFF0000BB007CFF0000BC007DFF0076
:1032700000BD007EFF0000BE007FFF0000BF008099
:10328000FF0000C00081FF0000C10082FF0000C2FB
:103290000083FF0000C30084FF0000C40085FF001E
:1032A00000C50086FF0000C60087FF0000C7008839
:1032B000FF0000C80089FF0000C9008AFF0000CAA3
:1032C000008BFF0000CB008CFF0000CC008DFF00C6
:1032D00000CD008EFF0000CE008FFF0000CF0090D9
:1032E000FF0000D00091FF0000D10092FF0000D24B
:1032F0000093FF0000D30094FF0000D40095FF006E
:1033000000D50096FF0000D60097FF0000D7009878
:10331000FF0000D80099FF0000D9009AFF0000DAF2
:10332000009BFF0000DB009CFF0000DC009DFF0015
:1033300000DD009EFF0000DE009FFF0000DF00E5D3
:10334000FF00005C00001C1F11111F000000061987
:103350001803130C00040E1F041C000000001010C2
:10336000101010100000141414141414000015157B
:103370001515151500000E1315110E00001C101860
:103380001705060500040A0A0A0A11110E0C12128A
:103390000C00000000001F1511151F00004265649D
:1033A00000456E636C6F73757265002568753A250C
:1033B000303268750025303268753A2530326875CC
:1033C000002D2D2D005344002020202020202000FF
:1033D00020202020006E6F74696669636174696FD4
:1033E0006E20006E6F74696669636174696F6E2028
:1033F0000063616E63656C005072696E7420416297
:103400006F72746564004469736D69737300554924
:103410002041626F72746564004D323520500A4D50
:10342000323400526573756D6500554920506175E1
:1034300073650050617573696E672E2E2E0072657C
:1034400073756D65004D32340050726F6265205A9D
:10345000204F6666736574004C6F6164206D6D006B
:10346000556E6C6F6164206D6D0046696C2E204452
:1034700069612E004520696E206D6D5E33004164E8
:1034800076616E6365204B004D333033205531201B
:103490004525692053256900504944204175746FC2
:1034A00074756E65202A005049442D44202A00502E
:1034B00049442D49202A005049442D50202A0020FB
:1034C000022046616374002002204D6178002002D2
:1034D000204D696E004F6666004F6E004175746F37
:1034E00074656D70005654726176204D696E005699
:1034F0006D696E00566D6178204500566D617820CB
:103500005A00566D6178205900566D617820580038
:10351000416D6178204500416D6178205A00416D10
:103520006178205900416D6178205800412D547216
:103530006176656C00412D5265747261637400415F
:103540006363656C0056652D4A65726B00565A2D93
:103550004A65726B0056592D4A65726B0056582D9C
:103560004A65726B0050726F6265205A204F666622
:103570007365740050726F62652059204F666673E0
:1035800065740050726F62652058204F66667365DF
:103590007400452073746570732F6D6D005A20534D
:1035A000746570732F6D6D00592053746570732F9F
:1035B0006D6D00582053746570732F6D6D004164FC
:1035C00076616E6365642053657474696E67730019
:1035D0003F0043616E63656C00496E6974004D3451
:1035E000323800496E697469616C697A65204545B5
:1035F00050524F4D0046696C616D656E74005465A4
:103600006D70657261747572650053746570732FA7
:103610006D6D0050726F6265204F666673657473DE
:10362000004A65726B00416363656C657261746921
:103630006F6E0056656C6F63697479005365742012
:10364000486F6D65204F66667365747300436F6ED7
:1036500066696775726174696F6E003F004E6578C8
:103660007420506F696E7400446F6E65004E65780B
:103670007400486F6D696E672058595A003F0043C7
:10368000616E63656C204F626A656374004E4F0023
:103690005945530043616E63656C204F626A6563F0
:1036A00074203D004D61696E0053746F770044656E
:1036B000706C6F790053656C662D5465737400539C
:1036C000572D4D6F646500526573657400426564E3
:1036D000004E6F7A7A6C650046616E2053706565A6
:1036E0006400436F6E66696775726174696F6E001E
:1036F0004C6F61642053657474696E677300526522
:1037000073746F72652044656661756C74730053E1
:10371000746F72652053657474696E6773005072BC
:103720006568656174202420436F6E66004F66668D
:10373000004F6E00506F776572204F75746167653A
:1037400000424C546F7563680050726F6265205A76
:10375000204F666673657400416476616E636564CC
:103760002053657474696E6773004D61696E004D16
:1037700037303220542564004D363030204230201E
:10378000542564004D373032203B2564004D3730DE
:10379000312054256400436F6E74696E7565005066
:1037A00075726765206D6F726500524553554D45C2
:1037B000204F5054494F4E533A005052494E5420D6
:1037C0005041555345440020204E6F7A7A6C653A3B
:1037D00020005061726B696E672E2E2E000000571C
:1037E00061697420666F720066696C616D656E74E4
:1037F000206368616E676500746F20737461727412
:10380000005761697420666F720066696C616D654E
:103810006E7420756E6C6F616400004E6F7A7A6C06
:10382000652068656174696E6700506C65617365D9
:1038300020776169742E2E2E0000507265737320FC
:10384000627574746F6E00746F2068656174206EA9
:103850006F7A7A6C650000496E73657274206669D0
:103860006C616D656E7400616E6420707265737357
:1038700020627574746F6E00746F20636F6E74696C
:103880006E7565005761697420666F720066696CB9
:10389000616D656E74206C6F6164000050726573B9
:1038A0007320427574746F6E00746F207265737547
:1038B0006D65207072696E740000576169742066CE
:1038C0006F72207072696E7400746F207265737508
:1038D0006D652E2E2E00005761697420666F720090
:1038E00066696C616D656E74207075726765000045
:1038F0003E2000256C642E25696D00457874727534
:1039000064656420546F74616C003E20004C6F6EDF
:1039100067657374204A6F622054696D65003E20AC
:1039200000546F74616C205072696E742054696D1C
:103930006500436F6D706C65746564003A200050DB
:1039400072696E7420436F756E74003A20003135D1
:10395000300035004245443A204154432031303450
:1039600047542D320052756E61776179205761742A
:1039700063683A204F4E004D61782054656D7000A9
:10398000343530004D696E2054656D70003500454A
:10399000313A20536C696365456E6720343530C217
:1039A000B043005053550047656E6572696300501F
:1039B000726F746F636F6C00312E300042617564FA
:1039C0000032353030303000437265616C69747993
:1039D00033442052414D50530042696C696E656119
:1039E00072204C6576656C696E67004578747275F7
:1039F0006465727300310074696E796D6163686922
:103A00006E657333642E636F6D00544D33442045EF
:103A10006E6465723400323032312D30342D3138DD
:103A200000322E302E375F4457372E33004D6172EF
:103A30006C696E005072696E7465722053746174A3
:103A40007300546865726D6973746F727300426FAE
:103A500061726420496E666F005072696E7465729F
:103A600020496E666F004D61696E004D3130303017
:103A70000053746F70205072696E740052657375D4
:103A80006D65205072696E7400506F776572204FBB
:103A90007574616765004D3139305335350A4732E9
:103AA000380A4732390A4D3430300A4D31303453F8
:103AB0003231350A4732380A4D31303953323135D7
:103AC0000A4D34323053310A473158313030593190
:103AD000303046353030300A47315A300A4D3530B3
:103AE000300A4D31313720536574205A204F6666B5
:103AF000736574004D313036533132380A4D3330EE
:103B0000334338533231354530550A4D3530300A5C
:103B10004D313137205049442054756E6520446F33
:103B20006E65004D3139305335350A4D31303453DF
:103B30003231350A4732380A4732394C310A473177
:103B400020583130305931303046353030300A4726
:103B5000315A30004D3530300A4D31313720536500
:103B60007474696E67732053746F72656400507269
:103B7000657020666F72205A2041646A7573740004
:103B80005049442054756E650053746F726520531C
:103B9000657474696E6773005365747570004D6168
:103BA000696E003F004261636B0053746F700043A5
:103BB00068616E67652046696C616D656E74005062
:103BC00072656865617420437573746F6D0050721F
:103BD00065686561742024004261636B00507269FE
:103BE0006E742066726F6D204D6564696100436874
:103BF000616E6765204D65646961004D3231004139
:103C0000626F7574205072696E74657200436861EA
:103C10006E67652046696C616D656E74004D363067
:103C200030204230004C6576656C696E6720546FB9
:103C30006F6C7300436F6E66696775726174696F4C
:103C40006E0054656D7065726174757265004D6FBC
:103C500074696F6E00486F737420537461727400DE
:103C6000526573756D65205072696E74004E6F20D9
:103C70004D656469610043616E63656C204F626AE3
:103C80006563740054756E650053746F70205072D4
:103C9000696E74005061757365205072696E7400AE
:103CA000496E666F2053637265656E0043616E6E88
:103CB0006F74206F70656E20737562646972200086
:103CC000534420496E6974204661696C0053442056
:103CD00063617264206F6B0A006F70656E526F6F64
:103CE00074206661696C65640A00766F6C756D6539
:103CF0002E696E6974206661696C65640A004E6F96
:103D000020534420636172640A000A4D3234004D2E
:103D10003233202573002E0A006F70656E206661B5
:103D2000696C65642C2046696C653A200046696CB4
:103D3000652073656C65637465640A002053697A55
:103D4000653A200046696C65206F70656E65643A5F
:103D50002000454E4420535542524F5554494E453C
:103D60000A002220706F73002220706172656E74E9
:103D70003A2200535542524F5554494E4520434133
:103D80004C4C207461726765743A2200537562630B
:103D9000616C6C204F766572666C6F770045786356
:103DA0006565646564206D617820535542524F55B6
:103DB00054494E452064657074683A002E0A0044E8
:103DC000656C6574696F6E206661696C65642C2032
:103DD00046696C653A200046696C652064656C65CF
:103DE0007465643A005344207072696E74696E673A
:103DF000206279746520004E6F74205344207072E5
:103E0000696E74696E670A002F6175746F25632E81
:103E1000670057726974696E6720746F2066696CF9
:103E2000653A2000667265736800646F696E6700AA
:103E30002066696C653A20004E6F772000026001B1
:103E4000F4017001EA019001E001B001D601D00156
:103E5000CC010002C2013002B8016002AE01900242
:103E6000A401D0029A012003900170038601C003CF
:103E70007C0130047201A004680120055E01B005D8
:103E8000540160064A0120074001F0073601F0089E
:103E90002C01100A2201500B1801C00C0E01500E0B
:103EA00004013010FA002012F0005014E600C01691
:103EB000DC007019D200501CC800501FBE007022D8
:103EC000B400B025AA00F028A000202C9600302FC6
:103ED0008C0010328200A0347800F0366E00E0389A
:103EE0006400803A5A00403B5500E03B5000F03CF3
:103EF0004600C03D3C00603E3200E03E2800303FBE
:103F00001E00503F1900703F1400A03F0A00C03F40
:103F10000000D03FF6FFE03FECFF2020506C616EC8
:103F20006E657242756666657242797465733A2091
:103F3000002046726565204D656D6F72793A2000EC
:103F4000436F6D70696C65643A2041707220323441
:103F500020323032310A00204C6173742055706475
:103F6000617465643A20323032312D30342D31386D
:103F7000207C20417574686F723A2054696E794DC7
:103F8000616368696E657333440A00322E302E37E0
:103F90005F4457372E330A004D61726C696E002002
:103FA000536F6674776172652052657365740A0099
:103FB000205761746368646F672052657365740A83
:103FC000002042726F776E206F75742052657365A2
:103FD000740A002045787465726E616C20526573B6
:103FE00065740A00506F77657255700A00737461CA
:103FF00072740A004732385859004D313030310060
:104000006572726F722077726974696E6720746F5F
:104010002066696C650A00446F6E6520736176697D
:104020006E672066696C652E0A004D323900456E58
:104030006473746F707300255320256320256320FB
:10404000256320256300205A3A0020593A00205861
:104050003A00656E6473746F7073206869743A20F7
:104060000000000A0B02090C0D0E080703040100F2
:104070000000000000000000000000000000000040
:1040800000000000000000000000000000121110FD
:104090000000000000000000000000000000000020
:1040A00000000000000000004D6F76652025736D54
:1040B0006D004D6F766520302E316D6D004D6F7641
:1040C0006520316D6D004D6F76652031306D6D006E
:1040D0004D6F766520417869730045787472756418
:1040E0006572004D6F7665205A004D6F76652059D8
:1040F000004D6F76652058005072696E74206672AC
:104100006F6D204D656469610050726F62696E6702
:10411000204661696C656400205A3A200020593AB3
:10412000200042656420583A2000220A00556E6B38
:104130006E6F776E20636F6D6D616E643A20220042
:104140002042002050006F6B00544D334420456ED8
:10415000646572342052656164792E005072696E14
:1041600074696E672E2E2E005072696E7420506135
:104170007573656400204500205A00205900204DC9
:10418000393220580020453A00205A3A0020593A46
:1041900000583A0020746F6F206C6F6E672065784E
:1041A00074727573696F6E2070726576656E746572
:1041B000640A0020636F6C6420657874727573699B
:1041C0006F6E2070726576656E7465640A00526564
:1041D00073656E643A200000002200250028002B41
:1041E000002E003100340002010000050108010B1F
:1041F0000100002100240027002A002D0030003398
:104200000001010000040107010A01050505050779
:104210000508080808020202020A0A080804040441
:10422000040101010101010101030303030303036D
:1042300003040707070C0C0C0C0C0C0C0C020202FC
:104240000206060606060606060B0B0B0B0B0B0BEF
:104250000B0102102020080810204010204080028E
:1042600001020108040201010204081020408080BC
:104270004020100804020180040201804020100840
:104280000402010804020101020408102040800118
:1042900002040810204080004E01B40011241FBE0B
:1042A000CFEFD1E2DEBFCDBF00E00CBF13E0A0E056
:1042B000B2E0E0EAFBEC02E00BBF02C007900D9217
:1042C000A839B107D9F728E1A8E9B3E001C01D92E8
:1042D000A231B207E1F711E2CDE4D1E200E006C07D
:1042E00021970109802FFE010F942862CC34D10759
:1042F00080E00807A9F70F94BF500D94BE650C9499
:1043000000000F931F93CF93DF93CDB7DEB7609775
:104310000FB6F894DEBF0FBECDBF8C01DC01ED916E
:10432000FC910280F381E02DBE016F5F7F4F1995F4
:10433000882309F464C08981807CC9F56F8163702A
:1043400070E0762F6627770F770F8885B4E08B9F14
:10435000C0011124682B792B8985829586958695D5
:104360008370682B6F5F7F4F90E080E02A85237019
:10437000220F3B8537FB332730F9232B3E813F70DB
:10438000230F3327331F2750310904C0660F771FCF
:10439000881F991F2A95D2F760960FB6F894DEBF52
:1043A0000FBECDBFDF91CF911F910F910895803443
:1043B00019F568856695669570E090E080E0CB0120
:1043C000772766272A85622B098510E0102F0027A2
:1043D000012E000C220B330B602B712B822B932BA5
:1043E0006F5F7F4F8F4F9F4F4AE0660F771F881F89
:1043F000991F4A95D1F7D0CF8BE0F801848360E014
:1044000070E0CB01C9CFFC0182810895EF92FF9249
:104410000F931F93E0922704F0922804009329043D
:1044200010932A0460932B0470932C0480932D0422
:104430009FEFFF27621B730B840B30F48095709500
:104440006195790B890B992790933C05A6E06A9FAB
:1044500000923005512DEE277A9F500DE11D8A9F65
:10446000E00D50933105E0933205AFE06A9F009272
:104470003405512DEE277A9F500DE11D8A9FE00DE6
:1044800050933505E0933605AAE06A9F00923805FF
:10449000512DEE277A9F500DE11D8A9FE00D50931C
:1044A0003905E0933A051F910F91FF90EF90089521
:1044B0009F92AF92BF92CF92DF92EF92FF920F93B3
:1044C0001F93CF93DF9300D01F921F92CDB7DEB71B
:1044D000EBE6FAE00027BB27462F572FA82FAA2389
:1044E00041F4A52F542FB85FAA2319F4A52F5527FF
:1044F000B85FA03138F45295A295452F4F70507F88
:10450000A42BBC5FA03428F4550FAA1F550FAA1F77
:10451000BE5FA03818F4550FAA1FB395550FAA1FF8
:10452000EA0FF01F449151E0AA27B85081F1C8F07A
:10453000B0FF02C0440F551FB1FF04C0440F551F08
:10454000440F551FB2FF06C052954295142F1F709D
:10455000407F512BB3FF1BC0A52F542F44270C9431
:10456000C722B195B0FF02C055954795B1FF04C071
:104570005595479555954795B2FF05C05295407F93
:104580004295452B5F70B3FF02C0452F5527DD24B0
:10459000CC24BB24B2E0649FD018C108B00AB00B91
:1045A000749FC018B108B00B849FB018B109659F03
:1045B000C018B108B00B759FB018B109859FB0192C
:1045C0006A9FB018B1097A9FB0194D9DA12C99240A
:1045D0003327992722275D9DA00C911C301F901F27
:1045E000201FAD9D900C311D901F201F4C9DA00CD5
:1045F000911C301F901F201F5C9D900C311D901F3F
:10460000201FAC9D300D911D201F4B9D900C311D26
:10461000901F201F5B9D300D911D201FAB9D900DA5
:10462000211D4B9F300D911D201F5B9F900D211D63
:10463000AB9F200DB1E0BB24CC24DD24639FD018B8
:10464000C108B00AB00B739FC018B108B00B839FAC
:10465000B018B109699FC018B108B00B799FB018A4
:10466000B109899FB019629FB018B109729FB01942
:10467000D61AC70AB80A20F0B1E03B0F901F201FDE
:104680001124792F632F90E0822F0F900F900F90BD
:104690000F900F90DF91CF911F910F91FF90EF90AE
:1046A000DF90CF90BF90AF909F900895CF92DF9210
:1046B000EF92FF9280911608882309F457C0C090AA
:1046C0001208D0901308E0901408F090150820E02C
:1046D00030E0A901C701B6010F943F5B882309F4BC
:1046E00045C020E030E040E05FE3C701B6010F9431
:1046F000A55B9B01AC010F94A55B2BED3FE049E46A
:1047000050E40F94A55B9B01AC0160E070E080E891
:104710009FE30F942B636B017C01C0929D03D092A9
:104720009E03E0929F03F092A00360910C027091AF
:104730000D02072E000C880B990B0F94465B2AE0A4
:1047400037ED43E25CE30F94A55BA70196010F945C
:10475000A55B609378027093790280937A029093BC
:104760007B02FF90EF90DF90CF900895C12CD12C69
:1047700080E8E82E8FE3F82ED0CF60910C02709184
:104780000D02072E000C880B990B0F94465B2AE054
:1047900037ED43E25CE30F94A55B20919D033091DC
:1047A0009E0340919F035091A0030F94A55B6093DB
:1047B00078027093790280937A0290937B02089535
:1047C000E0919B03E23030F4F0E0E15DF64F809140
:1047D0009A07808308958091DA158823C1F081506B
:1047E0008093DA15E4E0F6E1882351F08150990BCB
:1047F0002BE1289FF001299FF00D1124E65CF94E72
:104800008BE1AFE1B6E101900D928A95E1F720913D
:10481000DA15211105C08091E51580628093E515B8
:1048200081E090E0A0E0B0E0211103C080E090E0E2
:10483000DC018093A1079093A207A093A307B093F4
:10484000A4071092970781E08093B10783E08093DB
:10485000770208952091030830910408211531054D
:10486000E9F08091010890910208029624503109E4
:10487000821793079CF490932705809326050F9445
:104880003D37605E70448D4F9F4F60932805709355
:10489000290580932A0590932B05089510922805E9
:1048A0001092290510922A0510922B050895CF9396
:1048B000DF93EC018D810E946CA760E08B81DF911A
:1048C000CF910D943135DF92EF92FF920F931F93AA
:1048D000CF93DF938C01C62FD22FF32EE42ED52E4B
:1048E0000E9457240F946E3C8C2F80640E9460A716
:1048F0008D2D0E9460A78E2D0E9460A78F2D0E9493
:1049000060A78D2F0E9460A787E8C11101C085E9CB
:104910000E9460A7CC3011F40E9465A7C0E00E94FD
:1049200065A7F801868387FF04C0CF3F11F0CF5FF2
:10493000F6CFDF91CF911F910F91FF90EF90DF9015
:10494000089561E0FC0183810F9431358FEF0C9461
:1049500060A70F931F93CF938C010E9457240F944D
:104960006E3CC82F882371F08DEF0E9460A70F94D2
:104970006E3CC82FC8010E94A1248C2FCF911F919B
:104980000F91089582E1F8018483F4CF8F929F9272
:10499000AF92BF92CF92DF92EF92FF920F931F934D
:1049A000CF93DF93EC016A017B01590120E030E0F5
:1049B000A90167E30E946324A501980167E1CE0184
:1049C0000E946324811127C08F81833039F089E0F0
:1049D000CC0CDD1CEE1CFF1C8A95D1F7A7019601BB
:1049E00069E1CE010E94632411E0882319F010E0F0
:1049F00087E08C83CE010E94A124812FDF91CF918B
:104A00001F910F91FF90EF90DF90CF90BF90AF90EC
:104A10009F908F90089589E08C8310E0EBCFCF9327
:104A2000DF93EC016EBDFA01CA019E5F0DB407FE73
:104A3000FDCF20812EBD0DB407FEFDCF21812EBDFF
:104A40003296E817F90791F70DB407FEFDCF8FEF07
:104A50000E9460A78FEF0E9460A70E9465A78E83C7
:104A60008F71853049F083E18C83CE010E94A124AF
:104A700080E0DF91CF91089581E0FBCF0F931F93EA
:104A8000CF93DF93EC018B010E9457240F946E3C6F
:104A900081110CC085E18C8310E0CE010E94A1241D
:104AA000812FDF91CF911F910F910895A8016CEF95
:104AB000CE010E940F25182F882361F3EECF0F93AC
:104AC0001F93CF93DF93EC0189018F81833039F0FD
:104AD00089E0440F551F661F771F8A95D1F79A0109
:104AE000AB0168E1CE010E94632481112AC0A801B4
:104AF0006EEFCE010E940F25182F8823B1F00F947E
:104B00006E3C182F8823D1F020E030E0A9016DE041
:104B1000CE010E946324882321F086E18C8310E07B
:104B200004C00E9465A78111F8CFCE010E94A12484
:104B3000812FDF91CF911F910F91089587E18C8391
:104B4000F4CF86E0EBCF1F93CF93DF93EC010E946D
:104B5000572420E030E0A9016CE0CE010E946324DC
:104B600011E0882319F010E083E08C83CE010E94CD
:104B7000A124812FDF91CF911F9108951F93CF938F
:104B8000DF93EC018F81833039F089E0440F551FAA
:104B9000661F771F8A95D1F79A01AB0162E1CE01BA
:104BA0000E94632411E0882319F010E085E08C83D3
:104BB000CE010E94A124812FDF91CF911F910895F2
:104BC0008F929F92AF92BF92EF92FF920F931F939B
:104BD000CF93DF938C01EB017A010F943D374B01AA
:104BE0005C012CE2820E21E0921EA11CB11C0E94ED
:104BF00065A7F80186838F3F69F40F943D376819E4
:104C000079098A099B0997FDF2CF81E1F801848334
:104C1000C0E021C08E3F71F5F1E0EF1AF1088FEF8F
:104C20008EBDFE012FEF0DB407FEFDCF8EB5819333
:104C30002EBDCF018C1B9D0B8E159F05A0F30DB4CF
:104C400007FEFDCF8EB5CE0DDF1D88830E9465A7C0
:104C50000E9465A7C1E0C8010E94A1248C2FDF91AA
:104C6000CF911F910F91FF90EF90BF90AF909F90C9
:104C70008F9008958FE0CACF0F931F93CF93DF9348
:104C8000EC018B010E94572440E052E0B801CE01B4
:104C9000DF91CF911F910F910C94E0250F931F93FB
:104CA000CF93DF93EC0189018F81833039F089E064
:104CB000440F551F661F771F8A95D1F79A01AB01E4
:104CC00061E1CE010E94632481110AC040E052E0FC
:104CD000B801CE01DF91CF911F910F910C94E02587
:104CE00084E08C83CE010E94A12480E0DF91CF91EB
:104CF0001F910F9108958F929F92AF92BF92CF9282
:104D0000DF92EF92FF920F931F93CF93DF93EC010B
:104D1000162F1F821C824B830F943D376B017C0141
:104D200020EDC20E27E0D21EE11CF11CA89561E027
:104D30008B810F9431358B810F94CA1B209A289A4E
:104D4000219A2398229A81E00E946CA785E08D83A6
:104D50000E946CA70AE08FEF0E9460A70150D9F76C
:104D6000A89520E030E0A90160E0CE010E94632414
:104D70008E83813081F00F943D376C197D098E0947
:104D80009F0997FDEECF81E08C83CE010E94A12484
:104D90001A8280E06AC0A8952AEA31E040E050E03B
:104DA00068E0CE010E946324853041F581E08F8365
:104DB000A8958F81812C912C5401823029F4812C6B
:104DC000912CA12C80E4B82E20E030E0A90167E30B
:104DD000CE010E946324A501940169E2CE010E94E4
:104DE00063248E838823F1F00F943D376C197D097D
:104DF0008E099F0997FDE8CF8AE0C6CF04E00E94A4
:104E000065A78E830150D9F78A3A11F482E0CFCF9B
:104E10000F943D376C197D098E099F0997FDBCCF12
:104E200082E0B2CF8F818230C1F420E030E0A9016E
:104E30006AE3CE010E946324882311F088E0A4CFA6
:104E40000E9465A7807C803C11F483E08F830E94E0
:104E500065A70E9465A70E9465A7CE010E94A124B4
:104E600081E08A83173070F41D83DF91CF911F9109
:104E70000F91FF90EF90DF90CF90BF90AF909F90F9
:104E80008F90089588E18C8384CF0F931F93CF93E5
:104E9000DF93EC018B0120E030E0A90169E00E9482
:104EA000632481110AC040E150E0B801CE01DF91D6
:104EB000CF911F910F910C94E02580E18C83CE015E
:104EC0000E94A12480E0DF91CF911F910F9108955E
:104ED000CF93C82FCB010E94399288EE97E00E94B1
:104EE000399289ED97E0CC2311F08EED97E00E9486
:104EF00039928AE0CF910C9411920F931F93CF9324
:104F0000811113C0C42F8B010E94CAA187EA9BE0C4
:104F10000E943992C8010E943992CC2331F08AE074
:104F2000CF911F910F910C941192CF911F910F91DE
:104F300008950D9449370D944937CF93DF938091AD
:104F40008A1590918B15891B80958F7019F40E949A
:104F500087A7F5CF80918A158F5F8F70A0918A15F2
:104F60009BE6A99FD0011124FD01EC5BF64FEF01F8
:104F700019929A95E9F798E09083A75AB64F90E175
:104F8000ECE9F5E101900D929A95E1F720918A15EF
:104F900090918B15291303C094E690938715809305
:104FA0008A15DF91CF910C942A8F0F9300912604DC
:104FB00021E002272BE834E04CE050E0BC0185E81A
:104FC00094E00E94E68F0F9108950F9300912604BC
:104FD00021E002272BE834E044E050E0BC0185E802
:104FE00094E00E94E68F0F9108950F93009126049C
:104FF00021E002272BE834E041E050E0BC0185E8E5
:1050000094E00E94E68F0F9108950F93009126047B
:1050100021E002272BE834E042E050E0BC0185E8C3
:1050200094E00E94E68F0F9108950F93009126045B
:1050300021E002272BE834E041E050E0BC0185E8A4
:1050400094E00E94E68F0F9108950F93009126043B
:1050500021E002272BE834E048E050E0BC0185E87D
:1050600094E00E94E68F0F9108950F93009126041B
:1050700021E002272BE834E04CE050E0BC0185E859
:1050800094E00E94E68F0F9108950F9301E02BE8C2
:1050900034E041E050E0BC0185E894E00E94E68FF6
:1050A0000F9108950F93AB010091260421E0022790
:1050B0002BE834E0BC0185E894E00E94E68F0F9174
:1050C00008952BE834E042E050E0BC0185E894E02C
:1050D0000C94E0A52BE834E04CE050E0BC0185E8FE
:1050E00094E00C94E0A52BE834E044E050E0BC01EF
:1050F00085E894E00C94E0A52BE834E041E050E032
:10510000BC0185E894E00C94E0A52BE834E041E094
:1051100050E0BC0185E894E00C94E0A52BE834E075
:105120004CE050E0BC0185E894E00C94E0A561E01F
:105130008AE997E00C94ED8D20E040E070E060E0BB
:105140008BE49AE20C94D7D880914109811114C064
:1051500080917C0290917D02019720910A153091F7
:105160000B152817390744F420E040E070E060E0B8
:1051700080E59AE20C94D7D80C949C2821E02093E7
:105180009803FC0180819181A281B3818093000208
:1051900090930102A0930202B093030220E040E04A
:1051A00070E060E080919807909199070C94D7D8AF
:1051B000CF93DF9300D01F92CDB7DEB78DEC9CEC80
:1051C000ACECBCE389839A83AB83BC83CE010196AC
:1051D0000E94BE280F900F900F900F90DF91CF91FB
:1051E0000895CF93DF9300D01F92CDB7DEB78DEC3B
:1051F0009CECACECBDE389839A83AB83BC83CE018A
:1052000001960E94BE280F900F900F900F90DF9193
:10521000CF910895CF93DF9300D01F92CDB7DEB723
:1052200080E090E0A0E8BFE389839A83AB83BC83EE
:10523000CE0101960E94BE280F900F900F900F9004
:10524000DF91CF910895CF93DF9300D01F92CDB718
:10525000DEB780E090E0A0E2B1E489839A83AB837B
:10526000BC83CE0101960E94BE280F900F900F9034
:105270000F90DF91CF9108956FEF80919A070D9471
:10528000F0347F928F929F92AF92BF92CF92DF9233
:10529000EF92FF920F931F93CF93DF93C0919A07E2
:1052A00061E081E00E947FD870909707D0E0CC0F3A
:1052B000DD1FC85AD84F10E09EE3E92E97E0F92E83
:1052C0002CE3C22E29E2D22E30E3A32E37E0B32EF8
:1052D00045E6842E47E0942E711035C080919607E4
:1052E0008823B9F080917702882361F081E0909162
:1052F0009607911180E003E023E04CE457E0612F32
:105300000E9478ED73941F5F143031F7109391076A
:105310000CC08091900710929007882319F30E9487
:105320007CDA8091B1078823E9F2DF91CF911F9158
:105330000F91FF90EF90DF90CF90BF90AF909F9034
:105340008F907F90089581E078122BC0FE018591A7
:10535000949190939A03809399038091960781305A
:1053600081F080917702882369F21F929F928F9239
:105370001F9381E090919607913009F474C080E00A
:1053800072C08091900710929007882351F380910A
:105390009A07682F0F94F0348091B107882309F39E
:1053A000C4CF82E0781242C0FE018591949190931F
:1053B0009A0380939903809196078230D1F080916F
:1053C0007702882309F49ECFDF92CF92BF92AF92EB
:1053D0001F9381E090919607923009F080E08F93BF
:1053E0000E94BBFD0F900F900F900F900F900F90A9
:1053F00089CF8091900710929007882301F30E9433
:105400003C298091B1078823D1F28FCF80919007FA
:10541000109290078823C1F060919A078FEF0F9444
:10542000F0348091B107882379F07FCF83E0781240
:1054300069CFFE018591949190939A03809399038B
:1054400080919607833011F380917702882309F4C5
:1054500059CF1F92FF92EF921F9381E09091960790
:10546000933009F08CCF8F930E94BBFD0F900F906B
:105470000F900F900F9046CF68ED73E682E00D9489
:10548000CB4C6DED73E681E00D94CB4C62EE73E690
:1054900080E00D94CB4C6FE871E683E00D94CB4C2B
:1054A000CF92DF92EF92FF920F931F9387E5C82E62
:1054B00086E0D82EF12CE12C09E516E02AE231E055
:1054C0004CE958E269E676E08EE696E00E94BAE0A2
:1054D0001F910F91FF90EF90DF90CF900895AF92C2
:1054E000BF92CF92DF92EF92FF920F931F93CF93D1
:1054F000DF93CDB7DEB7ADB6BEB68091B21269EE1E
:1055000077E0882311F062EB72E1FB01019000204B
:10551000E9F7CF01861B970B01962DB73EB7281BE5
:10552000390B0FB6F8943EBF0FBE2DBF8DB79EB797
:1055300001967C0180E2EDB7FEB78183C701019639
:105540000F948F658DE1C82E86E0D82E0FE116E00E
:105550002AE231E042EC5AE26BE276E082E396E046
:105560000E94BAE00FB6F894BEBE0FBEADBEDF918A
:10557000CF911F910F91FF90EF90DF90CF90BF9050
:10558000AF90089589EE97E00F945F3F0E94B9D9DC
:105590000D941D2E0F931F93CF93DF93FC01238156
:1055A000222331F080E0DF91CF911F910F91089578
:1055B0008B01EC01FB018789803139F582E08B8317
:1055C0001D8A1E8A1F8A188E808D918DB0E0A0E002
:1055D00025E0880F991FAA1FBB1F2A95D1F7898B39
:1055E0009A8BAB8BBC8B1A8F098F81E089831886CD
:1055F00019861A861B861C821D821E821F82188AAB
:105600001C861D861E861F86CECF803259F683E00B
:105610008B83428D538D648D758D4D8B5E8B6F8B1F
:10562000788F9E012F5E3F4FC8010F946B4381110D
:10563000DACFB8CFCF93DF93EC010F94E1431B8215
:10564000DF91CF910895CF93DF93EC01462F417006
:105650006C857D858E859F850F944840882351F009
:10566000888920E2829FC00111248C509D4EDF91D9
:10567000CF91089590E080E0FACFCF93DF93EB01D4
:10568000FC012381211104C080E0DF91CF910895B6
:105690002250223028F48FE28883198281E0F5CFEE
:1056A00060E00E94232B009779F3DC0160E080E04A
:1056B0009EE22D91203299F0883031F49E01260F20
:1056C000311DF90190836F5F9E01260F311DAD01E1
:1056D00041505109FA014081F90140836F5F8F5FAA
:1056E0008B3039F7FE01E60FF11D1082D7CF3F92C4
:1056F0004F925F926F927F928F929F92AF92BF92E2
:10570000CF92DF92EF92FF920F931F93CF93DF938D
:10571000CDB7DEB72C970FB6F894DEBF0FBECDBF66
:105720005C01DC0159968D909C90F40181859285F5
:10573000A385B4859C01AD012F5F3F4F4F4F5F4F55
:1057400029873A874B875C87D50114964D905D90E9
:105750006D907C901797411451046104710409F411
:1057600059C0BFEF4B1A5B0A6B0A7B0A312C7301DD
:1057700062011D821E821F821886F4018185928536
:10578000A385B4852D813E814F815885281739071F
:105790004A075B0708F056C089859A85AB85BC85AA
:1057A0008C159D05AE05BF0550F482E0C82ED12CA6
:1057B000E12CF12C92E0492E512C612C712C9E0190
:1057C0002F5F3F4FB701A601C4010F94E842882321
:1057D000C9F189819A81AB81BC81892B8A2B8B2B62
:1057E00001F1260137019FEF491A590A690A790A1E
:1057F0002D813E814F8158852F5F3F4F4F4F5F4F27
:105800002D833E834F8358873FEFC31AD30AE30AA1
:10581000F30AB3CF40805180628073803324339485
:10582000A6CFC414D504E604F70411F70FEF1FEF59
:105830002FEF3FE0B701A601C4010F945642782E26
:1058400081111AC0712C872D2C960FB6F894DEBFEB
:105850000FBECDBFDF91CF911F910F91FF90EF90C1
:10586000DF90CF90BF90AF909F908F907F906F9080
:105870005F904F903F900895F50144815581668176
:105880007781411551056105710539F09701860150
:10589000C4010F9456428823A9F2D5011496CD92E3
:1058A000DD92ED92FC921797332051F0D701C6019B
:1058B0000196A11DB11DF40180839183A283B3835E
:1058C000F50185899689A789B08D892B8A2B8B2B29
:1058D00009F0B9CFC58AD68AE78AF08E81818068BF
:1058E0008183B1CF40E050E0BA010D9430444F9233
:1058F0005F926F927F92AF92BF92CF92DF92EF92C0
:10590000FF920F931F93CF93DF931F92CDB7DEB714
:105910008C017B015A01C22EDB0159968D919C911D
:10592000F801928F818FCB010E94722C712CF701AC
:1059300080859185A285B38541895289638974895F
:1059400084179507A607B70708F052C055E0B6952B
:10595000A795979587955A95D1F7F82FFF70DF2E69
:10596000D70113968C91823010F480E0DBC041E0C7
:1059700050E0BE016F5F7F4FC7010F9492470197C0
:10598000A1F7F70180859185A285B3854F96A11D6A
:10599000B11D80879187A287B387F0E2DF9EB001B7
:1059A00011246C507D4E61157105F9F2DB018C916B
:1059B000882341F0853E09F04CC0772029F07724F8
:1059C0007394B5CF71100EC08091F4149091F514BA
:1059D000A091F614B091F714F80184879587A687F3
:1059E000B787D08ADB018C918111E9CF772473943A
:1059F0008C2D8274823409F0B8CF772009F4A2C0CC
:105A0000F801D08861E0C8010E94232B009709F4B7
:105A1000ACCF20E2DC011D922A95E9F72BE0F501DD
:105A2000DC0101900D922A95E1F721E238E2FC01B8
:105A3000318B208B40E058E057874687338B228B91
:105A4000318F208F578B468B0F94FF3F811109C0F8
:105A50008CCF4BE050E0C5010F945065892B09F0C5
:105A600066CFF0E2DF9ED00111249D012C503D4E07
:105A7000F9018385817121F08C2D827109F001C1BA
:105A8000F801818D928D4091F4145091F51460913C
:105A9000F6147091F7144487558766877787D08A04
:105AA000FD01EC50FD4E44885588712C612C32016B
:105AB00055244424D80155964D925D926D927C9266
:105AC0005897428D538D70E060E04429552966292E
:105AD000772955964D935D936D937C935897D90193
:105AE0001B962C91287109F0BEC0848D958DA68DD2
:105AF000B78DF801818B928BA38BB48B81E083836C
:105B00008C2D8F70F8018183148215821682178282
:105B1000108611861286138681E0C4FE03C0C80178
:105B20000F94C4440F90DF91CF911F910F91FF907C
:105B3000EF90DF90CF90BF90AF907F906F905F908D
:105B40004F900895D70113968C911397823009F4E2
:105B50000CCF51968D919D910D90BC91A02D803EC2
:105B60009F4FAF41B10508F000CFC7010E94772BCE
:105B7000882309F4FACE0F94FF3F882309F4F5CE69
:105B8000D7015996ED91FC915A9714964D905D90DE
:105B90006D907C901797B2E04B1A5108610871081C
:105BA000858504C0440C551C661C771C8A95D2F769
:105BB00086859785A089B189480E591E6A1E7B1E6D
:105BC00081E08093F8144092F4145092F51460929E
:105BD000F6147092F714E4EFF2E180E092E0DF0156
:105BE0009C011D9221503040E1F7DD24D394D70170
:105BF0005996ED91FC918481D816C0F48091F914E6
:105C00009091FA14DC01ED91FC910288F389E02D6A
:105C100024EF32E1B301A2014D0D511D611D711D33
:105C20001995882309F4A1CED394E1CF258580E08E
:105C300092E0A0E0B0E004C0880F991FAA1FBB1F2C
:105C40002A95D2F7F7014189528963897489840FB3
:105C5000951FA61FB71F818B928BA38BB48B84EFEC
:105C600092E1D12CD6CE203161F498012F5E3F4FC6
:105C70000F946B43882329F084E0D80113968C930A
:105C80003FCFD80113961C9270CECF93C82F0E949D
:105C9000CAA184E50E9411928C2F0F947B3E80E272
:105CA0000E9411928DE098E1CF910C9439928F92DD
:105CB0009F92AF92BF92CF92DF92EF92FF92CF93DB
:105CC0006B017C01B42E20E030E0A9010F943F5B12
:105CD00087FF07C08DE20E941192F7FAF094F7F85F
:105CE000F094C0E060E070E080E09FE3CB1541F00D
:105CF0002DEC3CEC4CEC5DE30F94A55BCF5FF6CF55
:105D0000A70196010F9431626B017C010F94A4638B
:105D10004B015C014AE00F94143ECC2379F1C5019C
:105D2000B4010F94445B9B01AC01C701B6010F9411
:105D300030626B017C018EE20E941192C150F0F042
:105D400020E030E040E251E4C701B6010F94A55BCA
:105D50006B017C010F94A4634B015C014AE00F943A
:105D6000143EC501B4010F94445B9B01AC01C70113
:105D7000B6010F9430626B017C01E0CFCF91FF90B0
:105D8000EF90DF90CF90BF90AF909F908F9008954D
:105D9000EF92FF920F931F93CF937C018B01C2E48C
:105DA0004F3F09F0C4E580E20E9411928C2F0E94BF
:105DB00011928AE30E941192F701608171818281C0
:105DC000938142E00E94572E89EF97E10E94399219
:105DD000F801608171818281938142E00E94572E97
:105DE00062E070E080E090E0CF911F910F91FF9012
:105DF000EF900D940A371F93CF93DF9300D000D01C
:105E00001F921F92CDB7DEB7182F60910C157091BD
:105E10000D15072E000C880B990B0F94465B6D83B4
:105E20007E838F83988760910A1570910B15072EDA
:105E3000000C880B990B0F94465B69837A838B83E4
:105E40009C834AEFBE016B5F7F4FCE0101960E949B
:105E5000C82E6091030870910408072E000C880B6F
:105E6000990B0F94465B6D837E838F839887609137
:105E7000010870910208072E000C880B990B0F94F3
:105E8000465B69837A838B839C834FEFBE016B5F94
:105E90007F4FCE0101960E94C82E609105081F3FDA
:105EA00039F085E11802F0011124EA5FFA4E6085AD
:105EB00070E081E098E10E94EE946091050870E046
:105EC0008CEF97E10E94EE9428960FB6F894DEBF0F
:105ED0000FBECDBFDF91CF911F9108952F923F92BA
:105EE0004F925F926F927F928F929F92AF92BF92EA
:105EF000CF92DF92EF92FF920F931F93CF93DF9396
:105F0000CDB7DEB764970FB6F894DEBF0FBECDBF36
:105F1000898B6A8B81E0809367021A821B821C82C4
:105F20001D8219861A861B861C861D862CE32E87E9
:105F30003CE13F8746E4488B312C212C50E85B8BB9
:105F40008FEB8C8B198291E09887812C912C5401D6
:105F50000091030810910408B801012E000C880B71
:105F6000990B0F94465B6B017C01232D322D4B89DD
:105F70005C890F943F5B882389F0809101089091A0
:105F80000208A989A111F1C0B1E0B9830817190766
:105F90000CF019823C2C2D2CEB8AFC8A0F943D3797
:105FA0006B017C01DC01CB0129853A854B855C8541
:105FB000821B930BA40BB50BB7FD2FC0D701C601F5
:105FC00088519C4FAF4FBF4F89879A87AB87BC875B
:105FD00080E00E94FB2E89E098E10E9439928114B2
:105FE0009104A104B10409F4ECC0C501B4016857DF
:105FF0007C4E8F4F9F4F6C197D098E099F0928EEAB
:1060000033E040E050E00F948361CA01B9014AE0F7
:106010000E9418928AE00E94119280E00E9487A755
:106020000F943D376093D3077093D4078093D507BF
:106030009093D6076091010870910208072E000C1A
:10604000880B990B0F94465B6E837F838C019B01B9
:10605000AC01632D722D8B899C890F9430622B01CA
:106060003C0120E030E0A9010F94916487FF04C057
:1060700077FA709477F8709481149104A104B104B4
:1060800009F0A3C020E030E040E85FE3C301B201C3
:106090000F943F5B87FF10C09885812C912C540191
:1060A000992331F082E8882E86E0982EA12CB12C1D
:1060B0008C0C9D1CAE1CBF1CA981AA2391F12A81C6
:1060C0003B814C815D81211531054105510541F030
:1060D000D701C601821B930BA40BB50BB7FD21C0E2
:1060E0002E813F81A8016D857E858F8598890F94CB
:1060F000306220E030E040E85FE30F943F5B87FDD3
:1061000037C0D701C601805A9541AF4FBF4F8A8330
:106110009B83AC83BD839E819D87AF81AE870F87B4
:10612000188BBA89BB2351F0809190071092900789
:10613000882321F0109267020F94833780916702C1
:106140008823B1F081149104A104B10461F028E81E
:10615000C21A23E1D20AE108F108C818D908EA08EE
:10616000FB08F7FE05C01886F3CE081719071CF5C3
:10617000209167022983222321F0109267020F9455
:106180001D2E898164960FB6F894DEBF0FBECDBF79
:10619000DF91CF911F910F91FF90EF90DF90CF9003
:1061A000BF90AF909F908F907F906F905F904F9037
:1061B0003F902F9008953C2C2D2CEB8AFC8A19825D
:1061C000EDCE8FE30E94119225CF20E030E040E435
:1061D00050E4C301B2010F94916418160CF06CCF17
:1061E0004601570169CF2F923F924F925F926F9273
:1061F0007F928F929F92AF92BF92CF92DF92EF9257
:10620000FF920F931F93CF93DF93CDB7DEB76697BF
:106210000FB6F894DEBF0FBECDBF8A8B6B8B4C8B55
:1062200020913C04298B10923C0481E0809367020A
:106230001A821B821C821D8219861A861B861C8666
:106240001D863CE33E874CE14F8756E4588B312C4A
:10625000212C80E88D8B9FEB9E8B1982A1E0A88773
:10626000812C912C540100910C1510910D15B80141
:10627000012E000C880B990B0F94465B6B017C017F
:10628000232D322D4D895E890F943F5B882389F041
:1062900080910A1590910B15BB89B111F1C021E0D5
:1062A0002983081719070CF019823C2C2D2CED8A34
:1062B000FE8A0F943D376B017C01DC01CB012985FF
:1062C0003A854B855C85821B930BA40BB50BB7FD00
:1062D0002FC0D701C60188519C4FAF4FBF4F898750
:1062E0009A87AB87BC878A890E94FB2E85E098E15C
:1062F0000E94399281149104A104B10409F4EFC001
:10630000C501B4016053784F8F4F9F4F6C197D09C1
:106310008E099F0928EE33E040E050E00F9483613E
:10632000CA01B9014AE00E9418928AE00E941192C3
:1063300080E00E9487A70F943D376093D307709346
:10634000D4078093D5079093D60760910A15709172
:106350000B15072E000C880B990B0F94465B6E8370
:106360007F838C019B01AC01632D722D8D899E89E9
:106370000F9430622B013C0120E030E0A9010F9422
:10638000916487FF04C077FA709477F87094811451
:106390009104A104B10409F0A6C020E030E040E877
:1063A0005FE3C301B2010F943F5B87FF10C0988584
:1063B000812C912C5401992331F08AE9882E82E0B6
:1063C000982EA12CB12C8C0C9D1CAE1CBF1CA9813D
:1063D000AA2391F12A813B814C815D8121153105F0
:1063E0004105510541F0D701C601821B930BA40B57
:1063F000B50BB7FD21C02E813F81A8016D857E853B
:106400008F8598890F94306220E030E040EC5FE3A4
:106410000F943F5B87FD37C0D701C601805A954175
:10642000AF4FBF4F8A839B83AC83BD839E819D8783
:10643000AF81AE870F87188BBC89BB2351F0809149
:10644000900710929007882321F0109267020F9412
:106450008337809167028823B1F081149104A104ED
:10646000B10461F020EDC21A27E0D20AE108F10878
:10647000C818D908EA08FB08F7FE05C01886F3CE4D
:106480000817190734F5309167023983332321F057
:10649000109267020F941D2E398930933C04898134
:1064A00066960FB6F894DEBF0FBECDBFDF91CF91D9
:1064B0001F910F91FF90EF90DF90CF90BF90AF9022
:1064C0009F908F907F906F905F904F903F902F9014
:1064D00008953C2C2D2CED8AFE8A1982EACE8FE39A
:1064E0000E94119222CF20E030E040E450E4C3014A
:1064F000B2010F94916418160CF069CF4601570150
:1065000066CF0F930FB70F9300916E000B7F009330
:106510006E0078940F930BB70F930CB70F921F92E6
:106520002F933F934F935F936F937F938F939F939B
:10653000AF93BF93EF93FF9311240E94553EFF91B9
:10654000EF91BF91AF919F918F917F916F915F91EB
:106550004F913F912F911F900F900CBF0F910BBF48
:106560000F910460F89400936E000F910FBF0F918C
:106570001895CF93DF9310923C04C6E0D5E11F82BB
:106580001E820F94493718862C98CDEFD7E01F82D2
:106590001E820E942A2418868091020180728093B4
:1065A0000001DF91CF9108950E94D08F0E94B932EF
:1065B0000C94B9D94F925F926F927F928F929F9273
:1065C000AF92BF92EF92FF920F931F93CF93DF93FF
:1065D000B0E2A0E06A2F70E0AB014B0F511D559562
:1065E0004795411117C0EDE1F7E185919491282F6E
:1065F000822FDF91CF911F910F91FF90EF90BF906D
:10660000AF909F908F907F906F905F904F90089584
:10661000B42FE2CFA41711F0B41303C0E9E9F7E1F6
:10662000E4CF9A0121503109220F331F220F331F6B
:10663000F901E55EF84EE590F490F901E15EF84E5F
:10664000059114918E159F051CF3A42F08171907A7
:106650000CF4C0CFBC01F901E35EF84EC591D491B2
:10666000F901EF5DF84EA590B4906E197F09072EE1
:10667000000C880B990B0F94465B2B013C01B50174
:106680006C1B7D0B072E000C880B990B0F94465B3F
:106690009B01AC01C301B2010F94A55B4B015C01EE
:1066A000B8016E197F09072E000C880B990B0F9407
:1066B000465B9B01AC01C501B4010F942B634B01F8
:1066C0005C01BE01DD0F880B990B0F94465B9B01AB
:1066D000AC01C501B4010F9431620F949D63262F64
:1066E000972F86CFCF93DF93C6E0D5E18A819B8138
:1066F0000F942B1B9D838C83CDEFD7E08A819B81E8
:106700000E94DA329D838C83A89510923B04DF911E
:10671000CF9108958F929F92AF92BF92CF92DF92C6
:10672000EF92FF920F931F93CF93DF93EC018A01B7
:10673000072E000C880B990B0F94465B4B015C01F4
:10674000C880D980EA80FB80A70196010F949164EC
:1067500018162CF488829982AA82BB8210C0B801D4
:10676000110F880B990B0F94465B4B015C01AC0138
:106770009B01C701B6010F94916418165CF3DF9179
:10678000CF911F910F91FF90EF90DF90CF90BF902E
:10679000AF909F908F900895EF92FF920F931F9369
:1067A000CF93DF93C82F7B018A01809183078130CB
:1067B000A1F40E94C6A1C7010E94399281ED96E121
:1067C0000E943992C7FD33C08C2F0C2E000C990B00
:1067D0000F94C31B8AE00E9411920E94B932A895BF
:1067E0008091FC04811138C081E08093FC0480E832
:1067F000809383070E94B932D5E1D150409AE1F0ED
:1068000069E170E080E090E00F940A37A895409825
:1068100068E270E080E090E00F940A37A89568E2A3
:1068200070E080E090E00F940A37A895E6CF8DECF9
:1068300096E10E943992CECF66EC76E1CF3F11F01F
:106840006AEC76E140E0C801DF91CF911F910F9192
:10685000FF90EF900C9462A5DF91CF911F910F9163
:10686000FF90EF9008952F923F924F925F926F9218
:106870007F928F929F92AF92BF92CF92DF92EF92D0
:10688000FF920F931F93CF93DF9300D0CDB7DEB766
:106890009B838A836B015A0129831801870181E058
:1068A00090E02F3F11F090E080E025E0289FF0017C
:1068B000299FF00D1124EF5CFB4F8481882309F49C
:1068C0008FC0EA81FB81148215821682178210869E
:1068D000EA81FB8184818230B9F0833009F400C100
:1068E000813009F067C02581368147815085F601E6
:1068F00060817181828193810F943F5B87FD5AC0D3
:1069000082E0EA81FB818483EA81FB818580968035
:10691000A780B084F601C080D180E280F380B80106
:10692000110F880B990B0F94465B2B013C01809152
:1069300037028823F9F0F981F1111CC080912F09E9
:106940008823A9F020E030E040E85EE3C301B20113
:106950000F94A55B9B01AC01C501B4010F9430629B
:10696000A70196010F943F5B18160CF464C080E8F1
:1069700080933502A3019201C501B4010F943062E6
:10698000A70196010F943F5B18160CF499C00F9461
:106990003D376B017C019101A8EEB3E00F94D76104
:1069A000C60ED71EE81EF91EEA81FB81C082D18285
:1069B000E282F3820F900F900F90DF91CF911F91A1
:1069C0000F91FF90EF90DF90CF90BF90AF909F908E
:1069D0008F907F906F905F904F903F902F90089591
:1069E000F5014080518062807380A3019201EA81A9
:1069F000FB8165817681878190850F943F5B882339
:106A000009F466CFEA81FB814582568267827086EF
:106A1000FF24F39420E030E0A901F5016081718149
:106A2000828193810F94916418160CF0F12CEA8105
:106A3000FB81F4824DCF23E830EC4AEA5EE3C301E8
:106A4000B2010F94A55B9B01AC01C501B4010F9489
:106A50003062A70196010F943F5B181614F080E690
:106A600087CF20E030E040E05FE3C301B2010F9444
:106A7000A55B9B01AC01C501B4010F943062A70175
:106A800096010F943F5B181614F080E471CF2DEC43
:106A90003CEC4CE45FE3C301B2010F94A55B9B01A6
:106AA000AC01C501B4010F943062A70196010F94A7
:106AB0003F5B181614F080E25BCF109235025ACF7C
:106AC0000F943D37EA81FB8100811181228133815E
:106AD000601B710B820B930B97FD6CCF83E084835B
:106AE0004BE957E16BEA77E189810F900F900F90A6
:106AF000DF91CF911F910F91FF90EF90DF90CF909A
:106B0000BF90AF909F908F907F906F905F904F90CD
:106B10003F902F900C94CC33CF93DF93EC014881BE
:106B200059816A817B818CEB96E10E94DD944C81D6
:106B30005D816E817F8188EB96E10E94DD944885BE
:106B400059856A857B8589E891E40E94DD948AE015
:106B5000DF91CF910C941192BC012091DD04309112
:106B6000DE044091DD045091DE042417350731F432
:106B700081E02617370709F080E008959A01F1CFE8
:106B80000F930FB70F9300916E000F930B7F00933D
:106B90006E0000916F000D7F00936F000F930BB795
:106BA0000F930CB70F921F922F933F934F935F93C6
:106BB0006F937F938F939F93AF93BF93EF93FF93C5
:106BC00011240E94F23FFF91EF91BF91AF919F91ED
:106BD0008F917F916F915F914F913F912F911F9076
:106BE0000F900CBF0F910BBF0F910260F8940093B0
:106BF0006F000F9100936E000F910FBF0F911895CA
:106C0000000000000000000080913E0780FF21C0CE
:106C1000899A8FEF80938E0480913E07869580FF3E
:106C20001BC08F9A8FEF80938F0480913E078695CB
:106C3000869580FF14C080910B01809582708093AF
:106C400009018FEF80939004000000000000000015
:106C50000895899881E0DECF8F9881E0E4CF80911C
:106C60000B0182708093090181E0ECCFDF92EF92FB
:106C7000FF920F931F93CF93DF93CDB7DEB7C65824
:106C8000D1090FB6F894DEBF0FBECDBFC358DF4F9A
:106C9000188219821A821B82CD57D04080918403BA
:106CA00090918503A0918603B0918703CF57DF4F62
:106CB00088839983AA83BB83C158D04084E690E03F
:106CC000909386048093850410928C0410928B0418
:106CD00010928D042BE834E044E050E0BE016F5781
:106CE0007F4F85E894E00E94E0A580918504909113
:106CF00086040296909386048093850410928C04F7
:106D000010928B0481E0CA57DF4F8883C658D04069
:106D1000CE018A579F4F0E9485282BE834E048E433
:106D200050E066EF7FE085E894E00E94E0A52BE864
:106D300034E040E150E067E179E085E894E00E94CA
:106D4000E0A58AE097EDA3EABCE3C358DF4F888350
:106D50009983AA83BB83CD57D040CE0183589F4FE0
:106D60000E94732883E298E00E948E287E018DE6BF
:106D7000E80EF11C8FEFD7018C93C7010E94852884
:106D800019821A821B821C828E010F5F1F4FC8015D
:106D90000E9473288091F8079091F907A091FA0753
:106DA000B091FB0789839A83AB83BC83C8010E949F
:106DB0007328C358DF4F188219821A821B82CD575D
:106DC000D04083E0F70180838983CE0183589F4FB1
:106DD0000E947328C7010E948528C8010E94852847
:106DE0004AE0D42EDA94DD2031F0CE0183589F4F53
:106DF0000E947328F7CF89E795E10E948E28C35837
:106E0000DF4F188219821A821B82CD57D0403AE098
:106E1000D32EDA94DD2031F0CE0183589F4F0E94AB
:106E20007328F7CF85E0D82ED982D701DC92C8012C
:106E30000E948528C7010E9485282BE834E048E09D
:106E400050E06EE174E085E894E00E94E0A52BE854
:106E500034E048E050E066E174E085E894E00E94A8
:106E6000E0A52BE834E044E650E062EB73E085E80F
:106E700094E00E94E0A519828FEFF7018083C8019A
:106E80000E947C28C7010E9485282BE834E044E05A
:106E900050E06FEC72E085E894E00E94E0A58091FC
:106EA0003F078983C8010E947C282BE834E04CE02E
:106EB00050E064E877E085E894E00E94E0A5198A54
:106EC0001A8A1B8A1C8A80E090E0A0E8BFE38D87C5
:106ED0009E87AF87B88B80910F1590911015A09168
:106EE0001115B091121589839A83AB83BC832CEA68
:106EF00035EC47E25EE360911315709114158091B3
:106F00001515909116150F942B636D837E838F83D7
:106F100098872CEA35EC47E25EE360911715709193
:106F200018158091191590911A150F94A55B698712
:106F30007A878B879C872BE834E044E150E0B801E6
:106F400085E894E00E94E0A584E190E09A8389833B
:106F5000C8010E9461288091060890910708A091BD
:106F60000808B091090889839A83AB83BC832CEA13
:106F700035EC47E25EE360910A0870910B0880915E
:106F80000C0890910D080F942B636D837E838F8383
:106F900098872CEA35EC47E25EE360910E08709129
:106FA0000F0880911008909111080F94A55B6987D4
:106FB0007A878B879C87C8010E946A288CE0E2E868
:106FC000F2E0D80101900D928A95E1F7C8010E9484
:106FD0006A281982C8010E9485288FE790E09A8369
:106FE0008983C8010E946128EEE8F2E0D80101908F
:106FF0000D92DA94E1F72BE834E045E050E0B80177
:1070000085E894E00E94E0A58091B1038983C801DE
:107010000E947C2880E2E3E9F2E0D80101900D9221
:107020008A95E1F72BE834E040E250E0B80185E8CA
:1070300094E00E94E0A5D7011C92C7010E947C2821
:1070400086E198E00E947C2882E198E00E94732803
:10705000C358DF4F188219821A821B82CD57D04045
:10706000CE0183589F4F0E94732880E2F80111924D
:107070008A95E9F72BE834E040E250E0B80185E872
:1070800094E00E94E0A5FE01F99688E0DF011D92E0
:107090008A95E9F744E650E060E070E049835A835E
:1070A0006B837C834D835E836F83788783E090E07E
:1070B000A0E0B0E089879A87AB87BC874D875E8761
:1070C0006F87788B498B5A8B6B8B7C8B8D8B9E8BD0
:1070D000AF8BB88F898F9A8FAB8FBC8F8D8F9E8F20
:1070E000AF8FB8A38EE190E0A0E0B0E089A39AA3AF
:1070F000ABA3BCA38DA39EA3AFA3B8A789A79AA750
:10710000ABA7BCA78DA79EA7AFA7B8AB89AB9AAB1F
:10711000ABABBCAB8DAB9EABAFABB8AF2BE834E049
:1071200040E450E0B80185E894E00E94E0A590E1D9
:10713000D92EF8018D2D11928A95E9F72BE834E0CC
:1071400040E150E0B80185E894E00E94E0A5D80154
:107150001D92DA94E9F72BE834E040E150E0B80101
:1071600085E894E00E94E0A587E299E00E947328F8
:107170002CE0D22EF8018D2D11928A95E9F72BE89B
:1071800034E04CE050E0B80185E894E00E94E0A5CE
:107190008CE6D8011D928A95E9F72BE834E04CE69D
:1071A00050E0B80185E894E00E94E0A589E794E00A
:1071B0000E946A282BE834E048E050E069EA73E076
:1071C00085E894E00E94E0A5F7011192DA94E9F7CE
:1071D000CB57DF4F1882C558D04080E090E0A0E444
:1071E000B0E4ED968CAF9DAFAEAFBFAFED97C701EA
:1071F0000E948E28CE018B579F4F0E948528CE017A
:1072000087589F4F0E94732880918D04811128C058
:10721000009185041091860480918B0490918C04D8
:10722000D7018D939C9384E690E09093860480939D
:1072300085042BE834E044E050E063ED72E085E83B
:1072400094E00E94E0A5C7010E94612891E001340A
:10725000134009F490E080918D04892B80938D0474
:1072600080918D04811105C060E083E89BE00E945D
:10727000D0DA90918D0481E08927CA57DF4F0FB68D
:10728000F894DEBF0FBECDBFDF91CF911F910F915C
:10729000FF90EF90DF900895CF93DF9300D01F927F
:1072A000CDB7DEB780912B07882389F083E390E088
:1072B0009C838B831A8219829E012F5F3F4F40E18E
:1072C00050E06CE277E0CE0103960E94E0A50F90BB
:1072D0000F900F900F90DF91CF910895CF93DF9390
:1072E00000D01F921F92CDB7DEB781E080932B07AD
:1072F00080E1ECE2F7E0DF011D928A95E9F70E9458
:107300004C3986E18D8382E390E09C838B831A82E3
:1073100019829E012F5F3F4F41E050E0BE016B5F3D
:107320007F4FCE0103960E94E0A50F900F900F9023
:107330000F900F90DF91CF910895CF92DF92EF924F
:10734000FF92CF93DF93EC0108960E9489826B0134
:107350007C0120E030E0A9010F943F5B20E030E0A9
:10736000A901882359F0CE010E946E8B9B01AC01CC
:10737000C701B6010F94A55B9B01AC0168857985B7
:107380008A859B850F943062688779878A879B8777
:10739000DF91CF91FF90EF90DF90CF900895833BE6
:1073A00021E0920714F083EB91E090930D15809308
:1073B0000C150D944937AF92BF92CF92DF92EF92A6
:1073C000FF920F931F93CF93DF93C6EFDFE003E0AD
:1073D00019E086E0A82E80E1B82EC12CD12C7601D0
:1073E000C39469917991899199910F94445B28890B
:1073F00039894A895B890F94A55B0F94A463F801CE
:1074000061937193819391938F01C616D706E80615
:10741000F90610F46B017C01AC16BD0611F76FEF95
:107420007FEFCB01A70196010F948361209313098D
:10743000309314094093150950931609DF91CF91A9
:107440001F910F91FF90EF90DF90CF90BF90AF9082
:1074500008950F931F93CF93DF930AE010E1C1E3E8
:10746000D9E0F80121913191419151918F0160E072
:1074700070E080E89FE30F942B636993799389937D
:107480009993F9E0C134DF0761F70F94372DDF914D
:10749000CF911F910F910C94DB3990918A158091B7
:1074A0008B15981306C08091420990914309892B4E
:1074B00021F080E00E9487A7F0CF089590918A156F
:1074C00080918B15981308C08091420990914309CF
:1074D000892B11F40C947D8F80E00E9487A7EECF5A
:1074E000CF92DF92EF92FF92CF93DF932091FC0730
:1074F000222329F1EC0108960E9489826B017C010C
:1075000020E030E0A9010F943F5B20E030E0A901CA
:10751000882359F0CE010E946E8B9B01AC01C701FC
:10752000B6010F94A55B9B01AC01688579858A85BE
:107530009B850F943162688779878A879B87DF9163
:10754000CF91FF90EF90DF90CF9008950F931F930E
:10755000CF93DF9350E0FC01E40FF51F8081440FCF
:10756000551F440F551F47595B4FEA01882329F1E6
:1075700088819981AA81BB81EB01088119812A81C7
:107580003B810097A105B10569F40C591F4F2F4F9E
:107590003F4FDA010D931D932D933C9313978FEF7B
:1075A000808306C0081B190B2A0B3B0B37FDF7CF56
:1075B000DF91CF911F910F910895188219821A823D
:1075C0001B82F6CF2F923F924F925F926F927F92E3
:1075D0008F929F92AF92BF92CF92DF92EF92FF92E3
:1075E0000F931F93CF93DF93CDB7DEB76C970FB692
:1075F000F894DEBF0FBECDBF8C015B015A83498377
:10760000FC01EF5AFF4F208131814281538129874C
:107610003A874B875C87CA01B9010F94445B6B01C1
:107620007C01D5012D913D914D915C910F94A55B0D
:107630000F940F632B013C01E981FA812081318194
:1076400042815381C701B6010F94A55B0F940F636C
:107650004B015C01C301B2010F94A463698B7A8B67
:107660008B8B9C8B683771058105910540F428E769
:1076700030E040E050E0298B3A8B4B8B5C8BC501AE
:10768000B4010F94A4636D877E878F87988B6837CA
:1076900071058105910540F448E750E060E070E035
:1076A0004D875E876F87788BF801E35AFF4F4080E4
:1076B000518062807380C301B2010F94465B69837D
:1076C0007A838B839C8369897A898B899C890F94BF
:1076D000445B6D8B7E8B8F8B988F20E030E0A9010F
:1076E00069817A818B819C810F943F5B882309F4A7
:1076F000E1C1A7019601C701B6010F94A55B4B013B
:107700005C012D893E894F89588DCA01B9010F94BA
:10771000A55B9B01AC01C501B4010F9430624B0124
:107720005C0129813A814B815C81CA01B9010F94C6
:1077300031629B01AC01C501B4010F942B630F941E
:107740000F630F94A4636D837E838F83988766276E
:107750007727CB0164197509860997090F94465B51
:107760004B015C016D857E858F8598890F94445B04
:107770002B013C0120E030E0A901C501B4010F94C8
:107780003F5B882309F49AC1A3019201C301B201AE
:107790000F94A55B698F7A8F8B8F9C8FA7019601C1
:1077A000C701B6010F94A55B9B01AC01698D7A8D71
:1077B0008B8D9C8D0F9430626B017C01A50194012F
:1077C000C501B4010F9431629B01AC01C701B60140
:1077D0000F942B630F94D363D80195968D909D9051
:1077E000AD90BC909897750164012D813E814F81C9
:1077F0005885C21AD30AE40AF50A0F94A463C61A7C
:10780000D70AE80AF90AF7FE8EC02D893E894F890A
:10781000588DCA01B9010F94A55B6B017C012981C8
:107820003A814B815C81CA01B9010F943162698749
:107830007A878B879C8720E030E0A90169817A8173
:107840008B819C810F943F5B882309F43BC1C50168
:10785000B4010F94445B29853A854B855C850F9470
:10786000A55BA70196010F9430626D837E838F83A1
:107870009887A3019201C301B2010F94A55B9B01FC
:10788000AC016D817E818F8198850F9431622B01CF
:107890003C0120E030E040E850E469817A818B814E
:1078A0009C810F94A55B9B01AC01C301B2010F94B5
:1078B0002B630F940F632B013C0120E030E0A90102
:1078C0000F94916418161CF0412C512C3201C30105
:1078D000B2010F94A4636D837E838F83988786168D
:1078E0009706A806B90620F48D829E82AF82B886DC
:1078F0006D817E818F8198850F94445B29853A85BF
:107900004B855C850F94A55BA70196010F943162AE
:107910000F94DF640F94A46369877A878B879C87B1
:10792000C12CD12C760169857A858B859C85298926
:107930003A894B895C89621B730B840B950B0F94FE
:10794000445B29813A814B815C810F942B6320E059
:1079500034E244EF59E40F94A55B0F94A4634B0108
:107960005C0169857A858B859C852D853E854F8553
:107970005889621B730B840B950B0F94445B298110
:107980003A814B815C810F942B6320E034E244EF19
:1079900059E40F94A55B0F94A4632B013C013FE6CF
:1079A00083169104A104B10408F090C0F401EE0F15
:1079B000FF1FEE0FFF1FE155F74F85919591A591A0
:1079C000B4918983292E3A2EBD8B4FE6441651047B
:1079D0006104710408F083C0F201EE0FFF1FEE0F87
:1079E000FF1FE155F74F45915591659174919A01AB
:1079F000CB014D815E816F817885D80199964D9339
:107A00005D936D937C939C974C0D5D1D6E1D7F1D4A
:107A1000F80145A756A767A770ABEB5AFF4F4989F6
:107A20005A896B897C894083518362837383D5969D
:107A30008D929D92AD92BC92D897F80141AE52AE14
:107A400063AE74AEFD9649814083218232825D89A6
:107A500053833496208331838283938369857A8527
:107A60008B859C85D1966D937D938D939C93D497B4
:107A700078962D853E854F855889208331834283B2
:107A800053836C960FB6F894DEBF0FBECDBFDF9167
:107A9000CF911F910F91FF90EF90DF90CF90BF900B
:107AA000AF909F908F907F906F905F904F903F909E
:107AB0002F90089560E070E0CB0141CE60E070E06F
:107AC000CB0188CE60E070E0CB01F3CEC501B401FC
:107AD0000E9458226983272E382E9D8B76CFC301B2
:107AE000B2010E9458229B0184CF90916F0081E0E7
:107AF00091FD02C080E0089590916F009D7F90936A
:107B00006F0008950F931F93CF93DF93C82F0E94A8
:107B1000753DD82F4091EC045091ED046091EE0436
:107B20007091EF048091F0049091F104A091F2041F
:107B3000B091F304C13039F58A019B01081B190B80
:107B40002A0B3B0BC901B8010F94465B20E030E0E3
:107B500040E05FE30F94A55B0F949D6314E0C19F29
:107B6000F0011124E052FB4F608371838283938381
:107B700081E08093DF04DD2369F0DF91CF911F91D5
:107B80000F910C942A8F8C019D01040F151F261F45
:107B9000371FD8CFDF91CF911F910F910895CF92CA
:107BA000DF92EF92FF9280913D07811105C0809195
:107BB000D207882309F474C08091560465996AC07D
:107BC000816080935604909103018091560491FF47
:107BD00063C0826080935604809156044B9B5EC0C4
:107BE000846080935604C090D004C0FE12C080917F
:107BF0003E0782958F7080FF0CC08091560480FFF5
:107C000008C08091820781608093820780E00E9493
:107C1000823DD12CF12CE12CD701C601B695A79558
:107C20009795879580FF13C080913E078295869532
:107C3000877080FF0CC08091560481FF08C080913E
:107C4000820782608093820781E00E94823D82E009
:107C5000F694E794D794C7948A95D1F7C0FE20C0D4
:107C600080913E078695869580FF1AC08091D20745
:107C70008823B1F08091560482FF12C08091820760
:107C800084608093820782E0FF90EF90DF90CF9036
:107C90000C94823D8E7F95CF8D7F9CCF8B7FA1CF23
:107CA000FF90EF90DF90CF9008950F931F93CF93A5
:107CB000DF9380913A028F3708F445C08F57909137
:107CC0000E1590932F059923E1F12C9A2091050828
:107CD00020932E059091020121119095907290931E
:107CE00000018F5F80933A0280912D0591E08927F2
:107CF00080932D0581110E9470DB80913902C1E0D3
:107D0000C80F85300CF0C0E0823009F4D8C03CF5D3
:107D10008823D9F1813009F4C6C0C09339020E948A
:107D2000CF3D8091420990914309009729F0019736
:107D30009093430980934209DF91CF911F910F9156
:107D400008952C98C3CF90912F05891708F02C988F
:107D500090912E05891728F290910201BFCF8430AF
:107D600009F4C5C00CF4BEC08530B9F690912C055D
:107D7000911102C080932C0580912C058150809335
:107D80002C05882351F2C5E0C8CF809138028F5F5F
:107D900080311CF480933802C0CF10923802809159
:107DA0003B04811113C080910615909107159093A3
:107DB0000915809308158091FD079091FE07909317
:107DC00000088093FF0781E080933B041092071521
:107DD000109206151092FE071092FD0700910815EB
:107DE0001091091580910C1590910D15D1E0181680
:107DF00019062CF080910E15811101C0D0E0809100
:107E0000610290916202081719073CF44BEB57E1AD
:107E100068EC77E180E00E94CC33DD2371F0809143
:107E20005F0290916002801791073CF44AED57E1A0
:107E300067EE77E180E00E94CC3380910308909157
:107E40000408D1E0181619062CF08091050881115C
:107E500001C0D0E02091FF073091000880912907F0
:107E600090912A07281739073CF44BEB57E168EC4F
:107E700077E18FEF0E94CC33DD2309F44ECF2091C0
:107E8000FF073091000880915D0290915E02821799
:107E900093070CF042CF4AED57E167EE77E18FEFA1
:107EA0000E94CC333ACF88E080937B0085E48093B6
:107EB0007C0080917A00806480937A002ECF80913C
:107EC0007A0086FD27C0209178003091790080915A
:107ED000061590910715820F931F909307158093B5
:107EE00006151BCF88E080937B0086E4E0CF80916D
:107EF0007A0086FD11C02091780030917900809140
:107F0000FD079091FE07820F931F9093FE078093C9
:107F1000FD0703CFC2E001CFC4E0FFCE0E94753D54
:107F200010922B0910922C0910922D0910922E09F3
:107F300081110C942A8F08950F931F9380918A15B5
:107F400090918B15891B8F7009F449C0909187150A
:107F5000992361F0833040F48FEF890F29F08093EB
:107F6000871590E080E038C01092871580918B15BE
:107F70002BE6829FC00111248C5B964FFC0120816F
:107F800020FDEFCF40912B0950912C0960912D09D4
:107F900070912E09ED59FF4F0081118122813381AB
:107FA000401B510B620B730B40932B0950932C0910
:107FB00060932D0970932E0920918B152F5F2F70E0
:107FC0002093881530918B1520918915321304C0A8
:107FD00020918815209389151F910F9108950E9473
:107FE0008E3FBFCF2F923F924F925F926F927F92C0
:107FF0008F929F92AF92BF92CF92DF92EF92FF92B9
:108000000F931F93CF93DF93CDB7DEB76B970FB668
:10801000F894DEBF0FBECDBF8FEF9FEF9093890026
:10802000809388002AE02983312C212C7894809138
:10803000D9049091DA04A091DB04B091DC04892B7F
:108040008A2B8B2B09F0B5C18091DF048823E1F0E6
:108050008091DD049091DE041092DF04892B09F4F5
:10806000A8C11092DE041092DD041092D004909109
:108070008A1580918B15981709F49BC180918B15F7
:108080008F5F8F7080938B158091DD049091DE045B
:10809000892B09F48EC14091D5045091D60460918A
:1080A000D7047091D8048091D1049091D204A0910A
:1080B000D304B091D4040091C70410E030E020E074
:1080C000841B950BA60BB70B081719072A073B074C
:1080D00010F4D901C8018A83840F951FA61FB71F0A
:1080E0008093D5049093D604A093D704B093D8047A
:1080F000E1E000919C0410919D0420919E04309138
:108100009F048091AC049091AD04A091AE04B09115
:10811000AF04080F191F2A1F3B1F0093AC041093D4
:10812000AD042093AE043093AF0437FD33C04091CB
:108130008E04042E000C550B660B770B8091EC041B
:108140009091ED04A091EE04B091EF04840F951F7F
:10815000A61FB71F8093EC049093ED04A093EE0448
:10816000B093EF048091980490919904A0919A049F
:10817000B0919B04B901A801481B590B6A0B7B0BFA
:10818000DB01CA018093AC049093AD04A093AE04CC
:10819000B093AF044091A0045091A1046091A20457
:1081A0007091A3048091B0049091B104A091B204A5
:1081B000B091B304480F591F6A1F7B1F4093B0044E
:1081C0005093B1046093B2047093B30477FD33C04D
:1081D000C0908F040C2C000CDD08EE08FF08809185
:1081E000F0049091F104A091F204B091F3048C0D8D
:1081F0009D1DAE1DBF1D8093F0049093F104A093CC
:10820000F204B093F3048091980490919904A091A2
:108210009A04B0919B044A015B01881A990AAA0A40
:10822000BB0AD501C4018093B0049093B104A0931C
:10823000B204B093B304C090A404D090A504E0901D
:10824000A604F090A7048091B4049091B504A09185
:10825000B604B091B7048C0D9D1DAE1DBF1D80935B
:10826000B4049093B504A093B604B093B704B7FDDB
:1082700033C080909004082C000C9908AA08BB0811
:10828000C090F404D090F504E090F604F090F70468
:10829000C80CD91CEA1CFB1CC092F404D092F50453
:1082A000E092F604F092F704C0909804D0909904FC
:1082B000E0909A04F0909B044C015D018C189D089D
:1082C000AE08BF0875016401C092B404D092B50431
:1082D000E092B604F092B7048090B8049090B9048C
:1082E000A090BA04B090BB04C090A804D090A90498
:1082F000E090AA04F090AB04C80CD91CEA1CFB1C4B
:10830000C092B804D092B904E092BA04F092BB04CF
:10831000F7FC1DC08090980490909904A0909A0456
:10832000B0909B04C818D908EA08FB08C092B804AA
:10833000D092B904E092BA04F092BB04F091C50463
:1083400090903E0793FED2C0F150F093C504E11126
:1083500004C0E0918400F091850037FF889A77FF90
:108360008E9AB7FD06C0E0910B01E095E870E093AE
:108370000901E0918400F0918500E0918400F09182
:10838000850037FF889877FF8E98B7FD05C08091EC
:108390000B01887080930901AA80AA2021F08091A6
:1083A0008400909185002A8121502A83E0E02111E8
:1083B000A0CE8091300290913102A0913202B09112
:1083C0003302892B8A2B8B2B09F0C6C08091C604FF
:1083D000882309F4AEC08091C5048090D5049090A4
:1083E000D604A090D704B090D804C090C104D09017
:1083F000C204E090C304F090C404C814D904EA0491
:10840000FB0408F075C020919204309193044091D0
:108410009604509197044217530708F069C08150A1
:108420008093C50421503109309393042093920422
:1084300080912C0290912D02A0912E02B0912F02DA
:108440002091C504222309F47FC000000000000031
:10845000000012160CF071C0169851E05093910470
:10846000000000000000000021E03091C50433232B
:1084700009F46AC0211104C0209184003091850064
:1084800000919104002E000C110B220B330B409134
:10849000F8045091F9046091FA047091FB04400FC4
:1084A000511F621F731F4093F8045093F9046093A7
:1084B000FA047093FB04149A209184003091850093
:1084C0002091C50427FF3EC02F5F2093C504209153
:1084D00084003091850014982091C504222321F056
:1084E000209184003091850020E0BFCFFF5F2DCF29
:1084F0008C149D04AE04BF0488F420919204309142
:10850000930440919404509195042417350730F456
:108510008F5F8093C5042F5F3F4F86CF4FEF5FEF94
:10852000BA0140932C0250932D0260932E02709357
:108530002F028FEF9FEFDC0183CF169A6FEF6093CE
:1085400091048ECF2150C1CF80933002909331029D
:10855000A0933202B093330280906F029090700229
:10856000A0907102B09072028A829B82AC82BD821E
:1085700089288A288B2809F06AC090E080E0FC01F5
:10858000EE0FFF1FDF01A952B84F2D913C9121152D
:10859000310509F446C0823009F037C05091090115
:1085A00052704091080141704093060100000000A4
:1085B0000000000040910B01121613060CF04095CC
:1085C000427040930901000000000000000040914B
:1085D0000B01409548704093090144E04A95000022
:1085E000E9F740910B014870409309010000000039
:1085F0000000000040910B015111409542704093E2
:1086000009010000000000000000E952F84F1216B6
:1086100013060CF0D3C02081318121503109318300
:10862000208301968330910509F0A9CF0E94308FF5
:10863000882309F4C8C080ED97E0A0E0B0E0809303
:108640006F0290937002A0937102B09372028091B6
:10865000D9049091DA04A091DB04B091DC04892B59
:108660008A2B8B2B11F00C942C4BA090DD04B09036
:10867000DE04BB8EAA8EAB2811F40C943F4C4090C4
:10868000D5045090D6046090D7047090D80480919F
:10869000D1049091D204A091D304B091D40448168F
:1086A00059066A067B0608F492C01092DE04109206
:1086B000DD041092D00490918A1580918B15981743
:1086C00011F40C943F4C80918B158F5F8F708093C9
:1086D0008B1510EDC12E17E0D12EE12CF12C8091DD
:1086E000DD049091DE04892B11F00C94244B0E9440
:1086F0009C3F9093DE048093DD04892B11F40C944D
:10870000244B8090DD049090DE049F828E82D40101
:108710008C9183FD02C00C9479495D968D909D905B
:10872000AD90BC909097FD0185899689A789B08D01
:10873000418D528D638D748D2C013D01440E551E6B
:10874000661E771E4092EC045092ED046092EE0497
:108750007092EF04841B950BA60BB70B8093F0046B
:108760009093F104A093F204B093F3048092F40484
:108770009092F504A092F604B092F70481A192A120
:10878000A3A1B4A18093F8049093F904A093FA04F0
:10879000B093FB041092DE041092DD041092D0041A
:1087A00090918A1580918B15981709F4A0CF80912C
:1087B0008B158F5F8F7080938B1599CF20813181BE
:1087C0002F5F3F4F2CCF8FEF9FEFDC0138CF809191
:1087D000CC049091CD04A091CE04B091CF04841527
:1087E0009505A605B70508F438C24091C804509114
:1087F000C9046091CA047091CB04EA8DFB8D85A9F0
:1088000096A9A7A9B0AD481759076A077B0708F0D2
:10881000FAC1411551056105710509F08FC08090BD
:108820002B0490902C04A0902D04B0902E0488E985
:1088300096E1A1E0FC01059115912591349108156F
:1088400019052A053B0558F4B694A7949794879484
:10885000AA0F0496E4EBF6E1E817F90759F7A0939D
:10886000C704F0E28F169104A104B10428F4A0E239
:108870008A2E912CA12CB12C20E2821A9108A108F9
:10888000B108811438E09306A104B10408F4C4C10E
:10889000A4E09A9EC001112488569D4EFC01329698
:1088A00025913491B82DEE27B39F8001B29F010D21
:1088B0001E1F06940E1F1E1F112430E020E0FC0135
:1088C000C590D490F12CE12CC01AD10AE20AF30A27
:1088D0004C0D5D1D6E1D7F1D4093C8045093C9044F
:1088E0006093CA047093CB048091C5049091C60430
:1088F000992309F43FC4882309F4F1CE2A8D3B8DD6
:10890000295B3F4FD9018D919C91B0E0A0E040914F
:108910002C0250912D0260912E0270912F0284172B
:108920009507A607B70709F4DACE10923002109225
:1089300031021092320210923302D1CEF12C0A850C
:10894000942F852E862F1B85BC85AD85FE85EF85F2
:1089500038892989E0912704E99FA12DFF273091CB
:108960002804399FA00DF11D10902904199EF00DC7
:10897000E89DA00DF11D389DF00DE89FF00D1A2F18
:10898000BF2F1A9FE12D332722271F9FE00D311D96
:108990002F1DBA9FE00D311D2F1DBF9F300D211DD2
:1089A000132FB22F1A9F012D332722271F9F000D4F
:1089B000311D2F1DBA9F000D311D2F1DBF9F300D82
:1089C000211D132FB22FEE2790912B0480902C04A1
:1089D00080912D0400903C050F2809F484C030914B
:1089E0003805319FE1199F098F088F0920913905BA
:1089F000219FE01991098F088F0900913A05019F85
:108A0000901981088F093B9FE01991098F088F0900
:108A10002B9F901981088F090B9F801881091A9F3D
:108A2000012D332722271F9F000D311D2F1DBA9FB7
:108A3000000D311D2F1DBF9F300D211D132FB22F93
:108A400030913405319FE10D9F1D8F1C8F1D2091AA
:108A50003505219FE00D911D8F1C8F1D009136055E
:108A6000019F900D811C8F1D3B9FE00D911D8F1C60
:108A70008F1D2B9F900D811C8F1D0B9F800C811DC6
:108A80001A9F012D332722271F9F000D311D2F1DF7
:108A9000BA9F000D311D2F1DBF9F300D211D132FBB
:108AA000B22F30913005319FE1199F098F088F094E
:108AB00020913105219FE01991098F088F090091BC
:108AC0003205019F901981088F093B9FE019910998
:108AD0008F088F092B9F901981088F090B9F801891
:108AE00081090C94F54530913805319FE10D9F1DAA
:108AF0008F1C8F1D20913905219FE00D911D8F1C2A
:108B00008F1D00913A05019F900D811C8F1D3B9F89
:108B1000E00D911D8F1C8F1D2B9F900D811C8F1DB3
:108B20000B9F800C811D1A9F012D332722271F9F29
:108B3000000D311D2F1DBA9F000D311D2F1DBF9F30
:108B4000300D211D132FB22F30913405319FE119C3
:108B50009F098F088F0920913505219FE019910900
:108B60008F088F0900913605019F901981088F09A0
:108B70003B9FE01991098F088F092B9F901981085D
:108B80008F090B9F801881091A9F012D33272227F7
:108B90001F9F000D311D2F1DBA9F000D311D2F1D70
:108BA000BF9F300D211D132FB22F30913005319F03
:108BB000E10D9F1D8F1C8F1D20913105219FE00D20
:108BC000911D8F1C8F1D00913205019F900D811CFE
:108BD0008F1D3B9FE00D911D8F1C8F1D2B9F900DB6
:108BE000811C8F1D0B9F800C811D11240A871B8700
:108BF000BC87AD87FE87EF87388B298B982C892E11
:108C0000B12CA82E14CEAA8DBB8DD1968D909D909F
:108C1000AD90BC90D4970BCED501C401B695A79565
:108C2000979587958C7F8856914FFC01C590D4907D
:108C3000FC01329625913491E82DE770E29FC00146
:108C4000E39F900D1124F3E096958795FA95E1F74F
:108C5000C81AD90AF12CE12C3BCE8090C104909027
:108C6000C204A090C304B090C4048E829F82A886E0
:108C7000B98684149504A604B70408F07FC28090D6
:108C8000BC049090BD04A090BE04B090BF0480913D
:108C9000C004EA8DFB8D8111C4C0EF5BFF4FE08003
:108CA000F18002811381EA8DFB8DE75AFF4F20810D
:108CB000318142815381AA8DBB8DD1966D917D9179
:108CC0008D919C91D4970E940622B1E0B093C0048C
:108CD000EA8DFB8D81A992A9A3A9B4A928E936E15F
:108CE00011E0F90145915591659174914817590723
:108CF0006A077B0770F4B695A79597958795110F2E
:108D00002C5F3F4F44EBC42E46E1D42EC216D3064F
:108D100041F71093C70480329105A105B10520F4F5
:108D200080E290E0A0E0B0E08097A109B109811550
:108D300028E09207A105B10508F4F9C144E0949F29
:108D40009001112428563D4EF901329645915491D7
:108D5000EE27859FB001849F610D7E1F06946E1FD4
:108D60007E1F1124CB01B0E0A0E0F901C590D490A2
:108D7000F12CE12CC81AD90AEA0AFB0A8C0C9D1CBA
:108D8000AE1CBF1C8092BC049092BD04A092BE0495
:108D9000B092BF048091C604882309F4E9C18E8192
:108DA0009F81A885B985810F911DA11DB11D8415D5
:108DB0009505A605B705D8F48091C504882309F464
:108DC0008ECCEA8DFB8DE95BFF4F80819181B0E015
:108DD000A0E040912C0250912D0260912E027091E2
:108DE0002F0284179507A607B70709F478CC1092CD
:108DF00030021092310210923202109233026A8DC8
:108E00007B8D695B7F4FDB018D919C91B0E0A0E091
:108E100080932C0290932D02A0932E02B0932F02E8
:108E20005ECC81AD92ADA3ADB4AD88169906AA060D
:108E3000BB0608F073C181149104A104B10449F484
:108E400080912B0490912C04A0912D04B0912E04BC
:108E500045CFB0E0AA89282D892D1A2DFB89EC89F0
:108E60007D896E895F89488D398D50912704529F85
:108E7000712D662740912804429F700D611D10904E
:108E80002904129E600D589F700D611D489F600D52
:108E9000519F600DF72FE62FF79F512D4427332761
:108EA000F69F500D411D3B1FE79F500D411D3B1F7D
:108EB000E69F400D311DF42FE32FF79FA12D44278E
:108EC0003327F69FA00D411D3B1FE79FA00D411DBD
:108ED0003B1FE69F400D311DF42FE32F55272091B6
:108EE0002B0480912C0410912D0400903C050B2A3A
:108EF00009F484C0409138054F9F51192B0B8B0BFF
:108F00001B0B309139053F9F501921098B0B1B0B0F
:108F1000A0913A05AF9F201981091B0B4E9F501954
:108F200021098B0B1B0B3E9F201981091B0BAE9F48
:108F300080191109F79FA12D44273327F69FA00D13
:108F4000411D3B1FE79FA00D411D3B1FE69F400DAC
:108F5000311DF42FE32F409134054F9F510D2B1FEE
:108F60008B1F1B1F309135053F9F500D211D8B1FFF
:108F70001B1FA0913605AF9F200D811D1B1F4E9F0B
:108F8000500D211D8B1F1B1F3E9F200D811D1B1F80
:108F9000AE9F800D111DF79FA12D44273327F69F0B
:108FA000A00D411D3B1FE79FA00D411D3B1FE69FEC
:108FB000400D311DF42FE32F409130054F9F511983
:108FC0002B0B8B0B1B0B309131053F9F5019210947
:108FD0008B0B1B0BA0913205AF9F201981091B0B36
:108FE0004E9F501921098B0B1B0B3E9F20198109A5
:108FF0001B0BAE9F801911090C94804840913805D5
:109000004F9F510D2B1F8B1F1B1F309139053F9F09
:10901000500D211D8B1F1B1FA0913A05AF9F200DE6
:10902000811D1B1F4E9F500D211D8B1F1B1F3E9F1F
:10903000200D811D1B1FAE9F800D111DF79FA12DBF
:1090400044273327F69FA00D411D3B1FE79FA00D2E
:10905000411D3B1FE69F400D311DF42FE32F409132
:1090600034054F9F51192B0B8B0B1B0B3091350582
:109070003F9F501921098B0B1B0BA0913605AF9F09
:10908000201981091B0B4E9F501921098B0B1B0BBB
:109090003E9F201981091B0BAE9F80191109F79F74
:1090A000A12D44273327F69FA00D411D3B1FE79FAD
:1090B000A00D411D3B1FE69F400D311DF42FE32FF6
:1090C000409130054F9F510D2B1F8B1F1B1F30915F
:1090D00031053F9F500D211D8B1F1B1FA091320595
:1090E000AF9F200D811D1B1F4E9F500D211D8B1FFB
:1090F0001B1F3E9F200D811D1B1FAE9F800D111D4C
:109100001124AA8BFB8BEC8B7D8B6E8B5F8B488F36
:10911000398F982F822FB0E0A12FE0CDEA8DFB8D03
:10912000E75AFF4F80819181A281B381D7CDAC01F5
:10913000BD0176956795579547954C7F4856514F99
:10914000FA0125913491FA013296659174918770F4
:10915000869FA001879F500D1124B3E05695479537
:10916000BA95E1F7241B350B6901F12CE12C06CEF1
:109170008091C504882309F4B2CAD7CB8091C50475
:109180008823E9F0EA8DFB8DE95BFF4F80819181B7
:10919000B0E0A0E040912C0250912D0260912E028F
:1091A00070912F0284179507A607B70741F0109218
:1091B00030021092310210923202109233028091EA
:1091C000280290912902A0912A02B0912B02B7FFA8
:1091D00063C0EA8DFB8DEF5AFF4FC080D180E280E3
:1091E000F38088E996E121E0FC0145915591659174
:1091F00074914C155D056E057F0568F4F694E7944F
:10920000D794C794220F0496F4EB8F2EF6E19F2E8D
:109210008816990649F72093C70420E2C216D104A4
:10922000E104F10428F470E2C72ED12CE12CF12CDA
:1092300030E2C31AD108E108F108C11448E0D406AD
:10924000E104F10408F432C054E0D59EC0011124B9
:1092500088569D4EFC013296259134917C2D6627CF
:10926000739FA001729F410D561F0694461F561F03
:10927000112470E060E0FC0185919491B0E0A0E0E1
:10928000841B950BA60BB70B8093280290932902A1
:10929000A0932A02B0932B02C0902802D0902902FA
:1092A000E0902A02F0902B020C946F43D701C60184
:1092B000B695A795979587958C7F8856914FFC0119
:1092C00025913491FC013296459154918C2D8770F3
:1092D000C82EC49EC001C59E900D112463E09695D2
:1092E00087956A95E1F7281B390BC901B0E0A0E02A
:1092F000CBCFEE81FF81E959FF4F80819181A2811F
:10930000B3818093D6089093D708A093D808B093E0
:10931000D908AE81BF8155964D915D916D917C913B
:10932000589759968D909D90AD90BC905C9781E038
:10933000481559056A057B0509F070C2FD01EB5B14
:10934000FF4F908180E0411551056105710549F09D
:10935000292F21709695917081E0291380E02913BF
:109360005DC2EE81FF81C58CD68CE78CF0A0C11464
:10937000D104E104F10409F084608093D0041092D8
:10938000BC041092BD041092BE041092BF0410924F
:10939000C8041092C9041092CA041092CB04EE8142
:1093A000FF8185A196A1A7A1B0A58093D104909338
:1093B000D204A093D304B093D4044424552432019E
:1093C000481A590A6A0A7B0A4092AC045092AD04CA
:1093D0006092AE047092AF044092B0045092B10417
:1093E0006092B2047092B3044092B4045092B504F7
:1093F0006092B6047092B7044092B8045092B904D7
:109400006092BA047092BB0441A052A063A074A001
:10941000440C551C661C771C440F551F661F771F94
:1094200040939C0450939D0460939E0470939F040A
:10943000880C991CAA1CBB1C8092A0049092A104C9
:10944000A092A204B092A304CC0CDD1CEE1CFF1C65
:10945000C092A404D092A504E092A604F092A704BE
:109460004092A8045092A9046092AA047092AB049E
:10947000880F991FAA1FBB1F80939804909399048B
:10948000A0939A04B0939B041092D5041092D60432
:109490001092D7041092D80481A592A5A3A5B4A5D3
:1094A0008093CC049093CD04A093CE04B093CF04CA
:1094B00085A596A5A7A5B0A98093C1049093C204E1
:1094C000A093C304B093C404EA5BFF4F80818093F0
:1094D000C604882309F4A4C1EE81FF81E55BFF4F38
:1094E000808191819093970480939604EE81FF810F
:1094F000E75BFF4F80819181909395048093940462
:109500001092300210923102109232021092330205
:10951000EE81FF81E95BFF4F80819181B0E0A0E0A7
:1095200080932C0290932D02A0932E02B0932F02D1
:10953000EE81FF81EB5BFF4F808190913E078917A1
:1095400021F080933E070E9400360E94CF3DAA245E
:10955000AA94BA2C6501A0922802B0922902C09266
:109560002A02D0922B02EE81FF81FD96E080F180ED
:1095700002811381AE81BF81D1962D913D914D9194
:109580005C91D497AB5ABF4FBF83AE836D917D91F1
:109590008D919C910E9406221092C004EE81FF8161
:1095A000408151816281738188E996E121E0FC016B
:1095B000C590D590E590F490C416D506E606F7065A
:1095C00068F47695679557954795220F0496E4EBD6
:1095D0008E2EE6E19E2E8816990649F72093C70441
:1095E000403251056105710520F440E250E060E031
:1095F00070E04052510961097109411528E0520794
:109600006105710508F419C134E0539FC0011124AC
:1096100088569D4EFC01329625913491AA27439F8E
:10962000F001429FE10DFA1F0694EA1FFA1F112470
:10963000AF0170E060E0FC01C590D490F12CE12C0A
:10964000C41AD50AE60AF70AC092D904D092DA04FD
:10965000E092DB04F092DC048A809B80AC80BD80C9
:1096600089288A288B28D1F48091D9049091DA0432
:10967000A091DB04B091DC048A3F9105A105B105FE
:1096800068F4FAEFAF2EB12CC12CD12CA092D904E2
:10969000B092DA04C092DB04D092DC0440916F02F5
:1096A0005091700260917102709172020091D90420
:1096B0001091DA042091DB043091DC044F3F8FEFEE
:1096C00058076807780799F0D901C801B695A7959A
:1096D00097958795481759076A077B0740F4809349
:1096E0006F0290937002A0937102B0937202C090C7
:1096F0006F02D0907002E0907102F090720240917F
:109700003002509131026091320270913302460171
:1097100057019FEFC916D906E104F10428F0882407
:109720008A94982CA12CB12C4E835A83F62FE72FC4
:10973000041715072607370720F40E831A83F22F24
:10974000E32F8E819A81AF2FBE2F88169906AA0625
:10975000BB0610F4D501C401081B190B2A0B3B0BE7
:109760000093D9041093DA042093DB043093DC04D3
:109770004F3FEFEF5E076E077E0761F0481B590B06
:109780006A0B7B0B4093300250933102609332029C
:1097900070933302FFEFCF16DF06EF06FF0661F08E
:1097A000C81AD90AEA0AFB0AC0926F02D092700264
:1097B000E0927102F0927202F8942091840030914C
:1097C0008500205F3F4F498141504983442309F47C
:1097D00054C0280E391E2216330610F40C9416407D
:1097E000309289002092880078946B960FB6F89496
:1097F000DEBF0FBECDBFDF91CF911F910F91FF90C4
:10980000EF90DF90CF90BF90AF909F908F907F9020
:109810006F905F904F903F902F9008958260A1CD00
:1098200088248A94982C540180922C0290922D02C4
:10983000A0922E02B0922F027BCEDB01CA01B69518
:10984000A795979587958C7F8856914FFC01C59079
:10985000D490FC013296259134914770429FC0010B
:10986000439F900D112403E0969587950A95E1F7A3
:10987000C81AD90AF12CE12CE7CE1901B1CF80ED3D
:10988000C82E87E0D82EE12CF12C0C947743CF9290
:10989000DF92EF92FF92FC01C080D180E280F380E2
:1098A00020911610309117104091181050911910F6
:1098B000C701B6010F94A55B0F949E646093A81531
:1098C0007093A9158093AA159093AB15C092981523
:1098D000D0929915E0929A15F0929B1590918A1565
:1098E00080918B15981731F0FF90EF90DF90CF901B
:1098F0000C949D270E944D3A0E94753D4091A815F9
:109900005091A9156091AA157091AB154093F80478
:109910005093F9046093FA047093FB04882331F0A8
:10992000FF90EF90DF90CF900C942A8FFF90EF90F4
:10993000DF90CF9008954F925F926F927F928F92B7
:109940009F92AF92BF92CF92DF92EF92FF920F93CE
:109950001F93CF93DF93EC018B017A016901F90129
:1099600080819181A281B381FA014081518162811C
:109970007381F80180809180A280B38048805980F3
:109980006A807B8040928C1550928D1560928E1566
:1099900070928F158092901590929115A0929215C9
:1099A000B092931540939415509395156093961526
:1099B000709397158093981590939915A0939A1585
:1099C000B0939B15209116103091171040911810EC
:1099D00050911910F60160817181828193810F94F9
:1099E000A55B0F949E644B015C0120911210309195
:1099F00013104091141050911510F701608171817E
:109A0000828193810F94A55B0F949E646B017C010E
:109A100020910E1030910F104091101050911110A4
:109A2000F80160817181828193810F94A55B0F940D
:109A30009E642B013C0120910A1030910B10409143
:109A40000C1050910D10688179818A819B810F944F
:109A5000A55B0F949E6460939C1570939D158093F5
:109A60009E1590939F154092A0155092A11560925B
:109A7000A2157092A315C092A415D092A515E092DC
:109A8000A615F092A7158092A8159092A915A092FC
:109A9000AA15B092AB1590918A1580918B159817E5
:109AA00091F0DF91CF911F910F91FF90EF90DF9098
:109AB000CF90BF90AF909F908F907F906F905F906E
:109AC0004F900C949D270E944D3A0E94753DC09086
:109AD000A415D090A515E090A615F090A71540917B
:109AE0009C1550919D1560919E1570919F15009148
:109AF000A0151091A1152091A2153091A3154A012E
:109B00005B01800E911EA21EB31E8092EC04909207
:109B1000ED04A092EE04B092EF04401B510B620BD7
:109B2000730B4093F0045093F1046093F20470932C
:109B3000F304C092F404D092F504E092F604F0929B
:109B4000F7044091A8155091A9156091AA1570913C
:109B5000AB154093F8045093F9046093FA047093A2
:109B6000FB04882391F0DF91CF911F910F91FF901B
:109B7000EF90DF90CF90BF90AF909F908F907F90AD
:109B80006F905F904F900C942A8FDF91CF911F912F
:109B90000F91FF90EF90DF90CF90BF90AF909F908C
:109BA0008F907F906F905F904F9008958F929F92CB
:109BB000AF92BF92CF92DF92EF92FF920F931F93DB
:109BC000CF93DF93182F84E0189FE0011124123007
:109BD00008F04CC00E94753D082F0E94753D809092
:109BE000EC049090ED04A090EE04B090EF0481118D
:109BF0000E942A8F0E94753DC090F004D090F1041D
:109C0000E090F204F090F30481110E942A8F011178
:109C10000E942A8F113019F5C501B4016C197D0914
:109C20008E099F090F94465B20E030E040E05FE33F
:109C30000F94A55BCF5CD64F288139814A815B8127
:109C40000F94A55BDF91CF911F910F91FF90EF9043
:109C5000DF90CF90BF90AF909F908F900895C701F5
:109C6000B601680D791D8A1D9B1DDCCF0E94753DD4
:109C7000FE01E451FB4FC080D180E280F38081116E
:109C80000E942A8FC701B6010F94465BD3CFCF92B3
:109C9000DF92EF92FF92CF93DF93C82F0E94753D22
:109CA00094E0C99FE0011124FE01E052FB4FC08007
:109CB000D180E280F38081110E942A8FCF5CD64F41
:109CC000C701B6010F94465B288139814A815B81C7
:109CD0000F94A55BDF91CF91FF90EF90DF90CF9035
:109CE0000895CF930E94753DC82F80918B15809366
:109CF0008A15809389158093881584E6809387154B
:109D00000E948E3F80ED93E0909343098093420937
:109D1000C1110E942A8F81E08093DF04CF910895C2
:109D2000CF93DF9324E0829FC0011124EC01CF5137
:109D3000D74FFC01ED5DF74F895E974FDC012D9108
:109D40003D914D915C9160817181828193810F94ED
:109D50003162688379838A839B83DF91CF910895F1
:109D600080FF04C090919C0390FD8E7F81FF05C011
:109D700090919C03969590FD8D7F82FF06C09091F7
:109D80009C039695969590FD8B7F08958F929F9258
:109D9000AF92BF92CF92DF92EF92FF92CF93DF9379
:109DA00020910E02222309F49EC0EC0180919C03B5
:109DB000C82ED12CF12CE12C80FF2CC080901002F9
:109DC00090901102A0901202B09013022881398164
:109DD0004A815B81C501B4010F949164181624F483
:109DE00088829982AA82BB8280901C0290901D0278
:109DF000A0901E02B0901F02288139814A815B81A8
:109E0000C501B4010F943F5B87FF04C0888299822B
:109E1000AA82BB82D701C601B695A795979587956B
:109E200080FF2CC08090140290901502A090160222
:109E3000B09017022C813D814E815F81C501B40134
:109E40000F949164181624F48C829D82AE82BF8296
:109E50008090200290902102A0902202B0902302D4
:109E60002C813D814E815F81C501B4010F943F5B20
:109E700087FF04C08C829D82AE82BF8282E0F6940E
:109E8000E794D794C7948A95D1F7C0FE2CC0C090B0
:109E90001802D0901902E0901A02F0901B02288557
:109EA00039854A855B85C701B6010F949164181600
:109EB00024F4C886D986EA86FB86C0902402D09016
:109EC0002502E0902602F0902702288539854A85F0
:109ED0005B85C701B6010F943F5B87FF04C0C8864E
:109EE000D986EA86FB86DF91CF91FF90EF90DF90D5
:109EF000CF90BF90AF909F908F9008958091650410
:109F000090916604A0916704B091680480937302F5
:109F100090937402A0937502B093760280916304CB
:109F20009091640490936A028093690208958091ED
:109F3000730290917402A0917502B09176028093A1
:109F4000650490936604A0936704B09368048091BD
:109F5000690290916A02909364048093630484E69A
:109F600090E090936A02809369020895CF92DF9205
:109F7000EF92FF920F931F93C12CD12C76018C018D
:109F800029EF38E045EF58E061EF78E08DEE98E09A
:109F90000F94D52C1F910F91FF90EF90DF90CF90F1
:109FA00008954F925F926F927F928F929F92AF929D
:109FB000BF92CF92DF92EF92FF920F931F93CF93B6
:109FC000DF93CDB7DEB72C970FB6F894DEBF0FBE88
:109FD000CDBF2B013C0129873A874B875C8747011E
:109FE0005801F601E080F1800281138120E030E029
:109FF000A901B701C8010F943F5B882309F488C009
:10A000005E2D4F2D302F212F852F942FA32FB22F70
:10A0100089839A83AB83BC8320E030E0A901B70138
:10A02000C8010F943F5B811108C0E0906B02F09073
:10A030006C0200916D0210916E02C701D8018D83F0
:10A040009E83AF83B887A50194016091F508709154
:10A05000F6088091F7089091F8080F943F5B87FF0E
:10A060000CC08092F5089092F608A092F708B09282
:10A07000F808CE0101960E94B64F4092ED0850922A
:10A08000EE086092EF087092F00889859A85AB859A
:10A09000BC858093F1089093F208A093F308B093E5
:10A0A000F408CE0105960E94B64FA5019401609177
:10A0B000F5087091F6088091F7089091F8080F94D0
:10A0C0009164181664F48092F5089092F608A092B4
:10A0D000F708B092F808CE0101960E94B64F0E9490
:10A0E0004D3A2C960FB6F894DEBF0FBECDBFDF9170
:10A0F000CF911F910F91FF90EF90DF90CF90BF9085
:10A10000AF909F908F907F906F905F904F90089549
:10A1100050E040E030E820E477CFCF92DF92EF923A
:10A12000FF920F931F936A01E090F508F090F608F4
:10A130000091F7081091F808FB01208131814281DC
:10A140005381FC0160817181828193810E94D14F92
:10A150001F910F91FF90EF90DF90CF900895CF92D5
:10A16000DF92EF92FF920F931F936B01FC01E0804F
:10A17000F18002811381EDEEF8E024813581468182
:10A18000578160817181828193810E94D14F1F919B
:10A190000F91FF90EF90DF90CF900895AF92BF9214
:10A1A000CF92DF92EF92FF920F931F93CF93DF93A3
:10A1B00000D01F92CDB7DEB7FC01E080F1800281B4
:10A1C0001381611112C0A090F508B090F608C090FC
:10A1D000F708D090F8089501A601B701C8010F94BF
:10A1E0003F5B87FF02C07501860120E030E046E951
:10A1F00053E4B701C8010F943F5B87FD04C0E12C15
:10A20000F12C06E913E4C701D80189839A83AB8353
:10A21000BC836BEC72E0CE0101960E94AF500F90B0
:10A220000F900F900F90DF91CF911F910F91FF90A2
:10A23000EF90DF90CF90BF90AF9008950F931F9352
:10A24000CF93DF938B01CDEED8E02091780230914F
:10A25000790240917A0250917B02FC016081718108
:10A26000828193810F942B632C853D854E855F857C
:10A270000F9431626C877D878E879F87C8010E940B
:10A28000B64FDF91CF911F910F910C944D3A8F9261
:10A290009F92AF92BF92CF92DF92EF92FF921F9365
:10A2A000CF93DF93CDB7DEB760970FB6F894DEBFDC
:10A2B0000FBECDBF182F80E00E94D64D4B015C0130
:10A2C0008092570490925804A0925904B0925A0474
:10A2D00081E00E94D64D6B017C01C0925B04D0925C
:10A2E0005C04E0925D04F0925E0482E00E94D64D30
:10A2F00060935F04709360048093610490936204A0
:10A300001D861E861F86188A89829A82AB82BC822D
:10A31000CD82DE82EF82F88669877A878B879C8779
:10A3200083E00E94D64D6D877E878F87988B8091C2
:10A33000FC07882321F0CE0101960E949D391E3F23
:10A34000D9F480E1FE013196ADEEB8E001900D92B6
:10A350008A95E1F760960FB6F894DEBF0FBECDBFC9
:10A36000DF91CF911F91FF90EF90DF90CF90BF9042
:10A37000AF909F908F90089584E0189FF001112472
:10A38000DF01A351B74F81E090E08C0F9D1FE80FD4
:10A39000F91F40815181628173814D935D936D936B
:10A3A0007C931397D7CF0D94372D2F923F924F92D6
:10A3B0005F926F927F928F929F92AF92BF92CF9255
:10A3C000DF92EF92FF920F931F93CF93DF93CDB75E
:10A3D000DEB763970FB6F894DEBF0FBECDBF809196
:10A3E000300481112CC280912F0481111CC28091F4
:10A3F0003B04811119C063960FB6F894DEBF0FBEFF
:10A40000CDBFDF91CF911F910F91FF90EF90DF9023
:10A41000CF90BF90AF909F908F907F906F905F9004
:10A420004F903F902F9008950E9472330F943D37C4
:10A430004B015C0100910A1510910B15809165028A
:10A4400090916602801791070CF444C38091350403
:10A45000882309F424C360910C1570910D15072E03
:10A46000000C880B990B0F94465B6D837E838F8362
:10A470009887B801110F880B990B0F94465B69837D
:10A480007A838B839C834AE0E42EF12C0CE310E06A
:10A4900020E0AE014B5F5F4FBE016F5F7F4F8BE1EE
:10A4A00095E10E94333400910A1510910B158091AB
:10A4B000630290916402801791070CF022C1809191
:10A4C000650290916602081719070CF01AC1609195
:10A4D0000C1570910D156115710509F472C3601B9F
:10A4E000710B072E000C880B990B0F94465B2B0108
:10A4F0003C0120E030E040E251EC0F943F5B87FDEF
:10A5000060C38091350481115CC320E030E040E2FB
:10A5100051E4C301B2010F94916418160CF467C39F
:10A520008091250581116EC3C0901D05D0901E0538
:10A53000E0901F05F0902005809121059091220563
:10A54000A0912305B09124058D879E87AF87B88B96
:10A55000B801110F880B990B0F94465B9B01AC015E
:10A560006091110570911205809113059091140569
:10A570000F943062209117153091181540911915DC
:10A5800050911A150F94A55BA70196010F943062A4
:10A5900020ED3CEC4CE45DE30F94A55BA701960134
:10A5A0000F9431626B017C01C0921D05D0921E0593
:10A5B000E0921F05F092200520911315309114159B
:10A5C000409115155091161529873A874B875C875E
:10A5D0002D853E854F855889C301B2010F943162A4
:10A5E000162F072F382E292E20E030E0A9010F94D6
:10A5F0003F5B87FD11C329853A854B855C8560E00B
:10A6000070E08FE793E40F942B636D87798B8A8BCF
:10A610009B8B212F302F432D522D0F943F5B87FFB3
:10A6200004C01D8509893A882B88812F902FA32D7E
:10A63000B22D8093210590932205A0932305B0931A
:10A64000240520910F15309110154091111550914E
:10A650001215C301B2010F94A55B2B013C0140927E
:10A660001505509216056092170570921805212F56
:10A67000302F432D522D69857A858B859C850F94CB
:10A68000A55B9B01AC012093190530931A054093FB
:10A690001B0550931C05C301B2010F943162A70141
:10A6A00096010F94316220E030E0A9010F943162ED
:10A6B00069837A838B839C834FEF50E070E060E086
:10A6C000CE0101960E948A3300910A1510910B1554
:10A6D00069817A818B819C810F949D6375956795C3
:10A6E000F62EB801012E000C880B990B0F94465BD7
:10A6F00060931105709312058093130590931405D0
:10A7000001C0F12CF0920E15809102159091031565
:10A71000A0910415B09105150097A105B105C9F0E8
:10A72000A5019401281B390B4A0B5B0BDA01C90107
:10A73000B7FD0FC0809100159091011508171907FA
:10A740000CF00EC24FEE56E16EEF76E180E00E9413
:10A75000CC330091010810910208073911050CF063
:10A7600092C18091280590912905A0912A05B09168
:10A770002B050097A105B10511F1A5019401281B36
:10A78000390B4A0B5B0BDA01C901B7FD18C0809188
:10A79000260590912705081719070CF0BEC14FEE4A
:10A7A00056E16EEF76E18FEF0E94CC3360910308A3
:10A7B00070910408009101081091020804C0609192
:10A7C00003087091040880913A04882309F48EC12B
:10A7D000072E000C880B990B0F94465B6D837E83CC
:10A7E0008F839887B801110F880B990B0F94465BE4
:10A7F00069837A838B839C8392E0E92EF12C02E3B8
:10A8000010E02FEFAE014B5F5F4FBE016F5F7F4FD8
:10A8100084E295E10E94333480913A048823B9F0B0
:10A8200010920508E8CD10922F040E94714E0E94EC
:10A830004D3A8EEF0E9447510E94D351D8CD41E04E
:10A8400070E060E08DE097E10E9462A5CCCD0091C0
:10A85000010810910208C80105978239910520F07E
:10A8600060E060930508C7CD60910308709104080B
:10A870006115710509F4AAC1601B710B072E000C4C
:10A88000880B990B0F94465B6B017C0120E030E054
:10A8900040E251EC0F943F5B87FD98C120E030E02F
:10A8A00040E251E4C701B6010F94916418160CF40C
:10A8B00091C180910A0890910B08A0910C08B09169
:10A8C0000D0889879A87AB87BC87809134028111F4
:10A8D00086C120910D0530910E0540910F055091D4
:10A8E00010054090090550900A0560900B05709086
:10A8F0000C05C701B6010F943162B62EA72E982E13
:10A90000892E20E030E0A9010F943F5B87FD75C1DF
:10A9100029853A854B855C8560E070E08FE793E49C
:10A920000F942B63362E272E8D87998B2B2D3A2D46
:10A93000492D582D0F943F5B87FF03C051019D8423
:10A9400089888B2D9A2DA92DB82D80930D05909374
:10A950000E05A0930F05B0931005209106083091C5
:10A9600007084091080850910908C701B6010F94E3
:10A97000A55B6B017C01C0920105D0920205E092BB
:10A980000305F09204052B2D3A2D492D582D69858C
:10A990007A858B859C850F94A55B69877A878B87E1
:10A9A0009C87609305057093060580930705909337
:10A9B0000805B801110F880B990B0F94465B4B01EA
:10A9C0005C01AC019B016091FD047091FE048091DB
:10A9D000FF04909100050F94306220910E08309191
:10A9E0000F0840911008509111080F94A55BA30126
:10A9F00092010F94306220ED3CEC4CE45DE30F9447
:10AA0000A55BA30192010F9431622B013C0140929E
:10AA1000090550920A0560920B0570920C05809210
:10AA2000FD049092FE04A092FF04B09200052985D7
:10AA30003A854B855C85C701B6010F943162A3014D
:10AA400092010F94316220E030E0A9010F9431624D
:10AA50006B017C0120E030E0A9010F943F5B87FD92
:10AA6000FFCE20E030E04FE753E4C701B6010F947A
:10AA7000916418160CF4B1C0C701B6010F949D6320
:10AA800075956795EECE4BEB57E168EC77E18FEF6C
:10AA90000E94CC33009101081091020862CE80918F
:10AAA000310490913204A0913304B09134040097A2
:10AAB000A105B10509F4CFCCA5019401281B390BE0
:10AAC0004A0B5B0BDA01C901B7FDC5CC81E080936D
:10AAD0003504C1CC4BEB57E168EC77E180E00E9494
:10AAE000CC3300910A1510910B15B0CC809136042F
:10AAF00090913704A0913804B09139040097A105D2
:10AB0000B10509F465CE881A990AAA0ABB0AB7FCEE
:10AB10005FCE81E080933A045BCE60910308709130
:10AB200004086115710509F443C0C80102969B0130
:10AB30002450310982179307DCF590932705809301
:10AB400026050F943D37605E70448D4F9F4F609394
:10AB500028057093290580932A0590932B0526CE0E
:10AB600080910C1590910D150097C9F00E5F1F4F45
:10AB70000497081719079CF410930115009300150A
:10AB80000F943D37605B7C438F4F9F4F609302155E
:10AB9000709303158093041590930515DACD1092E8
:10ABA0000215109203151092041510920515D1CDBF
:10ABB000109228051092290510922A0510922B0553
:10ABC00002CE81E080932505F12C8BCD81E080932E
:10ABD000340246CE81E0809334026FE742CE109279
:10ABE0003402412C512C3201A301920182CE81E02A
:10ABF000809325053FE7F32E74CDB12CA12C912C29
:10AC0000812C9FCE109225051D861E861F86188AD0
:10AC1000C12CD12C76019CCC10E000E0312C212CF1
:10AC200004CD2F923F924F925F926F927F928F92BC
:10AC30009F92AF92BF92CF92DF92EF92FF920F93CB
:10AC40001F93CF93DF93CDB7DEB7A6970FB6F894D7
:10AC5000DEBF0FBECDBF81EC97E00E94C64E809153
:10AC6000F50F83FD7EC02091F9083091FA084091DC
:10AC7000FB085091FC086091CD077091CE07809140
:10AC8000CF079091D0070F943F5B882309F469C0E8
:10AC900010914109111161C080917C0290917D0257
:10ACA000019720910A1530910B15281739073CF4AC
:10ACB0000E94CAA186E398E00E94399211E0209197
:10ACC000F9083091FA084091FB085091FC08609116
:10ACD000CD077091CE078091CF079091D0070F9448
:10ACE00030626B017C0120E030E0A9010F94916497
:10ACF00087FF04C0F7FAF094F7F8F09420917802F7
:10AD00003091790240917A0250917B02C701B601DD
:10AD10000F94A55B20E030E84BE354E40F9491647A
:10AD20001816ECF40E94CAA187E198E00E943992BB
:10AD30008091CD079091CE07A091CF07B091D00719
:10AD40008093F9089093FA08A093FB08B093FC084D
:10AD50008DEC97E00E94474C04C010E0B0CF111179
:10AD6000E7CF2AE037ED43E25CE360917302709134
:10AD7000740280917502909176020F94A55B6B012D
:10AD80007C016091690270916A02072E000C880BA9
:10AD9000990B0F94465B9B01AC01C701B6010F9460
:10ADA000A55B698B7A8B8B8B9C8B8091FC078823AE
:10ADB00009F18090F8079090F907A090FA07B090F9
:10ADC000FB07C090C907D090CA07E090CB07F0906E
:10ADD000CC0720E030E0A901C501B4010F943F5B2E
:10ADE0008823D1F1A7019601C501B4010F949164A4
:10ADF000181694F1C12CD12C76018E010F5E1F4FD5
:10AE00002DEC37E049EC57E065EC77E081EC97E01A
:10AE10000F94D52C80E1E1ECF7E0ADEEB8E00190C5
:10AE20000D928A95E1F7A6960FB6F894DEBF0FBE95
:10AE3000CDBFDF91CF911F910F91FF90EF90DF90E9
:10AE4000CF90BF90AF909F908F907F906F905F90CA
:10AE50004F903F902F9008952091ED083091EE088B
:10AE60004091EF085091F0086091C1077091C207BE
:10AE70008091C3079091C4070F9430626D8B7E8BD5
:10AE80008F8B988F2091F1083091F2084091F30850
:10AE90005091F4086091C5077091C6078091C7076B
:10AEA0009091C8070F943062698F7A8F8B8F9C8F37
:10AEB0002091F5083091F6084091F7085091F80874
:10AEC000C701B6010F9430626D8F7E8F8F8F98A36C
:10AED0002091F9083091FA084091FB085091FC0844
:10AEE0006091CD077091CE078091CF079091D007E8
:10AEF0000F9430626B017C0120E030E0A9016D8984
:10AF00007E898F89988D0F943F5B81110CC020E062
:10AF100030E0A901698D7A8D8B8D9C8D0F943F5BFC
:10AF2000882309F467CF2D893E894F89588DCA013E
:10AF3000B9010F94A55B4B015C01298D3A8D4B8DB6
:10AF40005C8DCA01B9010F94A55B9B01AC01C501E1
:10AF5000B4010F9431624B015C012D8D3E8D4F8DFC
:10AF600058A1CA01B9010F94A55B9B01AC01C501B1
:10AF7000B4010F9431624B015C01A7019601C70136
:10AF8000B6010F94A55B9B01AC01C501B4010F9400
:10AF900031620F94DF644B015C012DEB37E346E82F
:10AFA00055E30F943F5B87FF0FC020E030E0A9011D
:10AFB000C701B6010F9491644601570187FF04C091
:10AFC000B7FAB094B7F8B0942DEB37E346E855E301
:10AFD000C501B4010F943F5B87FD1CCF20E030E03A
:10AFE00040EA51E4C501B4010F942B630F94A463AC
:10AFF0001B01672B19F422242394312CB10190E01A
:10B0000080E00F94445B9B01AC0160E070E080E85D
:10B010009FE30F942B632B013C01AC019B01C50105
:10B02000B4010F94A55B4B015C01A30192016D89F2
:10B030007E898F89988D0F94A55B6D8B7E8B8F8B0E
:10B04000988FA3019201698D7A8D8B8D9C8D0F94C1
:10B05000A55B698F7A8F8B8F9C8FA30192016D8D79
:10B060007E8D8F8D98A10F94A55B6D8F7E8F8F8FB6
:10B0700098A3A3019201C701B6010F94A55B69A330
:10B080007AA38BA39CA380E1EDEEF8E08E010F5F25
:10B090001F4FD80101900D928A95E1F70F943D372B
:10B0A0002B013C0128EC420E511C611C711C0DA3AC
:10B0B0001EA381E0281A310809F460C00F943D37BF
:10B0C0008B019C01041915092609370937FD59C060
:10B0D0002B013C0128EC420E511C611C711C80E0CC
:10B0E0000E9487A72D893E894F89588D69817A8171
:10B0F0008B819C810F94316269837A838B839C83DB
:10B10000298D3A8D4B8D5C8D6D817E818F819885E7
:10B110000F9431626D837E838F8398872D8D3E8D52
:10B120004F8D58A169857A858B859C850F943162F6
:10B1300069877A878B879C8729A13AA14BA15CA15B
:10B140006D857E858F8598890F9431626D877E87A6
:10B150008F87988B750164018E010F5E1F4F9E01D2
:10B16000235F3F4FAE01475F5F4FBE016B5F7F4F75
:10B170008DA19EA10F94D52C81119BCF75016401E7
:10B180003CCE0E94D551AECF8F929F92AF92BF928C
:10B19000CF92DF92EF92FF92CF93DF938090730272
:10B1A00090907402A0907502B0907602FC01C0806D
:10B1B000D180E280F38020E030E0A901C701B60130
:10B1C0000F943F5B882341F0C0927302D0927402C7
:10B1D000E0927502F0927602C0916902D0916A0203
:10B1E00084E690E090936A0280936902C0907802AE
:10B1F000D0907902E0907A02F0907B0280E090E0BB
:10B20000A0E8BFE38093780290937902A0937A023A
:10B21000B0937B020E941156809273029092740246
:10B22000A0927502B0927602D0936A02C09369022E
:10B23000C0927802D0927902E0927A02F0927B0278
:10B24000DF91CF91FF90EF90DF90CF90BF90AF90C4
:10B250009F908F9008950F931F93CF93DF93EC01EE
:10B260008B0181E00F94402E69E170E080E090E076
:10B270000E94478FB801CE010E94AF50C091820753
:10B2800080E00F94402E1092820782E00E94475186
:10B290000E94D351C2FBCC27C0F981E08C27DF91FB
:10B2A000CF911F910F910895CF93DF93CDB7DEB764
:10B2B0002C970FB6F894DEBF0FBECDBF0F947D2D37
:10B2C0000E94753D9CE0ECEEF4E0DE0111960190E9
:10B2D0000D929A95E1F781110E942A8FCE01019675
:10B2E0000E948C352C960FB6F894DEBF0FBECDBFF2
:10B2F000DF91CF9108952F923F924F925F926F927C
:10B300007F928F929F92AF92BF92CF92DF92EF92F5
:10B31000FF920F931F93CF93DF9300D0CDB7DEB78B
:10B320008090ED089090EE08A090EF08B090F008A3
:10B330004090F1085090F2086090F3087090F40883
:10B34000C090F508D090F608E090F708F090F80863
:10B350000E94DB390E94562307E71BE080E192E060
:10B360009B838A838BE6282E8BE0382E1982898175
:10B370000E94904EC8010E944981EA81FB8161933D
:10B38000719381939193FB83EA83C1010E94498168
:10B39000EA81FB816087718782879387F981FF5FEC
:10B3A000F9830C5F1F4F84E0280E311CF330F9F64F
:10B3B00060E087E894E00E94ED8D0E94CD8E0E94AF
:10B3C000293AA50194016091ED087091EE088091F1
:10B3D000EF089091F0080F943F5B81111CC0A3010E
:10B3E00092016091F1087091F2088091F3089091B8
:10B3F000F4080F943F5B81110EC02091F508309145
:10B40000F6084091F7085091F808C701B6010F946B
:10B410003F5B8823B9F00F900F900F90DF91CF9191
:10B420001F910F91FF90EF90DF90CF90BF90AF9062
:10B430009F908F907F906F905F904F903F902F9054
:10B440000C9454590F900F900F90DF91CF911F9152
:10B450000F91FF90EF90DF90CF90BF90AF909F90B3
:10B460008F907F906F905F904F903F902F900895B6
:10B47000CF93DF9300D01F92CDB7DEB784EF91E07A
:10B48000A0E0B0E089839A83AB83BC83BE016F5F89
:10B490007F4F8CE30E9429918DEF97E00E943992B3
:10B4A0008CB185FB882780F967EF77E091E08927E9
:10B4B0000E9468278091030161EF77E08695817093
:10B4C0000E94682789B16BEE77E083FB882780F9BB
:10B4D0000E9468274B9909C00E9464910F900F90B9
:10B4E0000F900F90DF91CF9108950E9449910F9096
:10B4F0000F900F900F90DF91CF91089580913D07AD
:10B50000811104C08091D207882331F062E070E09D
:10B5100080E090E00C94478F0895CF93DF93CDB7F0
:10B52000DEB72C970FB6F894DEBF0FBECDBFA6EFE7
:10B53000BFE090E080E0FC01E857F14F4591559164
:10B54000659174914D935D936D937D93FC01E858E3
:10B55000F14F459155916591749150964D935D933E
:10B560006D937C935397FC01E859F14F45915591A8
:10B570006591749190964D935D936D937C939397A1
:10B58000049680319105B9F680E29EE4A0E0B0E037
:10B590008093061090930710A0930810B0930910A1
:10B5A00080E090E8ABE3B4E480932A1090932B10F2
:10B5B000A0932C10B0932D1080E090E0AAE7B4E4A3
:10B5C00080932E1090932F10A0933010B0933110D1
:10B5D00080E090E0A6E9B3E48093321090933310BA
:10B5E000A0933410B093351010923610109237108B
:10B5F000109238101092391010923A1010923B109D
:10B6000010923C1010923D1080E090E0A0E2B1E476
:10B610008093170990931809A0931909B0931A09F8
:10B6200080E090E0A0EAB0E480931B0990931C09AD
:10B63000A0931D09B0931E094AE959E969E97EE31F
:10B6400040931F09509320096093210970932209A8
:10B650008093230990932409A0932509B093260988
:10B6600010922B0810922C0810922D0810922E0880
:10B6700010922708109228081092290810922A0880
:10B680001092230810922408109225081092260880
:10B6900010928704109288041092890410928A04F0
:10B6A0000E94A98D8CE0E3EBF2E0DE01119601909F
:10B6B0000D928A95E1F789819A81AB81BC81809353
:10B6C000791590937A15A0937B15B0937C158D8195
:10B6D0009E81AF81B88580937D1590937E15A09350
:10B6E0007F15B093801589859A85AB85BC8580933D
:10B6F000811590938215A0938315B093841584EBE4
:10B7000090E0909385078093840786E490E090937F
:10B71000870780938607109289071092880780EF29
:10B7200090E090938B0780938A078EE690E0909349
:10B730008D0780938C0710928F0710928E0786E6F4
:10B7400096E6A6E8B1E480930F1590931015A093A8
:10B750001115B09312158CE993E5A9E4BEE380932B
:10B76000131590931415A0931515B093161580EE2C
:10B7700095EBA5EAB3E48093171590931815A09361
:10B780001915B0931A1583EC95E9ACE2B4E48093F3
:10B79000060890930708A0930808B093090880E270
:10B7A0009BE1A2E9B1E480930A0890930B08A0936F
:10B7B0000C08B0930D0887EF9CEDABECB5E48093DB
:10B7C0000E0890930F08A0931008B09311081092E0
:10B7D000B1030E9400891092160880E090E0A0EE6C
:10B7E000BFE38093120890931308A0931408B093BA
:10B7F000150810923D0710923C070E947E5A109245
:10B800002709109228091092290910922A0980E02C
:10B8100090E0A7EDB3E48093A9039093AA03A093CB
:10B82000AB03B093AC038093AD039093AE03A093AE
:10B83000AF03B093B0032C960FB6F894DEBF0FBEE3
:10B84000CDBFDF91CF910C947B593F924F925F9285
:10B850006F927F928F929F92AF92BF92CF92DF9220
:10B86000EF92FF920F931F93CF93DF9300D01F921D
:10B87000CDB7DEB7382E80E090E0A0E2B1E4898356
:10B880009A83AB83BC83C0908115D0908215E090E1
:10B890008315F090841520E030E0A901C701B601BE
:10B8A0000F943F5B87FF0CC0A701960160E070E03A
:10B8B00080E291E40F94306269837A838B839C8366
:10B8C00060E0CE0101960E94CE504090ED0850906D
:10B8D000EE086090EF087090F0088090F10890906A
:10B8E000F208A090F308B090F408332089F10E9488
:10B8F00019A519821A821B821C82E090F508F0902B
:10B90000F6080091F7081091F808CE0101966C0135
:10B91000A5019401C301B2010E94D14F3092D20718
:10B920000E947E5A0F900F900F900F90DF91CF9151
:10B930001F910F91FF90EF90DF90CF90BF90AF904D
:10B940009F908F907F906F905F904F903F90089561
:10B950000E94D6A4CECF80918207882319F010923E
:10B960008207089540E070E060E08BEC97E00C9473
:10B9700062A53F924F925F926F927F928F929F92B9
:10B98000AF92BF92CF92DF92EF92FF920F931F93ED
:10B99000CF93DF93CDB7DEB768970FB6F894DEBFCD
:10B9A0000FBECDBFD82E2A013B01480159013E2CC4
:10B9B00020E030E0A901C501B8010F943F5B81117F
:10B9C00010C081E08D1508F0B6C060E070E080E73F
:10B9D00093E420E030E040E752E40F942B634B0106
:10B9E0005C018D8A9E8AAF8AB88E0D2D10E0F80119
:10B9F000E455F74FE491BB24B3941E160CF4B12C1C
:10BA0000CC24C39420E030E0A901C301B2010F941B
:10BA1000916418160CF0C12CBC1471F092E0D9128C
:10BA20000BC0332049F081E00F94402E69E170E0B3
:10BA300080E090E00E94478F80E00E94D64D6983AD
:10BA40007A838B839C8381E00E94D64D6D837E83B5
:10BA50008F83988782E00E94D64D69877A878B878B
:10BA60009C8783E00E94D64D6D877E878F87988B59
:10BA7000000F111F000F111FE1E0F0E0EC0FFD1FA0
:10BA80000E0F1F1FF80110821182128213829E0175
:10BA9000235F3F4FAE01475F5F4FBE016B5F7F4F3C
:10BAA000CE0101960E949B4CF80140825182628235
:10BAB0007382198A1A8A1B8A1C8A80914209909182
:10BAC0004309892B91F4CE0141967C018E010B5ED6
:10BAD0001F4F9E01235F3F4FAE01475F5F4FBE0187
:10BAE0006B5F7F4F40970F946E1C0E944D3ABC14C1
:10BAF00051F092E0D91205C0332019F080E00F9484
:10BB0000402E0E94AB5C68960FB6F894DEBF0FBE65
:10BB1000CDBFDF91CF911F910F91FF90EF90DF90FC
:10BB2000CF90BF90AF909F908F907F906F905F90DD
:10BB30004F903F90089560E070E88BE395E449CF23
:10BB40002F923F924F925F926F927F928F929F922D
:10BB5000AF92BF92CF92DF92EF92FF920F931F931B
:10BB6000CF93DF93CDB7DEB766970FB6F894DEBFFD
:10BB70000FBECDBFF82E282E312CF101E455F74F22
:10BB8000D49022E0821335C08091D207811103C086
:10BB900081E00E94255C0E9419A5811139C188EAC3
:10BBA00098E00E94498120E030E0A9010F943F5BBA
:10BBB0008823F9F06D2DDD0C770B880B990B0F9412
:10BBC000465B2B013C0188EA98E00E9449814B01C9
:10BBD0005C0120E030E040EA50E40F943F5B11E06C
:10BBE00087FF1CC0812C912C90EAA92E90E4B92EDD
:10BBF00015C06D2DDD0C770B880B990B0F94465BF0
:10BC00002B013C01C101880F991F880F991F805695
:10BC1000974F0E9449814B015C0110E0A301920102
:10BC2000C501B4010F94A55B4B015C016101CC0C13
:10BC3000DD1CCC0CDD1CC6018C56974F0E9449813F
:10BC4000EE24E394E12620E030E040EC5FE30F9443
:10BC5000A55BA30192010F94A55BAB01BC0100E0C1
:10BC600010E098018F2D0E94B95C20E030E0A9011E
:10BC7000C501B4010F943F5BF601E857F74FFA8B0B
:10BC8000E98B882309F44DC0F2E000E010E020E4E5
:10BC900031E4FF1619F000E010E09801B501A401AD
:10BCA0007058E12C8F2D0E94B95CA5019401C5014B
:10BCB000B4010F9431626B8B7C8B8D8B9E8B22E059
:10BCC000F216E9F0F101EB57F74F6491611107C0EB
:10BCD0000E94CAA183E698E00E9439926AE070E06F
:10BCE00090E080E00F94445B9B01AC0160E070E069
:10BCF00088E492E40F942B638B019C0104C000E064
:10BD000010E020EC30E4EE24E3944B895C896D89EB
:10BD10007E898F2D0E94B95C32E0F312D0C00E9460
:10BD2000D6A481E090E0A0E0B0E00F2C04C0880F22
:10BD3000991FAA1FBB1F0A94D2F72091D107282B65
:10BD40002093D10720919C03822B80939C038989A7
:10BD50009A890E944981F601E351F74F608371830C
:10BD60008283938382E0F8121AC02091811530916A
:10BD7000821540918315509184156091F50870915A
:10BD8000F6088091F7089091F8080F94306260935C
:10BD9000F5087093F6088093F7089093F808F60179
:10BDA000E95EF74F10821182128213828F2D0E945A
:10BDB000904E0E94D351F601E351F74F808191815B
:10BDC000A281B381F601EF53F84F80839183A28360
:10BDD000B38392E0F916A9F18CE0EFEBF2E0DE011B
:10BDE000119601900D928A95E1F7E1E0F0E0EC0FF9
:10BDF000FD1FEC0DFD1D80809180A280B38020E0AE
:10BE000030E0A901C501B4010F943F5B81111EC050
:10BE100066960FB6F894DEBF0FBECDBFDF91CF910F
:10BE20001F910F91FF90EF90DF90CF90BF90AF9058
:10BE30009F908F907F906F905F904F903F902F904A
:10BE400008950E944F818111E3CFC6CF20E030E0FA
:10BE5000A901C501B4010F94916487FF04C0B7FA2A
:10BE6000B094B7F8B094F601E351F74F6F01A30116
:10BE70009201C501B4010F94A55B9B01AC01F601D1
:10BE800060817181828193810F943062F6016083B9
:10BE9000718382839383F2E080E090E0A0E4B1E4D8
:10BEA000FF1621F080E090E0A8E4B2E48D879E8741
:10BEB000AF87B88BCE010D960E94B64FA9CF81E017
:10BEC00090E0A0E0B0E00F2C04C0880F991FAA1FDB
:10BED000BB1F0A94D2F72091D107282B2093D107BA
:10BEE00020919C03822B80939C0389899A890E94CC
:10BEF0004981F601E351F74F608371838283938315
:10BF00004ECF0F931F938091F607813019F50F9450
:10BF10003D370091710410917204209173043091A7
:10BF20007404601B710B820B930B28EE33E040E02E
:10BF300050E00F9483616091A1037091A2038091FE
:10BF4000A3039091A403620F731F841F951F1F9179
:10BF50000F91089560917504709176048091770433
:10BF600090917804D6CFCF92DF92EF92FF92CF9349
:10BF7000C82F8091F6078150823008F067C0109278
:10BF8000F6070F943D3760937504709376048093A1
:10BF9000770490937804C090A503D090A603E09016
:10BFA000A703F090A8030E94815FAB01BC014093FE
:10BFB000A5035093A6036093A7037093A8038091F1
:10BFC000300790913107A0913207B09133078C1957
:10BFD0009D09AE09BF09840F951FA61FB71F809347
:10BFE000300790933107A0933207B0933307C11104
:10BFF0000AC0C1E00E944C398C2FCF91FF90EF9086
:10C00000DF90CF90089580912E0790912F07019691
:10C0100090932F0780932E070E94815FC090340772
:10C02000D0903507E0903607F0903707C616D70650
:10C03000E806F906F0F60E94815F6093340770937A
:10C0400035078093360790933707D3CFC0E0D2CF20
:10C050001092F607109271041092720410927304F9
:10C060001092740410927504109276041092770462
:10C07000109278041092A1031092A2031092A303CD
:10C080001092A4030895CF93C091F60780E0C130C9
:10C0900069F1C23069F50E94815F6093A1037093DA
:10C0A000A2038093A3039093A40381E08093F607F7
:10C0B0000F943D37609371047093720480937304FE
:10C0C00090937404C23089F080912C0790912D07D1
:10C0D000019690932D0780932C071092A503109240
:10C0E000A6031092A7031092A80381E0CF910895B0
:10C0F0000E942860DACF8091F607813079F482E0DF
:10C100008093F6070F943D3760937504709376041F
:10C11000809377049093780481E0089580E00895F7
:10C12000CF92DF92EF92FF92FC01C080D180E2803B
:10C13000F38020E030E0A901C701B6010F943F5B16
:10C1400087FF68C0C701B601905820E030E040E2A8
:10C1500051E40F94A55B20E030E040EA50E40F94F6
:10C16000316220E030E040E251E40F942B630F9401
:10C170009D639B0160E22031F7E23F0730F0C90187
:10C1800060E177E20F940062605D6093B407283E3F
:10C1900083E0380708F445C0C90168EE73E00F94E6
:10C1A0000062CB016AE070E00F940062805D8093D2
:10C1B000B50780E22436310558F0C90164E670E025
:10C1C0000F940062CB016AE070E00F940062805D22
:10C1D0008093B60780E22A30310558F0EAE0F0E0BB
:10C1E000C901BF010F940062CB01BF010F9400622F
:10C1F000805D8093B707C9016AE070E00F94006228
:10C20000805D8093B80784EB97E0FF90EF90DF901C
:10C21000CF90089520E030E040E251E4C701B6013C
:10C2200098CF80E2C4CF8F929F92AF92BF92CF926D
:10C23000DF92EF92FF92FC01C080D180E280F38018
:10C2400020E030E040E251E4C701B6010F94A55B65
:10C2500020E030E040E251E40F94A55B4B015C012B
:10C2600020E030E0A901C701B6010F943F5B20E058
:10C2700030E040EA50E487FF04C020E030E040EACC
:10C2800050ECC501B4010F94316220E030E040E28F
:10C2900051E40F942B630F949D639B018BE237FF56
:10C2A00005C022273327261B370B8DE28093B30767
:10C2B000C90168EE73E00F941462CB01EAE0F0E08C
:10C2C000BF010F941462805D8093B407C90164E6D6
:10C2D00070E00F941462CB01BF010F941462805D73
:10C2E0008093B507C901BF010F941462282FCB01B9
:10C2F000BF010F941462805D8093B6078EE2809335
:10C30000B707205D2093B80783EB97E0FF90EF908D
:10C31000DF90CF90BF90AF909F908F900895CF9374
:10C32000DF9300D01F92CDB7DEB7809190071092B7
:10C330009007882359F0109298030E947CDA0F909E
:10C340000F900F900F90DF91CF9108956091A1070A
:10C350007091A2078091A3079091A40761157105C0
:10C360008105910561F10F94465B209100023091A7
:10C37000010240910202509103020F94A55B2091AB
:10C38000F9083091FA084091FB085091FC080F948D
:10C3900031626093F9087093FA088093FB089093D8
:10C3A000FC0883E00E9422DE81E0809377021092F5
:10C3B000A1071092A2071092A3071092A4078091E0
:10C3C0007702882309F4BBCF20919207309193071D
:10C3D00040919407509195076091F9087091FA087F
:10C3E0008091FB089091FC080F94306269837A83F6
:10C3F0008B839C83CE0101960E941361BC018AED60
:10C4000090E40E943AEB9BCF2F923F924F925F9223
:10C410006F927F928F929F92AF92BF92CF92DF9254
:10C42000EF92FF921F93CF93DF93CDB7DEB72C9798
:10C430000FB6F894DEBF0FBECDBF1C01162F809142
:10C440009007109290078823E1F0109298030E94C1
:10C450007CDA2C960FB6F894DEBF0FBECDBFDF910D
:10C46000CF911F91FF90EF90DF90CF90BF90AF9052
:10C470009F908F907F906F905F904F903F902F9004
:10C4800008958091A1079091A207A091A307B09170
:10C49000A4078D839E83AF83B887892B8A2B8B2B30
:10C4A00009F460C080910E02882309F4BDC0809118
:10C4B0000F028111B9C0613009F494C0623009F4EF
:10C4C000A2C08090100290901102A0901202B09031
:10C4D0001302C0901C02D0901D02E0901E02F0904A
:10C4E0001F02612E712C6D817E818F8198850F9442
:10C4F000465B20910002309101024091020250916E
:10C5000003020F94A55BD301AA0FBB1FAA0FBB1F89
:10C51000BC87AB87A351B74FBA87A9872D913D91AF
:10C520004D915C910F9431622B013C018D819E8174
:10C53000AF81B885B7FF8FC0A5019401C301B201D7
:10C540000F943F5B87FD7FC0EB85FC85E351F74F80
:10C550004082518262827382812F0E9422DE81E0BA
:10C56000809377021092A1071092A2071092A3075E
:10C570001092A40780917702882309F46ACFF4E02F
:10C580001F9FC0011124FC01E351F74F8F51974FBA
:10C59000DC012D913D914D915C9160817181828191
:10C5A00093810F9431626B017C01C982DA82EB8244
:10C5B000FC822DEC3CEC4CEC5DE360910002709150
:10C5C000010280910202909103020F94916487FD11
:10C5D00052C0CE0101960E941361BC01C1010E94AC
:10C5E0003AEB37CF8090140290901502A09016027B
:10C5F000B0901702C0902002D0902102E090220259
:10C60000F09023026ECF8090180290901902A090B3
:10C610001A02B0901B02C0902402D0902502E09034
:10C620002602F09027025DCF812C30E5932E33EC6B
:10C63000A32E37ECB32EC12C40E5D42E43ECE42ED0
:10C6400047E4F42E4ECFA985BA858D929D92AD9286
:10C65000BC92139781CFA7019601C301B2010F9439
:10C66000916418160CF070CFE985FA85C082D182EA
:10C67000E282F38271CF20E030E040E251E4C70172
:10C68000B6010F94A55B20E030E04AE754E40F9434
:10C69000A55B4B015C0120E030E0A901C701B601B8
:10C6A0000F943F5B20E030E040EA50E487FF04C095
:10C6B00020E030E040EA50ECC501B4010F94316253
:10C6C00020E030E040E251E40F942B630F949D632F
:10C6D0006B017C01F7FC62C020EA36E841E050E0E3
:10C6E0000F94A561CA01B9012AE030E040E050E0B2
:10C6F0000F94A561605D6093B207C701B60120E1A8
:10C7000037E240E050E00F94A5618AE0882E912C3A
:10C71000A12CB12CCA01B901A50194010F94A56106
:10C72000605D6093B307C701B60128EE33E040E0D7
:10C7300050E00F94A561CA01B901A50194010F94BD
:10C74000A561605D6093B4078EE28093B507C70171
:10C75000B60124E630E040E050E00F94A561CA0144
:10C76000B901A50194010F94A561605D6093B607BE
:10C77000C701B601A50194010F94A561162FCA0146
:10C78000B901A50194010F94A561605D6093B7079D
:10C79000105D1093B80782EB97E01FCFF094E09400
:10C7A000D094C094C11CD11CE11CF11C6DE2A3CF3C
:10C7B00062E083EE90E40C94046261E08AEE90E41F
:10C7C0000C94046260E081EF90E40C9404629C019C
:10C7D00097FF26C0EE27FF27E81BF90B2D398FEFB7
:10C7E00038070CF05DC08DE28093B507CF0164E699
:10C7F00070E00F941462CB012AE030E0B9010F948D
:10C800001462805D8093B607CF01B9010F94146262
:10C81000CB01B9010F941462805D8093B7072AC0E1
:10C82000283E83E03807B4F1C90168EE73E00F9445
:10C830001462CB01EAE0F0E0BF010F941462805D66
:10C840008093B507C90164E670E00F941462CB01D0
:10C85000BF010F941462805D8093B607C901BF01C8
:10C860000F941462CB01BF010F941462805D80931A
:10C87000B707F901CF016AE070E00F941462805DA0
:10C880008093B80785EB97E008958DE237FDC5CF1B
:10C8900080E2C3CFF90180E2243631050CF0A4CF49
:10C8A00080E28093B5078093B607EA30F1056CF318
:10C8B0008DE237FF80E28093B607CF016AE070E037
:10C8C0000F941462605D6093B707D4CF9C01EAE0D7
:10C8D000F0E0BF010F941462805D8093B8072A30A6
:10C8E0003105CCF0CB01BF010F941462805D8093C1
:10C8F000B7072436310594F0C90164E670E00F945F
:10C900001462CB01BF010F941462805D8093B6075F
:10C9100086EB97E0089588EB97E0089587EB97E022
:10C9200008959C0197FD2DC080E2243631055CF00E
:10C93000C90164E670E00F941462CB016AE070E014
:10C940000F941462805D8093B60780E22A3031052F
:10C950005CF0EAE0F0E0C901BF010F941462CB0182
:10C96000BF010F941462805D8093B707C9016AE02C
:10C9700070E00F941462805D8093B80786EB97E0B7
:10C9800008953195219531098DE2DDCF24E6829F0E
:10C99000C001112481589F4F6FEF70E00F94146213
:10C9A000262F81E3643609F080E28093B50790E298
:10C9B0002A3040F03AE0822F632F0F94E6610F9403
:10C9C000E661905D9093B607822F6AE00F94E6616E
:10C9D000905D9093B70785E28093B80785EB97E069
:10C9E00008958F929F92AF92BF92CF92DF92EF9273
:10C9F000FF920F931F93CF93DF93CDB7DEB72C97A2
:10CA00000FB6F894DEBF0FBECDBF8B0140E050E003
:10CA100068E472E44D835E836F83788740E050E082
:10CA200060EA70E449875A876B877C878130B9F167
:10CA3000823009F459C020E030E040E050E46091D9
:10CA4000F5087091F6088091F7089091F8080F9416
:10CA500031624B017C0120E030E046E953E40F9461
:10CA60009164181634F4812C912C86E9E82E93E415
:10CA7000F92EF801A084B184C284D3849401A70163
:10CA8000B501C6010F949164181614F054016701A2
:10CA9000C501D60189839A83AB83BC8348C0BE019C
:10CAA000675F7F4FC80108960E94AF50B8016C5F66
:10CAB0007F4FAE014B5F5F4FC8010E948D500E94B7
:10CAC00054592C960FB6F894DEBF0FBECDBFDF9140
:10CAD000CF911F910F91FF90EF90DF90CF90BF907B
:10CAE000AF909F908F900895F80120853185428501
:10CAF00053856091F5087091F6088091F708909140
:10CB0000F8080F9431626B017C0120E030E046E9C7
:10CB100053E40F943F5B87FD06C0C12CD12C26E95E
:10CB2000E22E23E4F22EC982DA82EB82FC82BE017D
:10CB3000675F7F4FCE010196B7CF2F923F924F9202
:10CB40005F926F927F928F929F92AF92BF92CF929D
:10CB5000DF92EF92FF920F931F93CF93DF9300D05A
:10CB600000D0CDB7DEB70F943D3700912507109167
:10CB70002607209127073091280701151105210567
:10CB8000310509F00AC32091AE15222309F44AC0E9
:10CB9000E091AC1521502093AE1521E02E0F20938B
:10CBA000AC153091AF15231302C01092AC1524E0E0
:10CBB000E29FF0011124E055FA4E0081118122819B
:10CBC000338100932107109322072093230730938A
:10CBD0002407600F711F811D911D609325077093BD
:10CBE0002607809327079093280780912307909129
:10CBF0002407892BB9F08FB78E83F89420902107F2
:10CC0000309022072101712C612C00912307109193
:10CC1000240780915C028532F1F08F3F09F495C0C2
:10CC20009E819FBF26960FB6F894DEBF0FBECDBF84
:10CC3000DF91CF911F910F91FF90EF90DF90CF90F8
:10CC4000BF90AF909F908F907F906F905F904F902C
:10CC50003F902F900895EDE3FEE394919D8397FD1F
:10CC6000DFCF85E20F94CA1B8D81882321F09D813F
:10CC7000923009F0BCC14801B12CA12C60E072E1F6
:10CC80008AE790E0A50198010F94A56129833A8372
:10CC90004B835C8369017A0121E0C21AD108E10863
:10CCA000F1088FEFC816D104E104F10409F00CF487
:10CCB0006EC160E472E48FE090E0A50198010F94EA
:10CCC000A56169017A0191E0C91AD108E108F1086A
:10CCD0002D81223009F00FC18FEFC816D104E10475
:10CCE000F10409F00CF4BFC260E970ED83E090E05C
:10CCF000A50198010F94A56169017A0191E0C91A13
:10CD0000D108E108F10883E02FEFC216D104E10455
:10CD1000F10409F00CF4A0C268E478EE81E090E040
:10CD2000A50198010F94A56169017A0181E0C81AF3
:10CD3000D108E108F1089FEFC916D104E104F1041C
:10CD400011F00CF0FCC084E087C285E280935C02A5
:10CD5000EDE3FEE324912D83822F2F3F09F460CF72
:10CD6000223009F468C058F4222379F1213009F403
:10CD700044C087FD55CF85E20F94CA1B78CF9D81B3
:10CD8000943009F49AC008F478C0953091F7109265
:10CD9000200110922101809121018860809321015E
:10CDA00080912101816080932101E0E3F2E4E4912C
:10CDB000F0E0EE0FFF1FE952FE4B85919491E6E7FC
:10CDC000F2E4E491E0933D044CCF14BC15BC84B56F
:10CDD000826084BD85B5816085BDE0E3F2E4E491C5
:10CDE000F0E0EE0FFF1FE952FE4B85919491E6E7CC
:10CDF000F2E4E491E093410434CF10928000109269
:10CE00008100809181008860809381008091810001
:10CE1000816080938100E0E3F2E4E491F0E0EE0FC2
:10CE2000FF1FE952FE4B85919491E6E7F2E4E4910D
:10CE3000E093400416CF1092B0001092B1008091A0
:10CE4000B00082608093B0008091B10081608093D7
:10CE5000B100E0E3F2E4E491F0E0EE0FFF1FE952ED
:10CE6000FE4B8591949190931A0780931907E6E7FA
:10CE7000F2E4E491E0931B07F4CE1092900010923C
:10CE80009100809191008860809391008091910041
:10CE9000816080939100E0E3F2E4E491F0E0EE0F32
:10CEA000FF1FE952FE4B85919491E6E7F2E4E4918D
:10CEB000E0933F0423E02D83D4CE1092A000109283
:10CEC000A1008091A10088608093A1008091A100C1
:10CED00081608093A100E0E3F2E4E491F0E0EE0FE2
:10CEE000FF1FE952FE4B85919491E6E7F2E4E4914D
:10CEF000E0933E04B6CE8FEFC816D104E104F104EE
:10CF000009F00CF472C068E478EE81E090E0A501CD
:10CF100098010F94A56169017A0191E0C91AD108BD
:10CF2000E108F1082D81222309F462C12FEFC21616
:10CF3000D104E104F10411F00CF063C104CF64E208
:10CF400074EF80E090E0A50194010F94A561690160
:10CF50007A0181E0C81AD108E108F10885E09FEF65
:10CF6000C916D104E104F10409F008F475C162E1C5
:10CF70007AE780E090E0A50194010F94A561690132
:10CF80007A0181E0C81AD108E108F1084CC181E0BA
:10CF90002D81211161C195B5987F892B85BD2FEF1A
:10CFA0003FEFA90145284628472809F048C09D8140
:10CFB000923009F4E2C00CF0C9C0992309F4CEC044
:10CFC000913009F02DCED0928900C0928800209334
:10CFD0004E0430934F044093500450935104809179
:10CFE0006F00826080936F001BCE82E0D1CFB12CA6
:10CFF000A12C60E072E18AE790E0A50198010F940E
:10D00000A56169017A0181E0C81AD108E108F10837
:10D01000C114D10491E0E906F104F4F491E02D810A
:10D02000213059F580918100887F892B8093810080
:10D030002FEF3FEFA90145284628472821F2980104
:10D04000220F331FD1010F94D76128EE33E040E067
:10D0500050E00F948361ABCF68E478EE81E090E01C
:10D06000A50198010F94A56169017A0181E0C81AB0
:10D07000D108E108F10893E0D2CF8D818330F9F433
:10D0800080919100887F892B809391002FEF3FEF53
:10D09000A90145284628472891F6D0929900C092C8
:10D0A000980020934A0430934B0440934C045093CF
:10D0B0004D0480917100826080937100B1CD2D810B
:10D0C000243001F58091A100887F892B8093A100F5
:10D0D0002FEF3FEFA90145284628472809F0AFCF99
:10D0E000D092A900C092A800209346043093470430
:10D0F0004093480450934904809172008260809369
:10D1000072008ECD8D81853009F049CF809121014B
:10D11000887F892B809321012FEF3FEFA9014528BC
:10D120004628472809F08BCFD0922901C0922801C8
:10D1300020934204309343044093440450934504A5
:10D14000809173008260809373006ACD8D818430FA
:10D1500039F20CF4A2CF853039F362CDC7BC2093ED
:10D1600052043093530440935404509355048091D7
:10D170006E00826080936E0053CDC092B300209306
:10D180001C0730931D0740931E0750931F07809183
:10D19000700082608093700043CD601B710B820B26
:10D1A000930B97FD3FCD40981092250710922607CC
:10D1B000109227071092280735CDC980DA80EB80BE
:10D1C000FC809AE0F594E794D794C7949A95D1F7A8
:10D1D00021E0C21AD108E108F10885E0DCCE8FEF2A
:10D1E000C816D104E104F10409F038F784E0D3CE85
:10D1F00083E09FEFC916D104E104F10409F00CF4B7
:10D20000CACE62E17AE780E090E0A50194010F9434
:10D21000A56169017A0181E0C81AD108E108F10825
:10D220009D819923E1F286E02FEFC216D104E1043B
:10D23000F10491F088F0C980DA80EB80FC808AE00C
:10D24000F594E794D794C7948A95D1F791E0C91AD9
:10D25000D108E108F10887E09091B100987F892B0F
:10D260008093B1009CCE82E0F7CF0F931F93CF93B2
:10D27000DF938C01EB019091AE152091AF159213C5
:10D2800005C00E949D650E94D551F5CF8091AD15D6
:10D2900034E0839FF0011124E055FA4E118300839E
:10D2A000D383C2839F5F9093AE158F5F281739F0A9
:10D2B0008093AD15DF91CF911F910F91089510923A
:10D2C000AD15F8CF8F929F92AF92BF92CF92DF921F
:10D2D000EF92FF92CF936B017C0120E030E0A90137
:10D2E0000F943F5B87FFA3C06DEB77E386E095EB80
:10D2F000A70196010F9431626B017C0120E030E0C0
:10D3000040E251E40F94A55B20E030E048EC52E4A9
:10D310000F94A55B4B015C0120E030E040E251EC52
:10D32000C701B6010F943F5B181654F420E030E0BB
:10D3300048EC52E4C701B6010F94916487FD8BC09D
:10D3400020E030E0A901C701B6010F943F5B87FFE1
:10D3500073C060E070E080EA90ECA50194010F9446
:10D36000316220E030E040E251E40F942B630F94EF
:10D370009D636B017C01F7FC64C020E137E240E073
:10D3800050E00F94A561CA01B9012AE030E040E005
:10D3900050E00F94A561605D6093B307C701B601CB
:10D3A00028EE33E040E050E00F94A5619AE0892E2A
:10D3B000912CA12CB12CCA01B901A50194010F94A3
:10D3C000A561605D6093B407C701B60124E630E053
:10D3D00040E050E00F94A561CA01B901A501940194
:10D3E0000F94A561605D6093B5078EE28093B607E8
:10D3F000C701B601A50194010F94A561C62FCA010A
:10D40000B901A50194010F94A561605D6093B70710
:10D41000C05DC093B80783EB97E0CF91FF90EF908A
:10D42000DF90CF90BF90AF909F908F9008956DEB5D
:10D4300077E386E095E35CCF60E070E080EA90E41B
:10D440008CCFF094E094D094C094C11CD11CE11C0A
:10D45000F11C6DE2A1CF20E030E0A901C701B601C7
:10D460000F943F5B87FF6AC060E070E080EA90EC59
:10D47000A50194010F94316220E030E040E251E4D4
:10D480000F942B630F949D634B015C0120E030E00F
:10D49000A901C701B6010F94916487FD0BC020E07C
:10D4A00030E040E251E4C701B6010F943F5B60E217
:10D4B00087FD13C0B7FC47C0C501B40128EE33E0B7
:10D4C00040E050E00F94A561CA01B9012AE030E0C4
:10D4D00040E050E00F94A561605D6093B407C50122
:10D4E000B40124E630E040E050E00F94A5618AE00A
:10D4F000C82ED12CE12CF12CCA01B901A70196014B
:10D500000F94A561605D6093B5078EE28093B607C6
:10D51000C501B401A70196010F94A561C62FCA01E8
:10D52000B901A70196010F94A561605D6093B707EB
:10D53000C05DC093B80784EB97E06FCF60E070E008
:10D5400080EA90E495CFB094A09490948094811C4C
:10D55000911CA11CB11C6DE2C0CFCF93DF93EC01F5
:10D560000E9492D920E040E070E060E0CE01DF91BF
:10D57000CF910C94D7D8FF920F931F93CF93DF9343
:10D5800061E081E00E947FD8D0919707C0E0FF243E
:10D59000F394D11148C080919607882391F180912E
:10D5A0007702882361F081E090919607911180E0E5
:10D5B00003E023E046EC57E06C2F0E9478ED809169
:10D5C0002F0980939A07D43009F04DC010929B0325
:10D5D00080919607843009F4E1C080917702882316
:10D5E00009F4B2C111E080919607843009F010E08F
:10D5F00080919A070E94C66400E09C0149EA57E0C6
:10D600002EC08091900710929007882341F20E94CB
:10D610007CDA8091B107882311F2DF91CF911F91BD
:10D620000F91FF900895D13009F063C08091960763
:10D63000813009F445C0809177028823A1F011E080
:10D6400080919607813009F010E0809169029091F5
:10D650006A020E94916400E09C0140EC57E06C2F4C
:10D66000812F0E94F5EC8091300980939A07D53084
:10D6700009F0BEC0F0929B0380919607853009F4B3
:10D68000A2C080917702882391F011E080919607E3
:10D69000853009F010E080919A070E94C66400E08E
:10D6A0009C0149EA57E06C2F812F0E94F5ECDF5F67
:10D6B000CF5FC43009F06DCF89E080939107ADCF83
:10D6C0008091900710929007882309F4B4CF10E05E
:10D6D00000E027EE33E04AE050E069E672E080ECDB
:10D6E00097E00F9475338091B107882309F4A3CF95
:10D6F00094CFD23009F0F0C0809196078230D1F0FB
:10D7000080917702882309F4AECF11E080919607CB
:10D71000823009F010E080910C1590910D150E9457
:10D72000916400E09C0149EB57E06C2F812F0E942F
:10D73000F5EC45CF8091900710929007882301F374
:10D740000F94F6300BE917E223EB31E050E040E0B4
:10D750006CE075E189EB97E00F9475338091B10728
:10D76000882371F25ACF80919007109290078823F6
:10D7700009F4BAC00F94F6300AE214E22CE830E063
:10D7800050E040E063E078E085EB97E00F9475337C
:10D790008091B107882309F4A7C03FCF80919007FB
:10D7A00010929007882309F418CF0F94F63060EE9A
:10D7B00073E289EA97E00F94AE348091B107882331
:10D7C00009F40BCF2ACF80919007109290078823FD
:10D7D00009F457CF0F94F63060EE73E289EA97E0D0
:10D7E0000F94AE348091B107882309F44ACF15CF46
:10D7F000D63089F5809196078630B1F08091770216
:10D80000882309F454CF11E080919607863009F0FF
:10D8100010E080910C0290910D020E94916400E052
:10D820009C0144EA57E03FCF809190071092900707
:10D83000882321F30DEB13E227EE33E04AE050E0BA
:10D840006CE072E084EA97E00F9475338091B10741
:10D850008823A1F2E2CED73009F05CC08091960710
:10D860008730D1F080917702882309F420CF11E02E
:10D8700080919607873009F010E060912709709138
:10D8800028098091290990912A090E94626900E083
:10D890009C014AE957E007CF8091900710929007CA
:10D8A000882301F367E279E08AE997E00F946A340C
:10D8B0008091B1078823B1F2B0CE80919007109289
:10D8C0009007882371F180E89BEE0E94AD6A8091F9
:10D8D000B107882331F1A1CED33009F070CE809109
:10D8E0009607833009F43FCF80917702882309F4AB
:10D8F000BACE11E080919607833009F010E0809154
:10D900000308909104080E94916400E09C0145EB9B
:10D9100057E00BCFD83009F0CACE809196078830F7
:10D9200061F280917702882309F4C1CE81E0909161
:10D930009607983009F080E00EE32EE34BE857E0BD
:10D940006C2F0E9478EDB3CE8091300980939A07B6
:10D95000AECE8F929F92AF92BF92CF92DF92EF9214
:10D96000FF920F931F93CF93DF9399249394809109
:10D970000C1590910D15892B09F4912C61E081E033
:10D980000E947FD8D0919707C0E08824839494EDBB
:10D99000C92E92E3D92E2CE5A22E27E0B22ED1116A
:10D9A000B4C080919607882309F494C080917702CF
:10D9B000882361F081E090919607911180E003E067
:10D9C00023E046E857E06C2F0E9478ED8091300903
:10D9D00080939A07D430E9F480929B038091960754
:10D9E000843009F43FC180917702882391F011E0DF
:10D9F00080919607843009F010E080919A070E9488
:10DA0000C66400E09C014FE657E06C2F812F0E9416
:10DA1000F5ECF12CE12C15E0E0929A07D11320C02F
:10DA2000F701EE0FFF1FE85AF84F859194919093FC
:10DA30009A0380939903809196078D1709F427C163
:10DA400080917702882361F081E09091960791138D
:10DA500080E00EE32EE345E657E06C2F0E9478ED60
:10DA6000812F9FEFE91AF90A16E08630A9F6809116
:10DA7000030890910408892B19F4992009F427C10F
:10DA8000D730E9F480919607873009F411C180916D
:10DA900077028823A1F0DF92CF92BF92AF92CF930B
:10DAA00081E090919607973009F080E08F930E9473
:10DAB000BBFD0F900F900F900F900F900F9088E08C
:10DAC00099249394DF5FCF5FC43009F068CF8093CF
:10DAD00091070EC08091900710929007882309F457
:10DAE00065CF0E947CDA8091B107882309F45ECF6C
:10DAF000DF91CF911F910F91FF90EF90DF90CF902A
:10DB0000BF90AF909F908F900895D13009F05FC083
:10DB100080919607813009F43FC080917702882375
:10DB200009F454CF11E080919607813009F010E09C
:10DB300080910C1590910D150E94916400E09C015C
:10DB40004FE757E06C2F812F0E94F5EC80912F0951
:10DB500080939A07D33009F039CF10929B038091BC
:10DB60009607833009F469C080917702882309F40D
:10DB700050CF11E080919607833009F010E080913A
:10DB80009A070E94C66400E09C014FE657E06C2FA4
:10DB9000812F0E94F5EC1ACF809190071092900788
:10DBA000882309F4BACF0F94F63009E917E223EB82
:10DBB00031E050E040E06CE075E18FE797E00F94D2
:10DBC00075338091B107882309F4A7CF91CFD23064
:10DBD00009F0BCCF809196078230B1F08091770236
:10DBE000882309F4F3CE11E080919607823009F082
:10DBF00010E080910308909104080E94916400E075
:10DC00009C014BE757E09ECF8091900710929007C0
:10DC1000882321F30F94F6300AE214E22CE830E076
:10DC200050E040E063E078E08BE797E00F947533D5
:10DC30008091B107882391F25BCF80919007109279
:10DC40009007882309F490CF0F94F63060EE73E2CA
:10DC50008FE697E00F94AE348091B107882309F4E2
:10DC600083CF46CF8091900710929007882309F4C4
:10DC7000BACE0F94F63060EE73E28FE697E00F9421
:10DC8000AE348091B107882309F4ADCE31CF8091B5
:10DC9000900710929007882309F4D2CE81E499E28C
:10DCA0000E94AD6A8091B107882309F4C9CE20CFC4
:10DCB0008091900710929007882309F4E8CE0E9483
:10DCC000D4328091B107882309F4E1CE11CF87E0E7
:10DCD000F9CE0F931F93CF93DF9361E081E00E9411
:10DCE0007FD8D0919707C0E013E0D11126C0809172
:10DCF0009607882389F080917702882341F181E09B
:10DD000090919607911180E003E023E044E856E00B
:10DD10006C2F0E9478ED1BC08091900710929007A5
:10DD2000882349F30E947CDA8091B107882319F394
:10DD3000DF91CF911F910F910895D130A9F5909166
:10DD40009607913061F08091770281111AC0DF5FF0
:10DD5000CF5FC43051F686E080939107E9CF809180
:10DD6000900710929007882371F380910E028D27FF
:10DD700080930E02109377028091B107882319F3E4
:10DD8000D7CF81E0913009F080E090910E022AED2A
:10DD900036E0911102C026ED36E001E046E756E09C
:10DDA0006C2F0E94F5ECD3CFD23009F077C0809170
:10DDB0009607823079F080917702882341F281E0E2
:10DDC00090919607923009F080E00EE32EE341EF48
:10DDD00050E49ECF8091900710929007882359F3CA
:10DDE00086E49AE20E94AD6A8091B107882319F314
:10DDF0009FCF80919607833081F0809177028823AE
:10DE000009F4A5CF81E090919607933009F080E066
:10DE10000EE32EE34AEE50E47BCF80919007109200
:10DE20009007882351F381E49AE20E94AD6A8091C1
:10DE3000B107882311F37CCF80919607843081F05D
:10DE400080917702882309F482CF81E09091960730
:10DE5000943009F080E00EE32EE343EE50E458CF17
:10DE60008091900710929007882351F38CE39AE2F7
:10DE70000E94AD6A8091B107882311F359CF809138
:10DE80009007109290078823A9F084EA98E20E94F4
:10DE9000AD6A8091B107882369F04ACFD33009F485
:10DEA000A8CFD43049F2D53009F051CF80919607F0
:10DEB000853029F380917702882309F448CF81E0E7
:10DEC00090919607953009F080E00EE32EE34AED3D
:10DED00050E41ECFCF92DF92EF92FF926B017C0154
:10DEE00020E030E0A9010F943F5B87FD26C06DEB79
:10DEF00077E386E095E3A70196010F9431626B0109
:10DF00007C0120E030E0A9010F943F5B20E030E08D
:10DF100040E05FE387FF04C020E030E040E05FEBDB
:10DF2000C701B6010F9431620F949D63CB01FF903E
:10DF3000EF90DF90CF900C9491646DEB77E386E0E7
:10DF400095EBD9CF2F923F924F925F926F927F9233
:10DF50008F929F92AF92BF92CF92DF92EF92FF92F9
:10DF60000F931F93CF93DF9361E081E00E947FD8EE
:10DF7000C0919707D0E0222423946FEA662E66E0D2
:10DF8000762E7CE9472E76E0572EC11182C0809113
:10DF90009607882309F45CC080917702882361F09A
:10DFA00081E090919607911180E003E023E04BE23D
:10DFB00057E06D2F0E9478ED80919C038770873029
:10DFC00009F02EC120E030E0A90160911E0470919B
:10DFD0001F0480912004909121040F943F5B8823BB
:10DFE00009F41EC1C73089F51091FC07809196078E
:10DFF0008730A1F48091900710929007882371F0E8
:10E00000122583E08093770288E894ED892B11F044
:10E010000E9488D48091B107811128C08091770235
:10E02000882309F409C281E090919607973009F09E
:10E0300080E02AED36E0111102C026ED36E001E065
:10E040004DED56E06D2F0E94F5EC48E0342EEAC00D
:10E050008091900710929007882309F49DCF0E9429
:10E060007CDA8091B107882309F496CFDF91CF91B4
:10E070001F910F91FF90EF90DF90CF90BF90AF90E6
:10E080009F908F907F906F905F904F903F902F90D8
:10E090000895C13019F580919607813081F0809103
:10E0A0007702882309F488CF81E090919607913018
:10E0B00009F080E00EE32EE340ED50E47ACF80914A
:10E0C000900710929007882351F389E69EE60E94FC
:10E0D000AD6A8091B107882311F3C8CFC23009F02F
:10E0E0008CC190919607923071F0809177028823CD
:10E0F00009F462CF81E0923009F080E000E22EE383
:10E100004DE157E056CF80919007109290078823F9
:10E1100061F327E237E03093410720934007809175
:10E12000B107882311F3A2CF90919607933071F035
:10E1300080917702882309F43FCF81E0933009F082
:10E1400080E000E22EE341E157E033CF8091900779
:10E1500010929007882361F328E137E0309341075C
:10E16000209340078091B107882311F37FCF9091CE
:10E170009607943071F080917702882309F41CCFC0
:10E1800081E0943009F080E000E22EE345E057E0C2
:10E1900010CF8091900710929007882361F32CE0B4
:10E1A00037E030934107209340078091B1078823DF
:10E1B00011F35CCF90919607953071F080917702C2
:10E1C000882309F4F9CE81E0953009F080E000E27F
:10E1D0002EE349EF56E0EDCE809190071092900724
:10E1E000882361F320E037E0309341072093400714
:10E1F0008091B107882311F339CF80919007109255
:10E200009007882309F40AC124EF36E030934107D0
:10E21000209340078091B107882309F4FFC026CFDF
:10E2200057E0352E8091F8079091F907A091FA07F1
:10E23000B091FB0780939A0790939B07A0939C074C
:10E24000B0939D073C1220C080919607831509F476
:10E250006CC0809177028823B9F011E08091960715
:10E260008C1310E060919A0770919B0780919C0736
:10E2700090919D070E946A6F00E09C014AEC56E075
:10E280006D2F812F0E94F5EC81E0830D8C1315C05A
:10E29000809196078C1709F47DC0809177028823BE
:10E2A00061F081E0909196079C1380E00EE32EE3ED
:10E2B0004CEB56E06D2F0E9478ED82E0830D8C13BD
:10E2C00013C0909196079C1709F475C0809177024E
:10E2D000882351F081E09C1380E000E22EE340EAC5
:10E2E00056E06D2F0E9478ED83E0830D8C1313C0F0
:10E2F000909196079C1709F46FC08091770288234C
:10E3000051F081E09C1380E000E22EE34BE856E000
:10E310006D2F0E9478EDCF5FDF5FD43009F035CEEE
:10E3200084E0830D80939107A1CE80919007109295
:10E330009007882309F48DCF0F94F63020E030E069
:10E34000A90160919A0770919B0780919C07909119
:10E350009D070F9431620F94A46397E9892E98E288
:10E36000992E29EBA22E2CEEB22E6B0114E6E12E93
:10E37000F12C00E010E020E030E0A9016AE977E04C
:10E380008AEC96E00F949D318091B107882309F4BF
:10E3900060CF6CCE8091900710929007882309F48B
:10E3A0007CCF81E799ED0E94AD6A8091B107882307
:10E3B00009F473CF5BCE8091900710929007882369
:10E3C00009F484CF70924107609240078091B107B1
:10E3D000882309F47BCF4ACE809190071092900752
:10E3E000882309F48ACF50924107409240078091D8
:10E3F000B107882309F481CF39CEC33009F494CE14
:10E40000C43009F4B4CEC53009F4D4CEC63009F016
:10E41000D3CD90919607963009F4EFCE8091770294
:10E42000882309F4C9CD81E0963009F080E000E24C
:10E430002EE34AEE56E0BDCD8091F8079091F907A2
:10E44000A091FA07B091FB0780939A0790939B07DE
:10E45000A0939C07B0939D0788E0382E15CFCF92EC
:10E46000DF92EF92FF920F931F93CF93DF93C82F0A
:10E4700011E01827811102C00E94CAA181E59EE027
:10E480000E9439928BE49EE00E9439928AE00E94B9
:10E490001192C11102C00E94CAA18EE29EE00E94A8
:10E4A00039928AE00E941192C11114C00E94CAA13F
:10E4B00087EA9BE00E9439928BE19EE00E943992AC
:10E4C00080911608882309F424C38AE00E941192DF
:10E4D0000E94CAA16091160870E087E09EE00E9449
:10E4E000EE944091120850911308609114087091B5
:10E4F000150884E09EE00E9458948AE00E941192E0
:10E5000041E064EF7DE08C2F0E947D27812F0F94E6
:10E51000E22D41E067ED7DE08C2F0E947D27C11147
:10E5200002C00E94CAA140911A1050911B10609124
:10E530001C1070911D108EEC9DE00E94589440912B
:10E540001E1050911F1060912010709121108BE7C8
:10E5500091E40E94589440912210509123106091B0
:10E5600024107091251088E791E40E9458944091FE
:10E57000261050912710609128107091291085E77E
:10E5800091E40E9458948AE00E94119241E06DEA61
:10E590007DE08C2F0E947D27C11102C00E94CAA17C
:10E5A0006091F60F7091F70F8091F80F9091F90F2D
:10E5B0000F94445BAB01BC0184EA9DE00E94589437
:10E5C0006091FA0F7091FB0F8091FC0F9091FD0FFD
:10E5D0000F94445BAB01BC018BE791E40E9458941B
:10E5E0006091FE0F7091FF0F8091001090910110CB
:10E5F0000F94445BAB01BC0188E791E40E945894FE
:10E600006091021070910310809104109091051098
:10E610000F94445BAB01BC0185E791E40E945894E0
:10E620008AE00E94119241E06BE57DE08C2F0E9410
:10E630007D27C11102C00E94CAA140912A105091A9
:10E640002B1060912C1070912D1082E59DE00E949E
:10E65000589440912E1050912F106091301070916D
:10E6600031108FE49DE00E945894409132105091F7
:10E67000331060913410709135108CE49DE00E944D
:10E6800058948AE00E94119241E06CEC7CE08C2F5F
:10E690000E947D27C11102C00E94CAA1609106108C
:10E6A0007091071080910810909109100F94445BAD
:10E6B000AB01BC0183EC9CE00E9458944091361061
:10E6C00050913710609138107091391080EC9CE0B7
:10E6D0000E94589440913A1050913B1060913C1028
:10E6E00070913D108CE49DE00E9458944091170970
:10E6F000509118096091190970911A098DEB9CE0ED
:10E700000E94589440911B0950911C0960911D0969
:10E7100070911E098BE791E40E94589440911F0963
:10E7200050912009609121097091220988E791E4B4
:10E730000E94589440912309509124096091250921
:10E740007091260985E791E40E9458948AE00E941E
:10E75000119241E060EB7CE08C2F0E947D27C1117B
:10E7600002C00E94CAA140912308509124086091E0
:10E7700025087091260887EA9CE00E9458944091F1
:10E780002708509128086091290870912A088BE782
:10E7900091E40E94589440912B0850912C0860916C
:10E7A0002D0870912E0888E791E40E9458948AE021
:10E7B0000E94119241E064E97CE08C2F0E947D2749
:10E7C000C11102C00E94CAA16091FC0770E08BE8F1
:10E7D0009CE00E94EE944091F8075091F9076091F7
:10E7E000FA077091FB0788E791E40E9458948AE049
:10E7F0000E94119220E030E0A90160911E04709106
:10E800001F0480912004909121040F943F5B882382
:10E8100081F182EBE82E83E0F82E10E0670100E042
:10E82000C11102C00E94CAA1602F81E89CE00E9431
:10E830005094612F8EE79CE00E94509488E791E409
:10E840000E943992F601608171818281938145E055
:10E850000E94572E8AE00E9411920F5FF4E1CF0EC2
:10E86000D11C0530E9F61F5F84E0E80EF11C15307D
:10E87000A9F641E062E67CE08C2F0E947D2704E847
:10E8800017E0D0E0C11102C00E94CAA16D2F89E536
:10E890009CE00E945094F80160817181072E000C69
:10E8A000880B990B0F94465BAB01BC0186E59CE09D
:10E8B0000E945894F80162817381072E000C880B26
:10E8C000990B0F94465BAB01BC0180E491E40E947C
:10E8D0005894F8016481758183E59CE00E94469418
:10E8E0008AE00E9411920A5F1F4FD13009F016C1D1
:10E8F00041E065E47CE08C2F0E947D27C11102C0BD
:10E900000E94CAA140910F155091101560911115E8
:10E91000709112158CE39CE00E9458942CEA35EC1F
:10E9200047E25EE3609113157091141580911515FF
:10E93000909116150F942B63AB01BC0189E39CE009
:10E940000E9458942CEA35EC47E25EE3609117157B
:10E95000709118158091191590911A150F94A55B57
:10E96000AB01BC0186E39CE00E9458948AE00E94BF
:10E970001192C11102C00E94CAA140910608509193
:10E98000070860910808709109088DE29CE00E94D8
:10E9900058942CEA35EC47E25EE360910A087091E6
:10E9A0000B0880910C0890910D080F942B63AB011C
:10E9B000BC018AE29CE00E9458942CEA35EC47E2C4
:10E9C0005EE360910E0870910F088091100890919D
:10E9D00011080F94A55BAB01BC0187E29CE00E948B
:10E9E00058948AE00E94119241E062E17CE08C2F11
:10E9F0000E947D27C11102C00E94CAA16091B1038B
:10EA000070E089E09CE00E94EE948AE00E941192FE
:10EA100040E06AEF7BE08C2F0E947D27C1110AC085
:10EA20008BE49EE00E9439928AEA9BE00E94399230
:10EA30000E94CAA10091851510918615F8014081A8
:10EA400051816281738181EF9BE00E945894F801AB
:10EA500044815581668177818BE791E40E945894C7
:10EA600040918115509182156091831570918415A4
:10EA700088E791E40E9458948AE00E94119241E054
:10EA800061EE7BE08C2F0E947D27C11102C00E94A5
:10EA9000CAA14091270950912809609129097091D4
:10EAA0002A0988ED9BE00E9458948AE00E94119206
:10EAB00041E06AEB7BE08C2F0E947D27C11102C0F0
:10EAC0000E94CAA18DEA9BE00E9439924091AD0359
:10EAD0005091AE036091AF037091B00388EB9BE05F
:10EAE0000E9458944091A9035091AA036091AB03EE
:10EAF0007091AC0385EB9BE00E9458948AE0DF9113
:10EB0000CF911F910F91FF90EF90DF90CF900C94D9
:10EB1000119280E19EE00E943992DACCD1E0B2CE2F
:10EB20002F923F924F925F926F927F928F929F921D
:10EB3000AF92BF92CF92DF92EF92FF920F931F930B
:10EB4000CF93DF93CDB7DEB7C558D1090FB6F89490
:10EB5000DEBF0FBECDBF2DB73EB7CC57DF4F3983D9
:10EB60002883C458D04001E02BE834E044E050E072
:10EB7000BE0167587F4F85E894E00E94E68F2BE83E
:10EB800034E042E050E0BE0163587F4F85E894E0F6
:10EB90000E94E68F43E050E0BE0167587F4F83ED4F
:10EBA00092E00F949665892B09F443C0ED968FADE2
:10EBB000ED97882339F08FE3EA968FAFEA97EB96CB
:10EBC0001FAEEB9781E080938D0480912604811124
:10EBD00007C080918307813019F480E00E942F7272
:10EBE00090918D0481E08927CC57DF4F28813981AE
:10EBF000C458D0400FB6F8943EBF0FBE2DBFCB57C0
:10EC0000DF4F0FB6F894DEBF0FBECDBFDF91CF91BF
:10EC10001F910F91FF90EF90DF90CF90BF90AF903A
:10EC20009F908F907F906F905F904F903F902F902C
:10EC30000895E9961CAE1DAE1EAE1FAEE997109268
:10EC40008C0410928B04CE018F579F4F0E94452851
:10EC5000ADB6BEB6CF57DF4FC880C158D040D12C1B
:10EC600033E0C30ED11CCC0CDD1CCC0CDD1C8DB7ED
:10EC70009EB78C199D090FB6F8949EBF0FBE8DBF2D
:10EC8000EDB7FEB73196CE57DF4FF983E883C25810
:10EC9000D0402DB73EB72C193D090FB6F8943EBFB2
:10ECA0000FBE2DBF8DB79EB701964C01EDB7FEB7D5
:10ECB000EC19FD090FB6F894FEBF0FBEEDBF2DB7DE
:10ECC0003EB72F5F3F4F7901B601CE57DF4F8881A6
:10ECD0009981C258D0400E9452280091260481E0B8
:10ECE00008272BE834E044E050E066E070E185E876
:10ECF00094E00E94E68FB601C4010E945228B6013A
:10ED0000C7010E94522800912604011157C0CF5715
:10ED1000DF4F8881C158D04090E00296A6EFBFE057
:10ED200050E040E030E020E064E97EE0E4E8CE2E10
:10ED3000EEE0DE2E821793070CF499C0CE57DF4F1A
:10ED4000E881F981C258D040E40FF51F408051801E
:10ED5000628073804D925D926D927D9282179307CF
:10ED60000CF48BC0F401E40FF51F20803180128178
:10ED7000E3812101612E7E2E50964D925D926D921F
:10ED80007C925397821793070CF480C0F701E40F2D
:10ED9000F51F208031801281E3812101612E7E2EBA
:10EDA00090964D925D926D927C9293972F5F3F4F1C
:10EDB0004C5F5F4F2430310509F0BCCF8AE290E10F
:10EDC0000E94E5278EE290E10E94E52782E390E130
:10EDD0000E94E52786E390E10E94E5278AE390E11F
:10EDE0000E94E52781E008272BE834E040E150E06D
:10EDF00067E179E085E894E00E94E68FCE018B58C8
:10EE00009F4F0E94E5270FB6F894BEBE0FBEADBE61
:10EE100083E298E00E943528CE0183599F4F0E94DB
:10EE2000F527CE0101967C010E94E52787E894E052
:10EE30000E94E527CE018B589F4F0E94E527C7010E
:10EE40000E944528CE0183599F4F0E944528098181
:10EE5000AE968FADAE97089F800111240150110925
:10EE6000F8F0CE018B589F4F0E94E527F7CFFB01AA
:10EE700045905590659074906DCFF60145905590F2
:10EE8000659074901201162DE72D73CFE4E7FEE034
:10EE900045905590659074901201162DE72D7DCF09
:10EEA00089E795E10E9435281AE01150CE0129F03A
:10EEB0008B589F4F0E94E527F8CF81589F4F0E94A3
:10EEC0004528CE0180589F4F0E944528C158DF4FEA
:10EED0008881CF57D040853009F0CCC1C058DF4F72
:10EEE0008881C058D040853009F0C4C18091260483
:10EEF000811102C00E945B8D8EE194E00E94252862
:10EF000086E194E00E9425280091260481E00827EC
:10EF10002BE834E044E650E062EB73E085E894E0EF
:10EF20000E94E68FC7010E941528CE0183599F4F8A
:10EF30000E94F5270091260411E001272BE834E018
:10EF400044E050E0B70185E894E00E94E68F8FE34B
:10EF500097E00E9415280091260401272BE834E051
:10EF60004CE050E064E877E085E894E00E94E68FAA
:10EF70000091260401272BE834E044E150E0B7017A
:10EF800085E894E00E94E68F00912604011138C0C4
:10EF900089809A80AB80BC80A5019401C501B40131
:10EFA0000F94236581112CC080920F15909210153B
:10EFB000A0921115B09212152CEA35EC47E25EE3EF
:10EFC0006D817E818F8198850F94A55B6093131569
:10EFD0007093141580931515909316152CEA35EC43
:10EFE00047E25EE369857A858B859C850F942B6368
:10EFF00060931715709318158093191590931A152F
:10F00000C7010E940528C7010E94D527011138C0F9
:10F0100089809A80AB80BC80A5019401C501B401B0
:10F020000F94236581112CC08092060890920708E6
:10F03000A0920808B09209082CEA35EC47E25EE39A
:10F040006D817E818F8198850F94A55B60930A08FE
:10F0500070930B0880930C0890930D082CEA35EC04
:10F0600047E25EE369857A858B859C850F942B63E7
:10F0700060930E0870930F08809310089093110806
:10F08000C7010E94D527C7010E94F527C7010E942A
:10F09000052885E0F70111928A95E9F711E001272B
:10F0A0002BE834E045E050E0B70185E894E00E94A9
:10F0B000E68F81EB93E00E9415280091260401273A
:10F0C0002BE834E040E250E0B70185E894E00E948C
:10F0D000E68FCE0183599F4F0E9415280091260488
:10F0E00001272BE834E049E050E0B70185E894E0DF
:10F0F0000E94E68F0091260401110FC08981809340
:10F1000016088A819B81AC81BD81809312089093FF
:10F110001308A0931408B093150811E001272BE8F9
:10F1200034E040E250E0B70185E894E00E94E68FC9
:10F130000091260401272BE834E040E450E0B701B9
:10F1400085E894E00E94E68F0091260401272BE8D1
:10F1500034E040E150E0B70185E894E00E94E68F9A
:10F160000091260401272BE834E040E150E0B7018C
:10F1700085E894E00E94E68FC7010E94E527009190
:10F18000260401110CC089819A81AB81BC818093D6
:10F19000270990932809A0932909B0932A0911E01F
:10F1A00001272BE834E04CE050E0B70185E894E01B
:10F1B0000E94E68F0091260401272BE834E04CE6FC
:10F1C00050E0B70185E894E00E94E68F19821A8228
:10F1D0001B821C821D821E821F82188619861A8637
:10F1E0001B861C86C7010E94D52700912604012793
:10F1F0002BE834E048E050E069EA73E085E894E009
:10F200000E94E68F0091260401272BE834E04CE0B1
:10F2100050E0B70185E894E00E94E68FCE01815866
:10F220009F4F0E94F527CE0183599F4F0E94E527EB
:10F2300080918504909186048134934069F4109202
:10F240008D0420918B0430918C04EF968EAD9FAD90
:10F25000EF972817390719F081E080938D0480918A
:10F2600026048111B2CC80918D048111AECC0E9414
:10F270007B59ABCCC7010E942528CE0183599F4FF3
:10F280000E942528C158DF4F0881CF57D040C05871
:10F29000DF4F8881C058D040089F80011124015061
:10F2A000110908F43FCECE018B589F4F0E94E527ED
:10F2B000F6CF84E690E090938604809385041092C4
:10F2C0008C0410928B040C94907581E0809326043A
:10F2D0000E9459791092260481110C9459790E9448
:10F2E0008D5A0E9436360E94CAA183E99BE00E9493
:10F2F000399280E008952F923F924F925F926F92E1
:10F300007F928F929F92AF92BF92CF92DF92EF92B5
:10F31000FF920F931F93CF93DF93CDB7DEB7C35404
:10F32000D1090FB6F894DEBF0FBECDBF4C015B0113
:10F330006A01222E19821C821C8E1F8E6115710596
:10F3400021F510E0CE014C960E943C8BCE01019637
:10F350000E943C8B812FCD5BDF4F0FB6F894DEBF50
:10F360000FBECDBFDF91CF911F910F91FF90EF9016
:10F37000DF90CF90BF90AF909F908F907F906F90D5
:10F380005F904F903F902F900895FC0183818111F1
:10F39000D8CFFA0180818F32A1F18B01CE01019685
:10F3A0007C013C0180E2382E2E019CE1490E511C6B
:10F3B0002396EFAE23972496FFAE249722963FAE76
:10F3C000229721963FAE21973FAE3EAE3DAE3CAE7A
:10F3D0003BAE3AAE39AE38AE3FAA960190E047E078
:10F3E000D9018D91882309F447C08F3209F444C0B4
:10F3F0008E3209F54A3009F4A4CF98E04AE09D0125
:10F40000EFCFFB01838182508B01823060F0618DF0
:10F41000728DCE014C960E94CA2A8E01045E1F4F47
:10F42000882309F48ECFC6016C010196F601208174
:10F430002F32D1F3B3CFEFE1F8E12491222321F071
:10F4400031968213FACF7DCF491708F47ACF8132F3
:10F4500008F477CF8F3709F474CF3FE9380F3A318A
:10F4600008F420EEE7E3F0E0EC0FFD1FE90FF11DDB
:10F47000820F80839F5FC3CF8FA9803209F461CF51
:10F480006901F90180812F5F3F4F8F32C9F38823D3
:10F4900001F121E0AE01495C5F4FB801C7010E9454
:10F4A000772C882309F44DCF0A151B0519F0C801E4
:10F4B0000E941A2B942D852D6E147F0431F0239613
:10F4C0009FAD239724968FAD24978701E92EF82EC0
:10F4D00075CF222DAE01495C5F4FB801C4010E9477
:10F4E000772C182F2FCF3F924F925F926F927F927F
:10F4F0008F929F92AF92BF92CF92DF92EF92FF9244
:10F500000F931F93CF93DF93CDB7DEB7EB970FB673
:10F51000F894DEBF0FBECDBF8091E515F12CE12C34
:10F5200083FF23C08FE196E10E94722C8BE1EFE113
:10F53000F6E1DE01919601900D928A95E1F7F12CAA
:10F54000E12CBE016F5F7F4FCE0181960F948B48F7
:10F5500018163CF4CE0101960F94CE3FE80EF11C34
:10F56000F0CFCE0181960E943C8B61E081E00E9449
:10F570007FD870909707612C470181E0881A910825
:10F580008BEEC82E83E2D82E9EE4A92E96E0B92EEB
:10F59000711014C080919607882351F180917702F1
:10F5A000882361F081E090919607911180E003E05B
:10F5B00023E042E556E0662D0E9478ED8091E51546
:10F5C00085FD5DC083FF5BC091E0791256C08091DC
:10F5D0009607813089F18091770281113AC082E0EB
:10F5E0007394639494E06912D3CF809391070CC015
:10F5F0008091900710929007882381F20E947CDA14
:10F600008091B107882351F2EB960FB6F894DEBFD4
:10F610000FBECDBFDF91CF911F910F91FF90EF9063
:10F62000DF90CF90BF90AF909F908F907F906F9022
:10F630005F904F903F9008958091900710929007AF
:10F64000882349F20E94EB238091B107882319F2A5
:10F65000DBCFDF92CF92BF92AF926F9281E0909119
:10F660009607913009F080E08F930E94BBFD0F90C8
:10F670000F900F900F900F900F9082E001C081E0EB
:10F6800090917702992309F4ABCF582E10E000E057
:10F69000852D0E151F0509F4A3CF5710A2C08FE1C9
:10F6A00096E10E94722C382C301A8BE1EFE1F6E1E2
:10F6B000DE01919601900D928A95E1F7412CBE01F1
:10F6C0006F5F7F4FCE0181960F948B4818167CF4A4
:10F6D000CE0101960F94CE3F882389F3341068C081
:10F6E000BE016F5F7F4F89EE97E00F94E93FCE0137
:10F6F00081960E943C8B8091E5159091960784FF3E
:10F7000074C0971163C0809190071092900788236E
:10F7100009F45CC019821C828091221664E076E1B3
:10F72000882311F06FE176E121E049EE57E0CE0148
:10F7300001960E947B798823E9F18BE1FE013196E5
:10F74000AFE1B6E101900D928A95E1F78091E51560
:10F750008F7D8093E515A091DA15AA3080F481E0C1
:10F760008A0F8093DA158BE18A9FD0011124A65C61
:10F77000B94EEFE1F6E101900D928A95E1F7CE01E5
:10F7800001960E943C8B1092970782E090E0A0E0E7
:10F79000B0E08093A1079093A207A093A307B09332
:10F7A000A40781E08093B10783E0809377022CCF98
:10F7B000439485CF0E94CAA169EE77E088E396E082
:10F7C0000E947DA78AE00E941192D9CF8091770292
:10F7D000882339F081E0971180E041E0662D0F9495
:10F7E0008F300F5F1F4F539453CF971559F080916F
:10F7F00077028823B1F381E090919607971180E01A
:10F8000040E0ECCF8091900710929007882379F325
:10F810008FE69AE20E94AD6A8091B107882339F39E
:10F82000F3CEEF92FF920F931F93CF93DF93CDB759
:10F83000DEB762970FB6F894DEBF0FBECDBF0E9451
:10F84000B04E882309F440C041E953E082FF02C072
:10F8500048E853E021E933E081FF02C02AE833E0C1
:10F8600080FD2FC081E993E05F934F933F932F93E7
:10F870009F938F9381E598E09F938F938E010F5F05
:10F880001F4F1F930F930F94D65A0E94CAA1C8010D
:10F890000F94EC1760E0C8010F94FD170FB6F894B1
:10F8A000DEBF0FBECDBF81E062960FB6F894DEBF1B
:10F8B0000FBECDBFDF91CF911F910F91FF90EF90C1
:10F8C00008958CE893E0D0CF80E0EECF282F909180
:10F8D000F707833021F495FD0FC094FD0FC0892FE9
:10F8E00090E0B0E0A0E004C0B695A7959795879505
:10F8F0002A95D2F78170089581E0089580E00895F7
:10F90000CF92DF92EF92FF92CF93DF93EC01CC8006
:10F91000DD80EE80FF8027E137EB41ED58EBC7013A
:10F92000B6010F94916487FD23C027E030E041E6E3
:10F9300053E4C701B6010F943F5B1816CCF0C880A2
:10F94000D980EA80FB8027E137EB41ED58EBC70116
:10F95000B6010F94916487FD0BC0C1E027E030E051
:10F9600046E653E4C701B6010F943F5B18160CF44A
:10F97000C0E08C2FDF91CF91FF90EF90DF90CF9080
:10F9800008952F923F924F925F926F927F928F9243
:10F990009F92AF92BF92CF92DF92EF92FF920F931E
:10F9A0001F93CF93DF93CDB7DEB72E970FB6F894A2
:10F9B000DEBF0FBECDBFE82ED62E042F122F282F6C
:10F9C00030E03C872B87462F50E05A87498765E017
:10F9D000F62EF29EC001F39E900D11249E878D8716
:10F9E000FA01E80FF91FEE0FFF1FEE0FFF1FEE5495
:10F9F000FC4F60817181828193819B01AC010F94E6
:10FA00002365882309F434C1E00E612F6D0DFE9C3F
:10FA1000F0011124A985BA85AE0FBF1FAA0FBB1F25
:10FA2000AA0FBB1FAE54BC4FAC901196BC9011975F
:10FA30001296CC9012971396DC90E00EFE9CA001DB
:10FA40001124A985BA85A40FB51FAA0FBB1FAA0F41
:10FA5000BB1FAE54BC4FEC901196FC9011971296C0
:10FA60000C91129713969C90862F90E0AD85BE85E1
:10FA7000A80FB91FAA0FBB1FAA0FBB1FAE54BC4FC4
:10FA80008C9011967C90119712966C901297139609
:10FA90005C90610F70E0AD85BE85A60FB71FAA0F01
:10FAA000BB1FAA0FBB1FAE54BC4F4C9011963C908D
:10FAB000119712961C91129713962C90E80FF91F2C
:10FAC000EE0FFF1FEE0FFF1FEE54FC4FB081B98306
:10FAD00021812A8332813B8383818C83FA01E60F63
:10FAE000F71FEE0FFF1FEE0FFF1FEE54FC4F90812C
:10FAF0009D83A181AE83B281BF8323812887970133
:10FB0000402F592DB701802F992D0F9423658823FD
:10FB100021F0E12CF12C00E0912C9501A601B5011A
:10FB2000C6010F942365882319F05701C02ED92CE4
:10FB3000242D332D412F522D642D732D812F922D85
:10FB40000F942365882321F0412C312C10E0212CC7
:10FB5000282D372D462D552D682D772D862D952D49
:10FB60000F942365882321F0842C732C612E522C52
:10FB70002D813E814F8158856D817E818F81988551
:10FB80000F942365882321F01D821E821F82188610
:10FB900029813A814B815C8169817A818B819C8149
:10FBA0000F942365882341F03D8139834E814A8338
:10FBB0005F815B8388858C8385E0EB85FC858E9FE8
:10FBC000D0018F9FB00D112429853A85A20FB31F54
:10FBD000AA0FBB1FAA0FBB1FAE54BC4FBA87A98781
:10FBE0009501A601B501C6010F9431629701402F1E
:10FBF000592D0F9430626B017C01282D372D462D35
:10FC0000552D682D772D862D952D0F943162242D3D
:10FC1000332D412F522D0F9430629B01AC01C7014F
:10FC2000B6010F9431626B017C0129813A814B81CD
:10FC30005C8169817A818B819C810F9431622D81F5
:10FC40003E814F8158850F9430629B01AC01C70102
:10FC5000B6010F94316220E030E040E450E40F94AC
:10FC60002B63A985BA856D937D938D939C93139790
:10FC70002E960FB6F894DEBF0FBECDBFDF91CF91A9
:10FC80001F910F91FF90EF90DF90CF90BF90AF90BA
:10FC90009F908F907F906F905F904F903F902F90AC
:10FCA0000895129A0895269A2E9A0895CF92DF9277
:10FCB000EF92FF920F931F93CF9390915B0291303D
:10FCC00009F461C0662351F01092940510929005DA
:10FCD000109291051092920510929305C82F0F94DF
:10FCE0003D37C0909005D0909105E0909205F0903E
:10FCF00093059B01AC012C193D094E095F0969016F
:10FD00007A01F7FC40C020919405C7FD15C04C2F27
:10FD10000C2E000C550B4C5F5F4FE22F022E000C97
:10FD2000FF0B4E175F077CF144EFC42EDD24D39404
:10FD3000E12CF12C2C1734F438EEC32E33E0D32E03
:10FD4000E12CF12CC60ED71EE81EF91EC0929005BC
:10FD5000D0929105E0929205F0929305022F0170E6
:10FD600010E084E2809FB001819F700D701B112410
:10FD700060597C4F82E390E00E9435698091940540
:10FD80008F5F80939405CF911F910F91FF90EF901B
:10FD9000DF90CF90089580935A028032B8F5909109
:10FDA0004806891724F091E0980F909348064091F7
:10FDB0004406509145066091460670914706082E0C
:10FDC00004C076956795579547950A94D2F7417088
:10FDD0004093F40F87FD1DC0282F082E000C330B15
:10FDE0003F938F938CE29CE19F938F938CE39CE1F4
:10FDF0009F938F931F920E94B5DA8DB79EB7079697
:10FE00000FB6F8949EBF0FBE8DBF08951092F40FE9
:10FE1000E1CF0D941D2E2F923F924F925F926F92E1
:10FE20007F928F929F92AF92BF92CF92DF92EF928A
:10FE3000FF921F93CF93DF93CDB7DEB72C970FB60A
:10FE4000F894DEBF0FBECDBF7A011901DC012D9100
:10FE50003D914D915C912D833E834F835887FB01EB
:10FE600040805180628073808090ED089090EE0811
:10FE7000A090EF08B090F008A50194016D817E81FB
:10FE80008F8198850F943F5B81110EC011E0A30113
:10FE900092016091F1087091F2088091F3089091BD
:10FEA000F4080F943F5B811110E0D1012D913D9139
:10FEB0004D915C9129873A874B875C87F701C08019
:10FEC000D180E280F3802091460230914702409138
:10FED000480250914902C701B6010F943F5B882345
:10FEE00009F44EC0C0924602D0924702E092480206
:10FEF000F09249028091F9089091FA08A091FB08CC
:10FF0000B091FC084091F1085091F2086091F3081B
:10FF10007091F4088092C1079092C207A092C30723
:10FF2000B092C4074093C5075093C6076093C707B4
:10FF30007093C807C092C907D092CA07E092CB0756
:10FF4000F092CC078093CD079093CE07A093CF0774
:10FF5000B093D00720E030E040E05FE360912210F2
:10FF60007091231080912410909125100F94A55B1F
:10FF700069837A838B839C83CE0101960E94C45847
:10FF80002D813E814F8158852093C1073093C20750
:10FF90004093C3075093C4074092C5075092C607C9
:10FFA0006092C7077092C807D1012D913D914D9184
:10FFB0005C916091CD077091CE078091CF079091B1
:10FFC000D0070F9431626093CD077093CE07809372
:10FFD000CF079093D00711112FC020E030E0A90186
:10FFE00069857A858B859C850F943F5B811133C031
:10FFF00060E070E088EC92E469837A838B839C8371
:020000021000EC
:10000000CE0101960E94C4582C960FB6F894DEBF1C
:100010000FBECDBFDF91CF911F91FF90EF90DF908A
:10002000CF90BF90AF909F908F907F906F905F9098
:100030004F903F902F9008952AEF3EE74AE25FE30A
:1000400060912610709127108091281090912910AE
:100050000F94A55BD1CF60E070E080EA91E4CCCF53
:10006000CF93DF9300D01F92CDB7DEB780E090E052
:10007000A0EAB0E489839A83AB83BC8361E0CE01BC
:1000800001960E94CE500F900F900F900F90DF912D
:10009000CF9108958091B6059091B705009731F002
:1000A0004AE050E070E060E00D945A5960E070E082
:1000B000CB0108958091010982FF0BC063E68AE6B7
:1000C0009DE10E94D0DA0F9483370E9458DE81E0D0
:1000D000089580E008958091B6059091B705009746
:1000E00031F04AE050E070E060E00D942C5860E0A0
:1000F00070E0CB0108950E946B8097FD0CC00E94B8
:100100006B806F3F71058105910509F034F40E9401
:100110006B80862F089580E008958FEF0895CF9229
:10012000DF92EF92FF920F931F93CF93DF936B01B8
:100130007A01EC01CE5BDA4F28813CE0389F8001E8
:10014000399F100D112427FF24C0FB01118210825A
:1001500088818F5F888388819801280F311D87FDF2
:100160003A95C90120917515F6012817190629F04D
:1001700024F088818C300CF43CC0808191810496FD
:1001800080349C4908F475C0F60180819181049601
:1001900072C088819801280F311D87FD3A95C901E9
:1001A000209175152817190699F294F28881A801F3
:1001B000480F511D87FD5A95FA01EE0FFF1FE40FFE
:1001C000F51FE35DFA4E808187FFC2CF8881F80179
:1001D000E80FF11D87FDFA95CF01EE0FFF1FE80F25
:1001E000F91FE35DFA4E808160E08F770F9431351F
:1001F000AFCF808191812881A801420F511D27FD39
:100200005A959A01FA01EE0FFF1FE20FF31FE35D0B
:10021000FA4E21813281820F931FF70191838083EF
:1002200088819801280F311D87FD3A95F901EE0F5D
:10023000FF1FE20FF31FE35DFA4E808187FF20C0AE
:100240008881080F111D87FD1A95F801EE0FFF1F19
:10025000E00FF11FE35DFA4E808161E08F77DF915F
:10026000CF911F910F91FF90EF90DF90CF900D9461
:10027000313580E49CE9F701918380838FEF888397
:10028000DF91CF911F910F91FF90EF90DF90CF9072
:100290000895FC01659175918591949108958091DF
:1002A000D207882319F080E00E94255C80E0089541
:1002B0004F925F926F927F928F929F92AF92BF9276
:1002C000CF92DF92EF92FF92CF93DF9300D000D0D6
:1002D0001F921F92CDB7DEB75C01DB01CD90DD90A0
:1002E000ED90FC90E0918515F0918615FE83ED83ED
:1002F00084819581A681B78189839A83AB83BC83EE
:100300009C01AD01C701B6010F9430622B013C0185
:10031000F50180809180A280B380AD81BE818D91F6
:100320009D910D90BC91A02D8D839E83AF83B88746
:1003300027E137EB41ED58EBC301B2010F94916413
:1003400087FDD0C027E030E041E653E4C301B201AD
:100350000F943F5B18160CF4C5C02D813E814F8170
:100360005885C501B4010F9430622B013C0127E18F
:1003700037EB41ED58EB0F94916487FDB3C027E054
:1003800030E046E653E4C301B2010F943F5B181618
:100390000CF4A8C020E030E0A9016D817E818F813E
:1003A00098850F9431622B013C0120E030E040E45D
:1003B00050E40F943F5B87FF05C0412C512C30E483
:1003C000632E762C27E137EB41ED58E3C301B201F0
:1003D0000F9430629B01AC01C501B4010F9491648C
:1003E00087FD80C020E030E046E653E46D817E81E9
:1003F0008F8198850F9431622B013C0120E030E021
:1004000049E553E40F949164181634F4412C512CAF
:1004100029E5622E23E4722E27E137EB41ED58E304
:10042000C301B2010F9431629B01AC01C501B4015B
:100430000F943F5B18160CF455C020E030E0A90182
:1004400069817A818B819C810F9431624B015C01BF
:1004500020E030E040E951E40F943F5B87FF06C0A5
:10046000812C912C90E9A92E91E4B92E27E137EB4C
:1004700041ED58E3C501B4010F9430629B01AC011A
:10048000C701B6010F94916487FD2CC020E030E0D5
:1004900041E653E469817A818B819C810F943162BA
:1004A0004B015C0120E030E04AE453E40F94916496
:1004B000181634F4812C912C8AE4A82E83E4B82EEB
:1004C00027E137EB41ED58E3C501B4010F943162E8
:1004D0009B01AC01B1E0B983C701B6010F943F5B4A
:1004E00018160CF41982898128960FB6F894DEBF8D
:1004F0000FBECDBFDF91CF91FF90EF90DF90CF90F7
:10050000BF90AF909F908F907F906F905F904F9033
:1005100008958F929F92AF92BF92CF92DF92EF9207
:10052000FF92CF93DF93EC018090F8079090F9074A
:10053000A090FA07B090FB0720E030E0A901C501C8
:10054000B4010F943F5B882309F452C0C880D9805E
:10055000EA80FB80A7019601C501B4010F943F5BBF
:1005600018160CF04AC02091B2053091B3054091A5
:10057000B4055091B505C701B6010F943F5B8823C0
:1005800021F1C092B205D092B305E092B405F09289
:10059000B5052091AE053091AF054091B005509161
:1005A000B105C701B6010F94A55B9B01AC0160E0EA
:1005B00070E080E89FE30F94306260934A0270938A
:1005C0004B0280934C0290934D0260914A027091CD
:1005D0004B0280914C0290914D02DF91CF91FF90A0
:1005E000EF90DF90CF90BF90AF909F908F90089545
:1005F00060E070E080E89FE3F0CF60E070E0CB0166
:10060000ECCF9B01AC01485F5F4FBC016C5F7F4F3B
:100610000C940B7F0F931F93CF93DF9300D000D0E8
:100620001F921F92CDB7DEB7FC018B0183A581110C
:1006300012C081E083A784819581A681B781B058DB
:1006400089839A83AB83BC83BE016F5F7F4F81EC4C
:1006500097E00E9401831D821E821F82188620E07F
:1006600030E040E05FE36091F5087091F60880911A
:10067000F7089091F8080F94316269837A838B832D
:100680009C839E012B5F3F4FAE014F5F5F4F61EF39
:1006900078E08DEE98E00E940B7F1D821E821F8203
:1006A000188620E030E040E05FE3F8016085718566
:1006B000828593850F94316269837A838B839C83CF
:1006C000B8016C5F7F4F9E012B5F3F4FAE014F5FC4
:1006D0005F4FC8010E940B7F28960FB6F894DEBFCB
:1006E0000FBECDBFDF91CF911F910F9108952F9233
:1006F0003F924F925F926F927F928F929F92AF92B2
:10070000BF92CF92DF92EF92FF920F931F93CF93FE
:10071000DF93CDB7DEB7A2970FB6F894DEBF0FBE5A
:10072000CDBF8C011B015E834D834090ED0850903E
:10073000EE086090EF087090F0088090F1089090BB
:10074000F208A090F308B090F408DB018D919D9120
:100750000D90BC91A02D8F87988BA98BBA8B9C0193
:10076000AD01C301B2010F9430626B017C01D10174
:1007700014968D919D910D90BC91A02D8B8B9C8B8F
:10078000AD8BBE8B9C01AD01C501B4010F943062ED
:100790006F8B788F898F9A8FAD81BE818D919D915E
:1007A0000D90BC91A02D8F839887A987BA879C0153
:1007B000AD01C301B2010F9430626B8F7C8F8D8FBE
:1007C0009E8FAD81BE8114968D919D910D90BC91AF
:1007D000A02D8B879C87AD87BE879C01AD01C5018D
:1007E000B4010F9430626F8F78A389A39AA3A701F5
:1007F0009601C701B6010F94A55B6B017C012F899F
:10080000388D498D5A8DCA01B9010F94A55B9B01A2
:10081000AC01C701B6010F9431624B015C012F8519
:10082000388949895A896F81788589859A850F9495
:1008300030622B013C012B893C894D895E896B8597
:100840007C858D859E850F9430626B017C01A301B0
:100850009201C301B2010F94A55B2B013C01A701DA
:100860009601C701B6010F94A55B9B01AC01C301C2
:10087000B2010F9431620F94DF646B017C012B8D08
:100880003C8D4D8D5E8DCA01B9010F94A55B2B0186
:100890003C012F8D38A149A15AA1CA01B9010F9479
:1008A000A55B9B01AC01C301B2010F9431629B01B6
:1008B000AC01C501B4010F9491641816B4F520E0A1
:1008C00030E0A901C701B6010F94916487FF2AC0E7
:1008D000C701B601905820E030E040EA50E40F94A0
:1008E0009164181614F5A1016D817E81C8010E94E2
:1008F0007783A2960FB6F894DEBF0FBECDBFDF910F
:10090000CF911F910F91FF90EF90DF90CF90BF900C
:10091000AF909F908F907F906F905F904F903F909F
:100920002F900895C701B601D6CF20E030E040E017
:1009300050E4C501B4010F949164181624F4B10178
:10094000C8010E940A8319821A821B821C82BE017E
:100950006F5F7F4FC1010E9401832DEC3CEC4CEC9A
:100960005CE3C701B6010F94A55B9B01AC01F801E4
:1009700060817181828193810F94A55B69837A8301
:100980008B839C83C8010F946230BE016F5F7F4FE1
:100990008D819E810E940183ACCF3F924F925F92E6
:1009A0006F927F928F929F92AF92BF92CF92DF927F
:1009B000EF92FF920F931F93CF93DF93CDB7DEB7E4
:1009C0006C970FB6F894DEBF0FBECDBFDB010C9164
:1009D000142F100F153008F067C11196DC90C22E4D
:1009E000CD0CB4E0BC1508F45FC1ED2DF0E0EB5583
:1009F000FA4F8080912CB12CA12C002E04C0B6940B
:100A0000A794979487940A94D2F780FE4DC1EC2D59
:100A1000F0E0EB55FA4F8080912CB12CA12C012EE7
:100A200004C0B694A794979487940A94D2F780FE52
:100A30003BC1322E642F7C01409016045090170465
:100A4000609018047090190480911E0490911F0406
:100A5000A0912004B0912104898F9A8FAB8FBC8F15
:100A6000660F770B072E000C880B990B0F94465BD3
:100A70004B015C01602F000F770B880B990B0F94D3
:100A8000465B298D3A8D4B8D5C8D0F94A55BA30140
:100A900092010F943162A50194010F9431626D8728
:100AA0007E878F87988B612F110F770B880B990B9F
:100AB0000F94465B298D3A8D4B8D5C8D0F94A55B11
:100AC000A30192010F943162A50194010F94306249
:100AD00069837A838B839C8340901A0450901B0413
:100AE00060901C0470901D04809122049091230456
:100AF000A0912404B0912504898F9A8FAB8FBC8F6D
:100B0000632D660F770B072E000C880B990B0F9443
:100B1000465B4B015C016D2DDD0C770B880B990B4F
:100B20000F94465B298D3A8D4B8D5C8D0F94A55BA0
:100B3000A30192010F943162A50194010F943162D7
:100B4000698B7A8B8B8B9C8B6C2DCC0C770B880BE9
:100B5000990B0F94465B298D3A8D4B8D5C8D0F94CC
:100B6000A55BA30192010F943162A50194010F943A
:100B700030626D837E838F839887F70180859185AE
:100B8000A285B38589879A87AB87BC878D8B9E8B1F
:100B9000AF8BB88F40EE50E061E070E0CE0141963F
:100BA0000E948A3340EE50E061E070E0CE0105968D
:100BB0000E948A3345EE50E061E070E0CE010D9670
:100BC0000E948A3345EE50E061E070E0CE0101966C
:100BD0000E948A3389889A88AB88BC8827E137EBE2
:100BE00041ED58EBC501B4010F94916487FD5CC0E1
:100BF00027E030E041E653E4C501B4010F943F5BC8
:100C000018160CF451C08D849E84AF84B88827E1F7
:100C100037EB41ED58EBC501B4010F94916487FDAA
:100C200043C027E030E046E653E4C501B4010F9429
:100C30003F5B1816CCF18D809E80AF80B88427E191
:100C400037EB41ED58EBC501B4010F94916487FD7A
:100C50002BC027E030E041E653E4C501B4010F9416
:100C60003F5B18160CF189809A80AB80BC8027E12D
:100C700037EB41ED58EBC501B4010F94916487FD4A
:100C800013C027E030E046E653E4C501B4010F94F9
:100C90003F5B18164CF0AE014F5F5F4FBE01635FC4
:100CA0007F4FC7010E9477836C960FB6F894DEBF22
:100CB0000FBECDBFDF91CF911F910F91FF90EF90AD
:100CC000DF90CF90BF90AF909F908F907F906F906C
:100CD0005F904F903F9008958C38910514F08CE808
:100CE00090E090930408809303080C942A24809148
:100CF000B6059091B705892B41F00E947B8091E069
:100D0000811101C090E0892F089591E0FCCF0E94ED
:100D10006B80CB0108950F931F93CF938091B605FD
:100D20009091B7050097E9F0FC018F01C1912C2F3C
:100D30002F7D81F0C53411F0C536B9F7F801108266
:100D400070E060E00F94CE56F801C083CF911F9100
:100D50000F91089570E060E0CF911F910F910D9475
:100D6000CE5660E070E0CB01F1CF2FEB280F2A3197
:100D700008F047C0E22FF0E08091E5059091E6058C
:100D8000A091E705B091E80504C0B695A7959795A1
:100D900087952A95D2F780FD02C081700895E953A6
:100DA000FA4FE081EE2341F18091DF079091E00757
:100DB000E80FF92FF11D808190ED980F9A3030F0F7
:100DC0008E3251F4818180538A3098F4F093B705C4
:100DD000E093B60581E008958D3211F08B3249F42D
:100DE000818190ED980F9A3088F38E3211F48281D0
:100DF000EACFF0E0E0E0EACF1092B7051092B60536
:100E0000E9CF80E008950E94B586882341F081E013
:100E10002091B6053091B705232B09F480E00895A1
:100E2000CF93DF93EB010E940387882319F00E9480
:100E30006B80EB01CE01DF91CF91089583E50E9495
:100E400003878823E9F00F943D376093D3077093AD
:100E5000D4078093D5079093D6070E948B8620E015
:100E600030E04AE754E40F94A55B0F94A4636093C9
:100E70004E0270934F028093500290935102089556
:100E80008091E50584FD0AC08091E70587FD06C0D5
:100E90008091E805837011F40C945E3A0E944D3AFB
:100EA00088E50E94B586882331F05F9A8091D1074A
:100EB0008E7F8093D10789E50E94B586882331F023
:100EC0008A9A8091D1078D7F8093D1078AE50E940D
:100ED000B586882359F080910801809581708093B0
:100EE00006018091D1078B7F8093D10785E40E9412
:100EF000B58681110C94517E0895CF93C62F0E9420
:100F00000387882319F0CF910C947B808C2FCF918D
:100F10000895CF92DF92EF92FF926A017B010E94C7
:100F20000387882331F0FF90EF90DF90CF900C94EF
:100F30008B86C701B601FF90EF90DF90CF900895A8
:100F40004F925F926F927F928F929F92AF92BF92D9
:100F5000CF92DF92EF92FF921F93CF93DF9300D057
:100F60001F92CDB7DEB719821A821B821C82CE0176
:100F700001964C018DEEC82E88E0D82E91ECE92E1A
:100F800097E0F92E21EEA22E28E0B22E10E088E59F
:100F9000810F0E940387F40181934F01882341F060
:100FA0000E948B862B013C018091F40F882359F01D
:100FB000F60180819181A281B381F70180839183C1
:100FC000A283B38314C0812F0E94667C882309F416
:100FD000D0C0F6012081318142815381C301B20129
:100FE0000F943162F70160837183828393831F5F63
:100FF000F4E0CF0ED11C84E0E80EF11C94E0A90EC1
:10100000B11C133021F685E40E9403878C8388236A
:1010100009F4B9C00E948B866B017C0183E00E94B9
:10102000667C882371F02091F9083091FA0840918C
:10103000FB085091FC08C701B6010F9431626B01A7
:101040007C01C092CD07D092CE07E092CF07F092FC
:10105000D0078091B103882359F18091E51582FF73
:1010600027C08C81882321F18981811103C08A8165
:101070008823F1F02DEC3CEC4CE45DE36091380802
:101080007091390880913A0890913B080F94316231
:101090009B01AC016091F5087091F6088091F7080A
:1010A0009091F8080F949164181614F40F94D84690
:1010B00040E050E0BA0186E40E94898720E030E0F9
:1010C000A9010F949164181684F40E948B8620E085
:1010D00030E040E752E40F942B6360937302709307
:1010E000740280937502909376028091F50F83FDD0
:1010F0002CC08091F40F811128C080912B07882388
:1011000021F12091F9083091FA084091FB085091A3
:10111000FC086091CD077091CE078091CF07909128
:10112000D0070F94306220913807309139074091F1
:101130003A0750913B070F943162609338077093E0
:10114000390780933A0790933B070F900F900F90C9
:101150000F90DF91CF911F91FF90EF90DF90CF9094
:10116000BF90AF909F908F907F906F905F904F90C7
:101170000895F5012081318142815381C301B2017B
:101180000F9430622FCF8091F9089091FA08A091C6
:10119000FB08B091FC088093CD079093CE07A093F5
:1011A000CF07B093D00755CFCF93DF93EB010E94C9
:1011B0000387882321F0DF91CF910C948786CE019D
:1011C000DF91CF910895CF93DF93C82FD62F0E9440
:1011D0000387882321F0DF91CF910C9477868C2FA1
:1011E0000E94B586811101C08D2FDF91CF910895A6
:1011F000EFE2F8E082EBDF011D928A95E9F70895AE
:101200008091B103811104C00E94F8880D94DC49DB
:101210008091E51582FD0D94D846089580912F08A0
:10122000882361F09091E008891308C08091E5154A
:1012300083FF04C08DE698E00D94E74980E00895AF
:101240004F925F926F927F928F929F92AF92BF92D6
:10125000CF92DF92EF92FF920F931F93CF93DF9382
:10126000CDB7DEB7C059D1090FB6F894DEBF0FBEB7
:10127000CDBF0E940E89882369F083E50E94B58660
:10128000882301F120E040E070E060E08CE292E031
:101290000E94D7D8C057DF4F0FB6F894DEBF0FBEFD
:1012A000CDBFDF91CF911F910F91FF90EF90DF9015
:1012B000CF90BF90AF909F908F907F906F905F90F6
:1012C0004F90089583E40E94B586882319F00E9408
:1012D000CAD9E0CF8090D6089090D708A090D808BF
:1012E000B090D9088091DF0880FF05C09091F50F7C
:1012F00098609093F50F86958170809341098BE2F9
:1013000093E20F94611880916508909166089E01A0
:101310002F5F3F4F7901009799F09F938F9382E25F
:1013200093E29F938F933F932F930F94D65AC701C5
:101330000F9433180F900F900F900F900F900F9005
:101340008091630890916408009799F09F938F9320
:1013500089E193E29F938F93FF92EF920F94D65A75
:10136000C7010F9433180F900F900F900F900F90AC
:101370000F906E0131E8C30ED11C6091420870914C
:1013800043088091440890914508860123E041E09C
:101390000F940C569F938F9387E093E29F938F93C4
:1013A000FF92EF920F94D65AC7010F9433188FEF24
:1013B00092E20F94611887E08093D10780939C0399
:1013C0000F900F900F900F900F900F9080915E08EC
:1013D0008823F9F060915F0870916008809161083E
:1013E0009091620823E041E00F940C569F938F93F5
:1013F00086EF92E29F938F93FF92EF920F94D65ACB
:10140000C7010F9433180F900F900F900F900F900B
:101410000F90809167088823A1F01F928F931F92ED
:101420001F9289EE92E29F938F93FF92EF920F9417
:10143000D65AC7010F9433180FB6F894DEBF0FBE0B
:10144000CDBF809168088823A9F01F928F931F92C7
:1014500081E08F9389EE92E29F938F93FF92EF92B8
:101460000F94D65AC7010F9433180FB6F894DEBF05
:101470000FBECDBF4090690850906A0860906B081D
:1014800070906C0820E030E0A901C301B2010F9414
:101490003F5B811104C08091DF0882FF20C086017C
:1014A00021E041E0C301B2010F940C569F938F934A
:1014B0008091DF0882FB882780F91F928F938CED43
:1014C00092E29F938F93FF92EF920F94D65AC701A7
:1014D0000F9433180FB6F894DEBF0FBECDBF6091E6
:1014E00034087091350880913608909137088E0144
:1014F0000F581F4F23E041E00F940C56782E692EB1
:1015000060913008709131088091320890913308D1
:10151000860123E041E00F940C566F927F929F93D7
:101520008F938BEC92E29F938F93FF92EF920F94A5
:10153000D65AC7010F943318609138087091390852
:1015400080913A0890913B0823E041E00F940C56BB
:1015500080EC92E20F946118DF92CF9286EB92E2D8
:101560009F938F93FF92EF920F94D65AC7010F94D7
:101570003318809141088F93809140088F938FEAB0
:1015800092E29F938F93FF92EF920F94D65AC701E6
:101590000F94331860913C0870913D0880913E088B
:1015A00090913F0823E041E00F940C569F938F9356
:1015B00085EA92E29F938F93FF92EF920F94D65A0F
:1015C000C7010F9433188CE0E6E4F8E0A3E2B8E03A
:1015D00001900D928A95E1F78CE0E2E5F8E0A7E151
:1015E000B8E001900D928A95E1F780E00E94904E5C
:1015F00081E00E94904E82E00E94904E8091DE0831
:101600008093F70781E08093B1030E9400898DE603
:1016100098E09F938F938FE09DE39F938F93FF922A
:10162000EF920F94D65A0FB6F894DEBF0FBECDBF1F
:10163000C7010F9433188091DD088F938091DC08E7
:101640008F938091DB088F938091DA088F93BF92FC
:10165000AF929F928F9287E992E29F938F93FF922E
:10166000EF920F94D65AC7010F9433180FB6F8941F
:10167000DEBF0FBECDBF0ECEFC01238121110C9425
:101680001A2B08950F931F9301E010E020E030E043
:10169000082E04C0000F111F221F331F0A94D2F717
:1016A0004091440650914506609146067091470668
:1016B000402B512B622B732B4093440650934506CD
:1016C000609346067093470690915A02891303C0AF
:1016D00081E08093F40F1F910F9108954F925F92D4
:1016E0006F927F928F929F92AF92BF92CF92DF9232
:1016F000EF92FF920F931F93CF93DF93EC01209112
:10170000160430911704409118045091190468810F
:1017100079818A819B810F9430626B017C012091D9
:101720001A0430911B0440911C0450911D046C81DB
:101730007D818E819F810F9430624B015C01A701F6
:10174000960160913E0270913F028091400290911B
:1017500041020F943F5B882309F450C0C0923E02BF
:10176000D0923F02E0924002F0924102209188051F
:101770003091890540918A0550918B05C701B601CA
:101780000F94A55B2B013C010F94D3636B017C018B
:1017900020E030E0A9010F943F5B87FD70C020E09E
:1017A00030E040E450E4C701B6010F94916418168C
:1017B0002CF4C12CD12CC0E4EC2EFE2CA7019601F8
:1017C000C301B2010F94306260938005709381056C
:1017D0008093820590938305C701B6010F949D63A2
:1017E00060937E05062E000C770B6F5F7F4F643091
:1017F000710514F064E070E060937C05D0913C02C8
:1018000010917E05A50194016091420270914302FE
:1018100080914402909145020F943F5B811133C047
:10182000D11381C020916405309165054091660512
:1018300050916705609180057091810580918205C6
:10184000909183050F94A55B2091680530916905FF
:1018500040916A0550916B050F943162DF91CF91F1
:101860001F910F91FF90EF90DF90CF90BF90AF90BE
:101870009F908F907F906F905F904F900895C12CB4
:10188000D12C76019BCF8092420290924302A0928B
:101890004402B092450220918C0530918D05409113
:1018A0008E0550918F05C501B4010F94A55B4B01C6
:1018B0005C010F94D3636B017C0120E030E0A9014F
:1018C0000F943F5B87FDF3C020E030E040E450E43C
:1018D000C701B6010F94916418162CF4C12CD12CB9
:1018E000B0E4EB2EFE2CA7019601C501B4010F94C4
:1018F000306260938405709385058093860590938C
:101900008705C701B6010F949D6360937F05062E7E
:10191000000C770B6F5F7F4F6430710514F064E04B
:1019200070E060937D05C0917F05D11305C0809163
:101930003D028C1709F470C080917E0590917F055F
:1019400090933D0280933C020C2E000CDD0B25E0B1
:101950001203C0011124FC01EC0FFD1FEE0FFF1F4D
:10196000EE0FFF1FEE54FC4F2081318142815381E5
:10197000209378053093790540937A0550937B0541
:1019800000917D05002E000C110BFC01E00FF11FF2
:10199000EE0FFF1FEE0FFF1FEE54FC4F60817181B1
:1019A000828193810F943062609374057093750502
:1019B000809376059093770520917C0535E023038D
:1019C000F0011124CE0FDF1FCC0FDD1FCC0FDD1F68
:1019D000CE54DC4F288139814A815B812093700588
:1019E000309371054093720550937305E00FF11F1A
:1019F000EE0FFF1FEE0FFF1FEE54FC4F6081718151
:101A0000828193810F94306260936C0570936D05B1
:101A100080936E0590936F05809084059090850566
:101A2000A0908605B09087052091740530917505CA
:101A30004091760550917705C501B4010F94A55BDF
:101A4000209178053091790540917A0550917B0578
:101A50000F9431626B017C01C0926805D0926905D8
:101A6000E0926A05F0926B0520916C0530916D054E
:101A700040916E0550916F05C501B4010F94A55BAF
:101A80002091700530917105409172055091730558
:101A90000F943162A70196010F9430626093640540
:101AA000709365058093660590936705BBCEC12C46
:101AB000D12C760118CF1F93CF93DF93CDB7DEB72C
:101AC0002C970FB6F894DEBF0FBECDBF182F88231A
:101AD00079F020E030E0A90160911E0470911F04AC
:101AE00080912004909121040F943F5B8823F9F0AA
:101AF0008091FC078117D9F00E944D3A8CE0E7ED08
:101B0000F2E0DE01119601900D928A95E1F7CE0187
:101B100001960E946E8B8091FC07882391F08DEED8
:101B200098E00E94703A1092FC070E94D3512C96C4
:101B30000FB6F894DEBF0FBECDBFDF91CF911F91DE
:101B4000089581E08093FC078DEE98E00E949D3916
:101B5000ECCF80E00E945B8D10921A0410921B045F
:101B600010921C0410921D04109216041092170477
:101B70001092180410921904109222041092230457
:101B8000109224041092250410921E0410921F0437
:101B90001092200410922104E2EBF3E026E134E0FD
:101BA00080E090E0A0ECBFE780839183A283B383C1
:101BB00084839583A683B78380879187A287B38721
:101BC00084879587A687B787808B918BA28BB38BF1
:101BD00074962E173F0741F708954F925F926F92C8
:101BE0007F928F929F92AF92BF92CF92DF92EF92AD
:101BF000FF921F93CF93DF93EC01162F2091F807EC
:101C00003091F9074091FA075091FB07688179817B
